:1030000081EF18F0FFFFFFFF13391339133913391C
:10301000400C1339400C1339133913391339133950
:1030200013391339133913391339400C400C400C40
:103030001339133913391339133913391339133930
:1030400076361339133913391237023713391339D6
:10305000400C400C13391339133913391339400C10
:103060001339133913391339133913391339133900
:1030700013391339133913391339133913391339F0
:10308000400C1339133913391339133913391339E0
:1030900013391339133913391339133913391339D0
:1030A000400C1339400C400C1339133913391339C0
:1030B00013391339133913391339133913391339B0
:1030C00013391339133913391339133913391339A0
:1030D0001339133913391339133913391339133990
:1030E0001339133913391339400C13391339133980
:1030F000400C400C400C400C133913391339133970
:10310000FF00C9EF5FF0007EE3C8DE26E26CBB6C17
:10311000CB0ACF2ECA28E338E434E44AE0B4E3BC57
:10312000E31AE3ACE30CE354D43AD2FCE20D0A2DEB
:10313000204F627365727665204C45447320756E2E
:103140006465722053465020636167652E20546881
:1031500065792073686F756C6420626520746F6791
:10316000676C696E6720666F72203130207365630B
:103170006F6E64732E0A0D4966207468657920614C
:103180007265206E6F7420746F67676C696E672C50
:103190002073656520746573742070726F63656455
:1031A00075726520666F72206D6F726520696E663C
:1031B0006F000D0A0A2D2D2D205465737420313AAD
:1031C0002055392E53444F202D2D3E205344492E57
:1031D0005531302E44444F202D2D3E204444492E5D
:1031E0005531312E53444F202D2D3E205344492E2E
:1031F000553132000D0A2D20436865636B696E6797
:1032000020492F4F20285350495F6E4353202D3EB5
:10321000205350495F534C4156455F524459292031
:103220003D200050524253204572726F7220436815
:1032300065636B20436F6D706C65746564202D2031
:103240004572726F7220636F756E74203D20000DA1
:103250000A2D20436865636B696E6720492F4F20F4
:10326000285245534554202D3E205350495F534426
:103270003029203D20000D0A0A2D2D2D2054657384
:103280007420343A205531322E53444F202D2D3E98
:10329000205344492E553131000D0A0A2D2D2D2081
:1032A0005465737420333A205531312E44444F20F5
:1032B0002D2D3E204444492E553132000D0A0A2D51
:1032C0002D2D205465737420353A2055392E4444F1
:1032D0004F202D2D3E204444492E553130000D0AFB
:1032E0000A2D2D2D205465737420363A2055392E21
:1032F00053444F202D2D3E205344492E553130004C
:103300000D0A0A2D2D2D205465737420323A205554
:1033100031322E44444F202D2D3E204444492E5519
:1033200039000A0D204D6178205265636F72646523
:10333000642054656D703A202564646567430A0D06
:10334000000D0A0A2D2D2D20505242532054455372
:103350005420434F4D504C45544521202D2D2D00D8
:103360002061732044444F206F75742050524253A3
:103370002067656E657261746F72202D2000206178
:10338000732053444F206F7574205052425320676E
:10339000656E657261746F72202D20000A0D0953ED
:1033A000657269616C204E756D626572204368615B
:1033B0006E6765640A0D000A0D0950415353574F5B
:1033C000524420494E434F52524543540D0A3E2029
:1033D000003278334720456E636170202B203278AD
:1033E00033472044656361702020000D0A2D094396
:1033F0006831206173205052425320636865636BCB
:1034000065723D20000D0A2D09436832206173204A
:103410005052425320636865636B65723D20000D16
:103420000A2D0943683320617320505242532063B0
:103430006865636B65723D20000D0A2D0943683491
:10344000206173205052425320636865636B65723C
:103450003D2000517561642033472D534449204479
:103460006563617073756C61746F72200051756172
:10347000642033472D53444920456E636170737552
:103480006C61746F722000317831324720456E6371
:103490006170202B203178313247204465636170A0
:1034A000004475616C203132472D534449204465F6
:1034B00063617073756C61746F72004475616C2028
:1034C0003132472D53444920456E63617073756CEA
:1034D00061746F72000A0D0950415353574F5244A3
:1034E0002041434345505445440D0A3E2000517548
:1034F00061642033472D53444920446563617073F0
:10350000756C61746F7200517561642033472D537F
:10351000444920456E63617073756C61746F72000D
:103520000D0A2D20424F4F544C4F414445522056D6
:10353000455253494F4E3A20000A0D09454E544515
:10354000522053455249414C204E554D4245523A26
:10355000003278334720456E636170202B2032782B
:103560003347204465636170000D0A2D204649529F
:103570004D574152452056455253494F4E3A20002F
:103580000D0A2D20475331327878782053746174B6
:1035900075733A20000D0A2D2053776974636820F3
:1035A000506F7328312D38293D000D0A0A2D2D2D1D
:1035B0002031324720505242532054455354000A80
:1035C0000D09454E5445522050415353574F5244D4
:1035D0003A20000D0A0A2D2D2D2048442050524239
:1035E000532054455354000A0D20546F74616C20CD
:1035F00052756E3A2025646420000D0A2D2D2D2071
:10360000434F4D504C455445202D2D2D000D0A2D76
:1036100020506F776572205374617475733A000D92
:103620000A0945514344322028553130293A2000B7
:103630000D0A0945514344322028553131293A2099
:10364000000D0A0945514344342028553132293AA6
:1036500020006661696C202D207472792061676199
:10366000696E000D0A094551434431202855392916
:103670003A20000D0A2D20556E697420547970652A
:103680003A200042433838302D3243482D315431EE
:103690005200424E3838302D3243482D3154315289
:1036A0000042433838302D3443482D3254325200D2
:1036B000424E3838302D3443482D32543252000DAA
:1036C0000A2D2041505020747970653A20000D0A6F
:1036D0002D20534650205374617475730042433853
:1036E00038302D4D495353494E4700424E383830FB
:1036F0002D4D495353494E47000D0A2D2045455045
:10370000524F4D203D200042433838302D3243483F
:103710002D325200424E3838302D3243482D32522D
:103720000042433838302D3443482D345200424E45
:103730003838302D3443482D345200424338383025
:103740002D3243482D325400424E3838302D32430A
:10375000482D32540042433838302D3443482D34FC
:103760005400424E3838302D3443482D3454000D27
:103770000A095346502031203D20000D0A095346C6
:10378000502032203D20000D0A09325635203D20C0
:10379000000D0A09315638203D20000D0A09564413
:1037A00044203D20000A0D535731206F6666000A01
:1037B0000D535732206F6666000A0D535733206F42
:1037C0006666000A0D535734206F6666000A0D5373
:1037D0005735206F6666000A0D535736206F6666B0
:1037E0000055702D31304720200055702D3235475F
:1037F0002020004552524F52203221004D49535350
:10380000494E472100562028676F6F642900446F96
:10381000776E2D31304700446F776E2D323547007B
:10382000556E6C6F636B6564005265736572766587
:1038300064000A0D535731206F6E000A0D53573242
:10384000206F6E000A0D535733206F6E000A0D5320
:103850005734206F6E000A0D535735206F6E000AE3
:103860000D535736206F6E0020202020202020008E
:1038700056202862616429004D697373696E670080
:1038800048442020202000334720202020003647B5
:1038900020202020004E2F412020200031324720C0
:1038A0002020004552524F5221000D0A2D2043681E
:1038B000004E6F4C6F636B00446F6E652E00424389
:1038C00038383000424E383830004661696C32007A
:1038D0006E312E35330025642E2564002564682062
:1038E000004F6E20200046616931004D414449007F
:1038F0003454345200365232540032523654004757
:103900006F6F6400676F6F64004E6F6E6500466195
:10391000696C006661696C00527852780054785284
:1039200078005478547800696E66006E616E0025E8
:10393000646D00496E2000312E3000313247004F57
:103940007574002563004844005344003347003633
:1039500047004F4B002566002A00340000FF446AF0
:103960000AC745F50BC746F50CC747F5000E3E6E76
:10397000000E3F6E000E406E000E416E4A6A426AB3
:10398000436A310E0601D065C8EF1CF0CAEF1CF087
:10399000E5EF1CF09551D8A4D0EF1CF0D2EF1CF04D
:1039A000E5EF1CF09651D8A4D8EF1CF0DAEF1CF02C
:1039B000E5EF1CF08EA9DFEF1CF0E1EF1CF09BEFB0
:1039C00024F0010E426E010E436EC5EC6AF0000950
:1039D000D8A4EDEF1CF0EFEF1CF0F1EF1CF09BEF23
:1039E00024F074EC64F04250D8B4F9EF1CF0FBEF13
:1039F0001CF077EF1DF0DC0E206E570EE5EC68F042
:103A0000486E4850D8B407EF1DF009EF1DF073EF72
:103A10001DF0496A070E496410EF1DF012EF1DF00A
:103A200014EF1DF073EF1DF048A019EF1DF01BEF10
:103A30001DF06DEF1DF0150E2A6EC60EE82EFED796
:103A40002A2EFCD700D04950E80F206E570EE5EC27
:103A500068F0486E020E4918D8A431EF1DF033EF1C
:103A60001DF045EF1DF04850D8B439EF1DF03BEF85
:103A70001DF040EF1DF006019489948D5EEF1DF05E
:103A800006019489949D5EEF1DF0030E4918D8A499
:103A90004CEF1DF04EEF1DF05EEF1DF04850D8B416
:103AA00054EF1DF056EF1DF05BEF1DF00601948BF7
:103AB000948F5EEF1DF00601948B949F150E2A6E75
:103AC000C60EE82EFED72A2EFCD700D0DC0E206EC4
:103AD0004AC521F5570E8BEC69F0D8904830486EF6
:103AE000492A0AEF1DF006018E999BEF24F04350FE
:103AF000D8B47DEF1DF07FEF1DF081EF1DF09BEF3F
:103B000024F0060195A187EF1DF089EF1DF00DEF60
:103B10001EF0090E07015E6F0601DB51D8A493EF7A
:103B20001DF095EF1DF0A1EF1DF05F0E096E070E61
:103B30000A6EB10E0B6E380E0C6E43EC6EF0FFEF9A
:103B40001DF0060EDB19D8A4A8EF1DF0AAEF1DF09A
:103B5000B6EF1DF05F0E096E070E0A6E9C0E0B6E1F
:103B6000380E0C6E43EC6EF0FFEF1DF0040EDB1907
:103B7000D8A4BDEF1DF0BFEF1DF0CBEF1DF05F0E21
:103B8000096E070E0A6E870E0B6E380E0C6E43EC34
:103B90006EF0FFEF1DF0050EDB19D8A4D2EF1DF07B
:103BA000D4EF1DF0E0EF1DF05F0E096E070E0A6EF8
:103BB0008E0E0B6E380E0C6E43EC6EF0FFEF1DF0A8
:103BC000030EDB19D8A4E7EF1DF0E9EF1DF0F5EFC8
:103BD0001DF05F0E096E070E0A6E800E0B6E380E1A
:103BE0000C6E43EC6EF0FFEF1DF05F0E096E070EDA
:103BF0000A6E950E0B6E380E0C6E43EC6EF05E0E78
:103C0000206E070E216E236A070E226E560E25ECDB
:103C10006BF0060195919BEF24F095A312EF1EF037
:103C200014EF1EF098EF1EF01A0E0701566F0601F2
:103C3000DC51D8A41EEF1EF020EF1EF02CEF1EF07A
:103C4000570E096E070E0A6EB10E0B6E380E0C6E13
:103C500043EC6EF08AEF1EF0060EDC19D8A433EFA9
:103C60001EF035EF1EF041EF1EF0570E096E070EE5
:103C70000A6E9C0E0B6E380E0C6E43EC6EF08AEFE3
:103C80001EF0040EDC19D8A448EF1EF04AEF1EF017
:103C900056EF1EF0570E096E070E0A6E870E0B6E5A
:103CA000380E0C6E43EC6EF08AEF1EF0050EDC1938
:103CB000D8A45DEF1EF05FEF1EF06BEF1EF0570E05
:103CC000096E070E0A6E8E0E0B6E380E0C6E43ECEC
:103CD0006EF08AEF1EF0030EDC19D8A472EF1EF00E
:103CE00074EF1EF080EF1EF0570E096E070E0A6E7D
:103CF000800E0B6E380E0C6E43EC6EF08AEF1EF0E9
:103D0000570E096E070E0A6E950E0B6E380E0C6E6E
:103D100043EC6EF0560E206E070E216E236A070EDE
:103D2000226E560E25EC6BF0060195939BEF24F066
:103D300095A59DEF1EF09FEF1EF037EF1FF02B0EA5
:103D400007014E6F5450D8B4A8EF1EF0AAEF1EF032
:103D5000B6EF1EF04F0E096E070E0A6E690E0B6E5F
:103D6000380E0C6E43EC6EF029EF1FF00601DD51AA
:103D7000D8A4BDEF1EF0BFEF1EF0CBEF1EF04F0E2C
:103D8000096E070E0A6EB10E0B6E380E0C6E43EC08
:103D90006EF029EF1FF0060EDD19D8A4D2EF1EF049
:103DA000D4EF1EF0E0EF1EF04F0E096E070E0A6E04
:103DB0009C0E0B6E380E0C6E43EC6EF029EF1FF06C
:103DC000040EDD19D8A4E7EF1EF0E9EF1EF0F5EFC1
:103DD0001EF04F0E096E070E0A6E870E0B6E380E20
:103DE0000C6E43EC6EF029EF1FF0050EDD19D8A420
:103DF000FCEF1EF0FEEF1EF00AEF1FF04F0E096EF3
:103E0000070E0A6E8E0E0B6E380E0C6E43EC6EF0C3
:103E100029EF1FF0030EDD19D8A411EF1FF013EFE7
:103E20001FF01FEF1FF04F0E096E070E0A6E800E77
:103E30000B6E380E0C6E43EC6EF029EF1FF04F0E38
:103E4000096E070E0A6E950E0B6E380E0C6E43EC63
:103E50006EF04E0E206E070E216E236A070E226E44
:103E6000560E25EC6BF0060195959BEF24F095A777
:103E70003CEF1FF03EEF1FF0D6EF1FF03C0E0701A6
:103E8000466F5450D8B447EF1FF049EF1FF055EF7D
:103E90001FF0470E096E070E0A6E690E0B6E380E84
:103EA0000C6E43EC6EF0C8EF1FF00601DE51D8A493
:103EB0005CEF1FF05EEF1FF06AEF1FF0470E096E18
:103EC000070E0A6EB10E0B6E380E0C6E43EC6EF0E0
:103ED000C8EF1FF0060EDE19D8A471EF1FF073EFC4
:103EE0001FF07FEF1FF0470E096E070E0A6E9C0E43
:103EF0000B6E380E0C6E43EC6EF0C8EF1FF0040E24
:103F0000DE19D8A486EF1FF088EF1FF094EF1FF0A2
:103F1000470E096E070E0A6E870E0B6E380E0C6E7A
:103F200043EC6EF0C8EF1FF0050EDE19D8A49BEF2E
:103F30001FF09DEF1FF0A9EF1FF0470E096E070E4F
:103F40000A6E8E0E0B6E380E0C6E43EC6EF0C8EFE0
:103F50001FF0030EDE19D8A4B0EF1FF0B2EF1FF070
:103F6000BEEF1FF0470E096E070E0A6E800E0B6E35
:103F7000380E0C6E43EC6EF0C8EF1FF0470E096E62
:103F8000070E0A6E950E0B6E380E0C6E43EC6EF03B
:103F9000460E206E070E216E236A070E226E560E05
:103FA00025EC6BF0060195979BEF24F095A9DBEFCC
:103FB0001FF0DDEF1FF0EEEF1FF0490E08012E6F2E
:103FC0002E0E206E080E216E236A110E226E560EE2
:103FD00025EC6BF0060195999BEF24F095ABF3EF80
:103FE0001FF0F5EF1FF006EF20F05F0E08011B6FCA
:103FF0001B0E206E080E216E236A120E226E560EC4
:1040000025EC6BF00601959B9BEF24F095AD0BEF33
:1040100020F00DEF20F01EEF20F0790E0801516F17
:10402000510E206E080E216E236A100E226E560E5F
:1040300025EC6BF00601959D9BEF24F095AF23EFE7
:1040400020F025EF20F036EF20F0910E0801406FB0
:10405000400E206E080E216E236A100E226E560E40
:1040600025EC6BF00601959F9BEF24F096A13BEFAA
:1040700020F03DEF20F04EEF20F0AB0E07011F6F58
:104080001F0E206E070E216E236A090E226E560E39
:1040900025EC6BF0060196919BEF24F096A353EF6D
:1040A00020F055EF20F066EF20F0BE0E0701156FEF
:1040B000150E206E070E216E236A090E226E560E13
:1040C00025EC6BF0060196939BEF24F096A56BEF21
:1040D00020F06DEF20F09CEF20F0D00E0701836FF1
:1040E000060199A576EF20F078EF20F084EF20F01C
:1040F000840E096E070E0A6EE10E0B6E380E0C6E02
:1041000043EC6EF08EEF20F0840E096E070E0A6EFF
:10411000090E0B6E390E0C6E43EC6EF0830E206EA2
:10412000070E216E236A050E226E560E25EC6BF0EB
:10413000060196959BEF24F096A7A1EF20F0A3EF40
:1041400020F0D2EF20F0DE0E07017D6F06019AA568
:10415000ACEF20F0AEEF20F0BAEF20F07E0E096E4B
:10416000070E0A6EE10E0B6E380E0C6E43EC6EF00D
:10417000C4EF20F07E0E096E070E0A6E090E0B6E5C
:10418000390E0C6E43EC6EF07D0E206E070E216E24
:10419000236A050E226E560E25EC6BF006019697EB
:1041A0009BEF24F096A9D7EF20F0D9EF20F0EAEFAB
:1041B00020F0E90E07013D6F3D0E206E070E216EC7
:1041C000236A070E226E560E25EC6BF006019699B7
:1041D0009BEF24F0FD51D8B4F0EF20F0F2EF20F087
:1041E000CEEF23F0300E2C6E496A0F0E4964FBEFC0
:1041F00020F0FDEF20F0FFEF20F02DEF21F0090E71
:10420000496005EF21F007EF21F01CEF21F0495044
:104210002A6E2B6A010E2A26000E2B222C0E2A242F
:10422000D96E050E2B20DA6E49C509F50A6AFCEC39
:1042300070F0DF6E2AEF21F049502A6E2B6A010ED2
:104240002A26000E2B222C0E2A24D96E050E2B2096
:10425000DA6EDF6A492AF5EF20F02C0E206E050E8B
:10426000216E236A110E226E570E25EC6BF00601AB
:10427000FD6BCEEF23F0100E0701766F760E206EE9
:10428000070E216E236A070E226E570E25EC6BF087
:1042900099EF24F0170E206E4AC521F5570E8BECCE
:1042A00069F099EF24F0400E07019B6F0A6A090E2E
:1042B000096EFCEC70F007019C6F9B0E206E070EE0
:1042C000216E236A060E226E570E25EC6BF099EFD5
:1042D00024F0460E206E4AC521F5570E8BEC69F08E
:1042E00099EF24F0480E0701956F950E206E070E8A
:1042F000216E236A060E226E570E25EC6BF099EFA5
:1043000024F04E0E206E4AC521F5570E8BEC69F055
:1043100099EF24F0500E0801006F000E206E080E79
:10432000216E236A1B0E226E570E25EC6BF099EF5F
:1043300024F06B0E206E4AC521F5570E8BEC69F008
:1043400099EF24F00801806B800E206E080E216E1C
:10435000236A090E226E560E25EC6BF099EF24F0BD
:10436000080E206E4AC521F5560E8BEC69F099EFC8
:1043700024F00F0E456E450E206E050E216E236A49
:10438000030E226E560E25EC6BF099EF24F0110E01
:104390000801766F760E206E080E216E236A090ED4
:1043A000226E560E25EC6BF099EF24F0190E206E5C
:1043B0004AC521F5560E8BEC69F099EF24F0200EDA
:1043C000456E450E206E050E216E236A030E226E89
:1043D000560E25EC6BF099EF24F0220E0701336F97
:1043E0005450D8B4F6EF21F0F8EF21F002EF22F0AC
:1043F000340E096E070E0A6E680E0B6E380E0C6EC8
:1044000043EC6EF0330E206E070E216E236A090E08
:10441000226E560E25EC6BF099EF24F02A0E206EDA
:104420004AC521F5560E8BEC69F099EF24F0310E58
:10443000456E450E206E050E216E236A030E226E18
:10444000560E25EC6BF099EF24F0330E0701296F1F
:104450005450D8B42EEF22F030EF22F03AEF22F091
:104460002A0E096E070E0A6E680E0B6E380E0C6E61
:1044700043EC6EF0290E206E070E216E236A090EA2
:10448000226E560E25EC6BF099EF24F03B0E206E59
:104490004AC521F5560E8BEC69F099EF24F0420ED7
:1044A000456E450E206E050E216E236A030E226EA8
:1044B000560E25EC6BF099EF24F0440E07018F6F38
:1044C0008F0E206E070E216E236A050E226E560E89
:1044D00025EC6BF099EF24F0480E206E4AC521F5CB
:1044E000560E8BEC69F099EF24F0590E456E450E8F
:1044F000206E050E216E236A030E226E560E25ECE9
:104500006BF099EF24F05B0E0701A16FA10E206EF6
:10451000070E216E236A040E226E560E25EC6BF0F8
:1045200099EF24F05E0E206E4AC521F5560E8BECF5
:1045300069F099EF24F0700E456E450E206E050E61
:10454000216E236A030E226E560E25EC6BF099EF56
:1045500024F0720E07016E6F6E0E206E070E216E34
:10456000236A070E226E560E25EC6BF099EF24F0AD
:10457000780E206E4AC521F5560E8BEC69F099EF46
:1045800024F0880E456E450E206E050E216E236ABE
:10459000030E226E560E25EC6BF099EF24F08A0E76
:1045A0000701666F660E206E070E216E236A070EE6
:1045B000226E560E25EC6BF099EF24F0900E206ED3
:1045C0004AC521F5560E8BEC69F099EF24F0A00E48
:1045D000456E450E206E050E216E236A030E226E77
:1045E000560E25EC6BF099EF24F0A20E08016C6FCB
:1045F0006C0E206E080E216E236A090E226E560E76
:1046000025EC6BF099EF24F0AA0E206E4AC521F537
:10461000560E8BEC69F099EF24F0B30E456E450E03
:10462000206E050E216E236A030E226E560E25ECB7
:104630006BF099EF24F0B50E0801626F620E206EE8
:10464000080E216E236A090E226E560E25EC6BF0C1
:1046500099EF24F0BD0E206E4AC521F5560E8BEC65
:1046600069F099EF24F0C60E456E450E206E050EDA
:10467000216E236A030E226E560E25EC6BF099EF25
:1046800024F0C80E0801936F930E206E080E216E61
:10469000236A080E226E560E25EC6BF099EF24F07B
:1046A000CF0E206E4AC521F5560E8BEC69F099EFBE
:1046B00024F0D40E456E450E206E050E216E236A41
:1046C000030E226E560E25EC6BF099EF24F0D60EF9
:1046D00008018A6F8A0E206E080E216E236A080E6A
:1046E000226E560E25EC6BF099EF24F0DD0E206E55
:1046F0004AC521F5560E8BEC69F099EF24F0E20ED5
:10470000456E450E206E050E216E236A030E226E45
:10471000560E25EC6BF099EF24F0E40E0701896F3B
:10472000890E206E070E216E236A050E226E560E2C
:1047300025EC6BF099EF24F0E80E206E4AC521F5C8
:10474000560E8BEC69F099EF24F0EF0E3E6E3E0EA4
:10475000206E050E216E236A030E226E560E25EC86
:104760006BF099EF24F0DE0E206E0C0E216E570ECA
:104770008BEC69F099EF24F0FA0E206E010E216E99
:10478000570E8BEC69F099EF24F0FB0E206E010EB2
:10479000216E570E8BEC69F099EF24F0D051000A8E
:1047A000D8B43BEF21F0010AD8B44AEF21F0030A54
:1047B000D8B453EF21F0010AD8B469EF21F0070A09
:1047C000D8B472EF21F0010AD8B481EF21F0030AC6
:1047D000D8B48AEF21F0010AD8B499EF21F00F0A7A
:1047E000D8B4A2EF21F0010AD8B4B0EF21F0030A47
:1047F000D8B4B9EF21F0010AD8B4C7EF21F0070A05
:10480000D8B4D6EF21F0010AD8B4DFEF21F0030AC3
:10481000D8B4EDEF21F0010AD8B40EEF22F01F0A50
:10482000D8B417EF22F0010AD8B425EF22F0030A1A
:10483000D8B446EF22F0010AD8B44FEF22F0070AAD
:10484000D8B45DEF22F0010AD8B46CEF22F0030A6D
:10485000D8B475EF22F0010AD8B483EF22F00F0A22
:10486000D8B492EF22F0010AD8B49BEF22F0030AE9
:10487000D8B4A9EF22F0010AD8B4B8EF22F0070AA1
:10488000D8B4C1EF22F0010AD8B4CFEF22F0030A66
:10489000D8B4DEEF22F0010AD8B4E7EF22F03F0AE5
:1048A000D8B4F5EF22F0010AD8B404EF23F0030ADC
:1048B000D8B40DEF23F0010AD8B41BEF23F0070A98
:1048C000D8B42AEF23F0010AD8B433EF23F0030A57
:1048D000D8B441EF23F0010AD8B450EF23F00F0A07
:1048E000D8B459EF23F0010AD8B467EF23F0030AD4
:1048F000D8B476EF23F0010AD8B47FEF23F0070A8B
:10490000D8B48DEF23F0010AD8B49CEF23F0030A4A
:10491000D8B4A5EF23F0010AD8B4B3EF23F01F0AEF
:10492000D8B4BCEF23F0010AD8B4C5EF23F099EF57
:1049300024F00601D02B12000501B26B000EB16FFE
:10494000180E096E010E0A6E740E0B6E050E0C6EBB
:10495000080E1DEC45F00501745106018F19D8B4FD
:10496000B4EF24F0B6EF24F0C5EF24F0968974C5B7
:104970008FF63E0E106E070E116E8F51C2EC60F076
:10498000600E0701416F430E426F06018F51050112
:10499000FD5DD8B0CEEF24F0D0EF24F0E2EF24F0AC
:1049A000780E06018F61D7EF24F0D9EF24F0E2EF03
:1049B00024F08FC6FDF50A6AE00E096EFDC50BF501
:1049C0009FEC6CF0060190A3E8EF24F0EAEF24F0EE
:1049D000EEEF24F006018E9110EF2AF0020E050191
:1049E000B16F000E096E010E0A6EB10E0B6E050E50
:1049F0000C6E080EBCEC4FF0030E096E010E0A6E31
:104A0000740E0B6E050E0C6E080E1DEC45F00501C4
:104A10007451D8A40EEF25F010EF25F014EF25F017
:104A2000010EB06F15EF25F0B06BB16B030E096E80
:104A3000010E0A6EB10E0B6E050E0C6E080EBCEC6C
:104A40004FF0320E096E240E0A6E740E0B6E050EB8
:104A50000C6E080E1DEC45F0060199B132EF25F001
:104A600034EF25F041EF25F0050174A13AEF25F070
:104A70003CEF25F041EF25F006019681998154EF36
:104A800025F0060199A147EF25F049EF25F054EFF5
:104A900025F0050174B14FEF25F051EF25F054EFEB
:104AA00025F0060196819991060199B35AEF25F0F8
:104AB0005CEF25F069EF25F0050174A562EF25F0A4
:104AC00064EF25F069EF25F00601968199837CEF6C
:104AD00025F0060199A36FEF25F071EF25F07CEF2B
:104AE00025F0050174B577EF25F079EF25F07CEF1F
:104AF00025F0060196819993060196A182EF25F093
:104B000084EF25F0EAEF25F099A189EF25F08BEFEE
:104B100025F09EEF25F099A390EF25F092EF25F078
:104B20009EEF25F0200E096E070E0A6EEA0E0B6E40
:104B3000370E0C6E43EC6EF0EAEF25F099B1A3EF5F
:104B400025F0A5EF25F0B8EF25F099A3AAEF25F001
:104B5000ACEF25F0B8EF25F0200E096E070E0A6EB7
:104B6000170E0B6E380E0C6E43EC6EF0EAEF25F06C
:104B700099A1BDEF25F0BFEF25F0D2EF25F099B355
:104B8000C4EF25F0C6EF25F0D2EF25F0200E096E18
:104B9000070E0A6EE10E0B6E370E0C6E43EC6EF0D4
:104BA000EAEF25F099B1D7EF25F0D9EF25F0EAEF3C
:104BB00025F099B3DEEF25F0E0EF25F0EAEF25F0E0
:104BC000200E096E070E0A6E0E0E0B6E380E0C6E5E
:104BD00043EC6EF0060194A9F0EF25F0F2EF25F01A
:104BE0001BEF26F094ADF7EF25F0F9EF25F0FEEF7F
:104BF00025F0010E0501B16F00EF26F00501B16B44
:104C0000550E096E010E0A6EB10E0B6E050E0C6E7E
:104C1000080EBCEC4FF00B0E0501B16F000E096ED3
:104C2000010E0A6EB10E0B6E050E0C6E080EBCEC7A
:104C30004FF00601949905019705D8A422EF26F0BC
:104C400024EF26F02CEF26F0060199B52AEF26F086
:104C50002CEF26F04FEF26F005019751D8A433EF43
:104C600026F035EF26F03FEF26F0060199B53BEF31
:104C700026F03DEF26F03FEF26F04FEF26F005013E
:104C80009705D8A446EF26F048EF26F04CEF26F023
:104C9000060199854EEF26F0060199959685050146
:104CA000B46B000EB36FB66B000EB56FB6BF62EF9C
:104CB00026F0B65109E1040EB55DD8A062EF26F0EA
:104CC00064EF26F066EF26F016EF27F0B00EB5255C
:104CD000D96E060EB621DA6E0A0E226E000E236E13
:104CE000B551225EB651235A740E2224E16E050E90
:104CF0002320E26EDE50E618D8B481EF26F083EF71
:104D000026F012EF27F00A0E216E000E226EB5512A
:104D1000215EB651225A740E2124D96E050E22202E
:104D2000DA6EB00EB525E16E060EB621E26EDFC476
:104D3000E7F40601958DB00E0501B525D96E060E76
:104D4000B621DA6EDF50216E2150106E116AB34B1E
:104D5000B42B510EB325126E080EB421136E3AEC2B
:104D600061F0030E0501B519B611D8A4BAEF26F00B
:104D7000BCEF26F0E0EF26F0B34BB42BB3C5B5F58E
:104D8000B4C5B6F5B6BFCEEF26F0B65109E1100EA8
:104D9000B55DD8A0CEEF26F0D0EF26F0D2EF26F00A
:104DA00016EF27F0B54BB62B510EB525D96E080E70
:104DB000B621DA6E200EDF6EB54BB62BC2EF26F0B1
:104DC000B00EB525D96E060EB621DA6E0A0EDF607A
:104DD000ECEF26F0EEEF26F0FAEF26F0B34BB42B13
:104DE000510EB325D96E080EB421DA6E2E0EDF6E89
:104DF00012EF27F0B00EB525D96E060EB621DA6E89
:104E0000640EDF6006EF27F008EF27F00CEF27F0C5
:104E1000B34BB42BEEEF26F0B34BB42BB34BB42B08
:104E2000EEEF26F0B54BB62B56EF26F0600E1A6E5D
:104E3000050E1B6E020E1C6EC6EC62F00501B66B11
:104E4000000EB56FB6BF2EEF27F0B65109E1060E82
:104E5000B55DD8A02EEF27F030EF27F032EF27F026
:104E6000A1EF27F0CA0EB525D96E070EB621DA6E6E
:104E7000600EB525E16E050EB621E26EDE50E61835
:104E8000D8B445EF27F047EF27F09DEF27F0600EED
:104E9000B525D96E050EB621DA6ECA0EB525E16EBE
:104EA000070EB621E26EDFC4E7F40601958B030E10
:104EB0000501B503F3C421F5F4C422F5B603F3509C
:104EC00022261C0E2124D96E080E2220DA6ECA0E6C
:104ED000B525E16E070EB621E26EE7507CEC6EF070
:104EE000DF6E030E0501B503F3C421F5F4C422F50A
:104EF000B603F35022261D0E2124D96E080E22205F
:104F0000DA6ECA0EB525E16E070EB621E26EE750E5
:104F1000B4EC6EF0DF6E030E0501B503F3C421F5AA
:104F2000F4C422F5B603F35022261E0E2124D96EB6
:104F3000080E2220DA6E3A0EDF6EB54BB62B22EF4A
:104F400027F0220E096E100E0A6E740E0B6E050EFF
:104F50000C6E040E1DEC45F00501B66B000EB56F2E
:104F6000B6BFBCEF27F0B65109E1100EB55DD8A071
:104F7000BCEF27F0BEEF27F0C0EF27F0F8EF27F0E7
:104F8000D00EB525D96E070EB621DA6E740EB52592
:104F9000E16E050EB621E26EDE50E618D8B4D3EF0E
:104FA00027F0D5EF27F0F4EF27F0740EB525D96E72
:104FB000050EB621DA6ED00EB525E16E070EB621CC
:104FC000E26EDFC4E7F406019589D00E0501B52530
:104FD000D96E070EB621DA6E2F0EB525E16E080EDA
:104FE000B621E26EDFC4E7F4B54BB62BB0EF27F085
:104FF000010EB16F030E096E010E0A6EB10E0B6E3B
:10500000050E0C6E080EBCEC4FF0320E096E240E2D
:105010000A6E740E0B6E050E0C6E080E1DEC45F03C
:1050200006019AB116EF28F018EF28F025EF28F0C6
:10503000050174A11EEF28F020EF28F025EF28F0DD
:10504000060196839A8138EF28F006019AA12BEF8A
:1050500028F02DEF28F038EF28F0050174B133EF78
:1050600028F035EF28F038EF28F0060196839A9162
:1050700006019AB33EEF28F040EF28F04DEF28F0FC
:10508000050174A546EF28F048EF28F04DEF28F011
:10509000060196839A8360EF28F006019AA353EFE6
:1050A00028F055EF28F060EF28F0050174B55BEFAC
:1050B00028F05DEF28F060EF28F0060196839A93C0
:1050C000060196A366EF28F068EF28F0CEEF28F0EF
:1050D0009AA16DEF28F06FEF28F082EF28F09AA3E5
:1050E00074EF28F076EF28F082EF28F0160E096EA4
:1050F000070E0A6EEA0E0B6E370E0C6E43EC6EF066
:10510000CEEF28F09AB187EF28F089EF28F09CEFD6
:1051100028F09AA38EEF28F090EF28F09CEF28F06B
:10512000160E096E070E0A6E170E0B6E380E0C6EF9
:1051300043EC6EF0CEEF28F09AA1A1EF28F0A3EF98
:1051400028F0B6EF28F09AB3A8EF28F0AAEF28F0DD
:10515000B6EF28F0160E096E070E0A6EE10E0B6E02
:10516000370E0C6E43EC6EF0CEEF28F09AB1BBEF29
:1051700028F0BDEF28F0CEEF28F09AB3C2EF28F068
:10518000C4EF28F0CEEF28F0160E096E070E0A6E57
:105190000E0E0B6E380E0C6E43EC6EF0060194ABE7
:1051A000D4EF28F0D6EF28F0FFEF28F094AFDBEF34
:1051B00028F0DDEF28F0E2EF28F0010E0501B16FD5
:1051C000E4EF28F00501B16B550E096E010E0A6E71
:1051D000B10E0B6E050E0C6E080EBCEC4FF00B0EF4
:1051E0000501B16F000E096E010E0A6EB10E0B6E55
:1051F000050E0C6E080EBCEC4FF00601949B0501E9
:105200009705D8A406EF29F008EF29F010EF29F050
:1052100006019AB50EEF29F010EF29F033EF29F0CF
:1052200005019751D8A417EF29F019EF29F023EFC2
:1052300029F006019AB51FEF29F021EF29F023EF9D
:1052400029F033EF29F005019705D8A42AEF29F0BA
:105250002CEF29F030EF29F006019A8532EF29F082
:1052600006019A9596870501B46B000EB36FB66B75
:10527000000EB56FB6BF46EF29F0B65109E1040E36
:10528000B55DD8A046EF29F048EF29F04AEF29F0A4
:10529000FAEF29F0AC0EB525D96E060EB621DA6EFE
:1052A0000A0E226E000E236EB551225EB651235AAD
:1052B000740E2224E16E050E2320E26EDE50E61805
:1052C000D8B465EF29F067EF29F0F6EF29F00A0E60
:1052D000216E000E226EB551215EB651225A740E17
:1052E0002124D96E050E2220DA6EAC0EB525E16EB2
:1052F000060EB621E26EDFC4E7F40601958FAC0E10
:105300000501B525D96E060EB621DA6EDF50216E85
:105310002150106E116AB34BB42B400EB325126EA0
:10532000080EB421136E3AEC61F0030E0501B519B5
:10533000B611D8A49EEF29F0A0EF29F0C4EF29F010
:10534000B34BB42BB3C5B5F5B4C5B6F5B6BFB2EF24
:1053500029F0B65109E1100EB55DD8A0B2EF29F0E1
:10536000B4EF29F0B6EF29F0FAEF29F0B54BB62BE0
:10537000400EB525D96E080EB621DA6E200EDF6E0E
:10538000B54BB62BA6EF29F0AC0EB525D96E060E9F
:10539000B621DA6E0A0EDF60D0EF29F0D2EF29F0E5
:1053A000DEEF29F0B34BB42B400EB325D96E080EB7
:1053B000B421DA6E2E0EDF6EF6EF29F0AC0EB525B5
:1053C000D96E060EB621DA6E640EDF60EAEF29F0C0
:1053D000ECEF29F0F0EF29F0B34BB42BD2EF29F02A
:1053E000B34BB42BB34BB42BD2EF29F0B54BB62B48
:1053F0003AEF29F0B005D8A400EF2AF002EF2AF026
:10540000EAEF24F0B16B030E096E010E0A6EB10EC5
:105410000B6E050E0C6E080EBCEC4FF0EAEF24F09C
:1054200012000501986B72C599F573C59AF574C59C
:105430009BF575C59CF59CBF22EF2AF020EF2AF062
:1054400036EF2AF0010E986F99C509F59AC50AF54D
:105450009BC50BF59CC50CF560EC6EF009C599F584
:105460000AC59AF50BC59BF50CC59CF505019E6B0D
:10547000000E9D6FB6C688F5B7C689F59851D8B4A9
:1054800044EF2AF046EF2AF058EF2AF09851D8A4BA
:105490004CEF2AF04EEF2AF053EF2AF07E6B2B0EE2
:1054A0007D6F56EF2AF07E6B2D0E7D6F7DC598F5D2
:1054B00099C509F59AC50AF59BC50BF59CC50CF570
:1054C00046EC60F009040A10D8A469EF2AF06BEFEB
:1054D0002AF0A1EF2AF005019851D8B472EF2AF012
:1054E00074EF2AF07CEF2AF098C59CF88807D8A0C2
:1054F00089079E6B010E9D6F9C0E9D25096E080EFF
:105500009E210A6E270E0B6E390E0C6E43EC6EF068
:105510000501FD0E8827FF0E892370C519F571C599
:105520001AF59C0E1B6E080E1C6E88C51DF589C5EC
:105530001EF589EC66F019C570F51AC571F507EF0F
:105540002FF099C509F59AC50AF59BC50BF59CC5C1
:105550000CF546EC60F009500A10D8A4B2EF2AF01E
:10556000B4EF2AF0D3EF2AF005019851D8B4BBEF7D
:105570002AF0BDEF2AF0C5EF2AF098C59CF88807FD
:10558000D8A089079E6B010E9D6F9C0E9D25096E0C
:10559000080E9E210A6E2B0E0B6E390E0C6E43EC1C
:1055A0006EF088EF2AF0000E05019F6F000EA06FCD
:1055B000800EA16F3F0EA26F876B000E866F99C59C
:1055C00009F59AC50AF59BC50BF59CC50CF5000EAF
:1055D0000D6E000E0E6E000E0F6E000E106ECCECF7
:1055E00063F0D8B0F6EF2AF0F8EF2AF0D7EF2BF0FF
:1055F00005EF2BF08AC59FF58BC5A0F58CC5A1F5ED
:105600008DC5A2F50501864B872B9FC517F5A0C553
:1056100018F5A1C519F5A2C51AF5000E1B6E000EEE
:105620001C6E200E1D6E410E1E6E0AEC43F017C557
:105630008AF518C58BF519C58CF51AC58DF50501C8
:105640008A51995D096E8B519A590A6E8C519B59FA
:105650000B6E8D519C590C6E7FEC6BF00CBE3CEFC9
:105660002BF00C500B100A1009E1020E095CD8A0B7
:105670003CEF2BF03EEF2BF0FAEF2AF08AC530F525
:105680008BC531F58CC532F58DC533F599C534F52B
:105690009AC535F59BC536F59CC537F5C7EC5EF068
:1056A000D8A055EF2BF057EF2BF0FAEF2AF00501B9
:1056B0009F51995D096EA0519A590A6EA1519B594B
:1056C0000B6EA2519C590C6E7FEC6BF00CBE76EF0A
:1056D0002BF00C500B100A1007E1020E095CD8B039
:1056E00074EF2BF076EF2BF0BEEF2BF09FC599F502
:1056F000A0C59AF5A1C59BF5A2C59CF5D7EF2BF0E7
:105700009FC530F5A0C531F5A1C532F5A2C533F569
:10571000000E346E000E356E200E366E410E376E62
:10572000CCEC4AF030C59FF531C5A0F532C5A1F5E6
:1057300033C5A2F505018607D8A087079F51995D5B
:10574000096EA0519A590A6EA1519B590B6EA25134
:105750009C590C6E7FEC6BF00CBEBCEF2BF00C5028
:105760000B100A1007E1020E095CD8B0BAEF2BF05B
:10577000BCEF2BF0BEEF2BF076EF2BF099C530F598
:105780009AC531F59BC532F59CC533F59FC534F5F7
:10579000A0C535F5A1C536F5A2C537F5C7EC5EF055
:1057A000D8A0D5EF2BF0D7EF2BF080EF2BF076C5FC
:1057B00080F580C581F50601B9BFE1EF2BF0E3EF7D
:1057C0002BF0E9EF2BF0B8C679F5B9C67AF5EDEF15
:1057D0002BF005017A6B060E796F79C584F57AC5D1
:1057E00085F50501844B852B660E8119D8A4FBEF46
:1057F0002BF0FDEF2BF01CEF2CF087BF04EF2CF00B
:1058000002EF2CF00FEF2CF0000E9F6F000EA06F38
:10581000800EA16F3F0EA26F876B000E866F670E22
:105820008019D8B416EF2CF018EF2CF01CEF2CF0E8
:1058300086518427875185238F6B000E8E6F99C503
:1058400090F59AC591F59BC592F59CC593F59FC5BA
:105850008AF5A0C58BF5A1C58CF5A2C58DF5ACEF79
:105860002CF090C530F591C531F592C532F593C550
:1058700033F59FC534F5A0C535F5A1C536F5A2C5EC
:1058800037F5CCEC4AF030C549F531C54AF532C59B
:105890004BF533C54CF524EC56F049C594F54AC593
:1058A00095F54BC596F54CC597F594C509F595C585
:1058B0000AF596C50BF597C50CF544EC5EF009C5E5
:1058C00082F50AC583F590C530F591C531F592C5CD
:1058D00032F593C533F594C51BF595C51CF596C5F2
:1058E0001DF597C51EF59FC517F5A0C518F5A1C5EF
:1058F00019F5A2C51AF50AEC43F017C534F518C519
:1059000035F519C536F51AC537F55CEC6DF030C5BF
:1059100090F531C591F532C592F533C593F59FC524
:1059200030F5A0C531F5A1C532F5A2C533F5000E9D
:10593000346E000E356E200E366E410E376ECCEC96
:105940004AF030C59FF531C5A0F532C5A1F533C584
:10595000A2F505018E4B8F2B84518E5D8F51800AED
:105960004D6E8551800A4D58D8A0B9EF2CF0BBEF91
:105970002CF031EF2CF09FC517F5A0C518F5A1C587
:1059800019F5A2C51AF5000E1B6E000E1C6EA00EB6
:105990001D6E400E1E6E0AEC43F017C594F518C537
:1059A00095F519C596F51AC597F590C530F591C5C9
:1059B00031F592C532F593C533F594C534F595C5E7
:1059C00035F596C536F597C537F5C7EC5EF0D8B016
:1059D000ECEF2CF0EEEF2CF0F9EF2CF0000E0501BF
:1059E000946F000E956F000E966F000E976F22EF6A
:1059F0002DF090C509F591C50AF592C50BF593C533
:105A00000CF594C50DF595C50EF596C50FF597C522
:105A100010F5CCEC63F0D8A010EF2DF012EF2DF0C4
:105A200022EF2DF0050182B118EF2DF01AEF2DF0C5
:105A300022EF2DF0000E946F000E956F000E966F02
:105A4000000E976F99C509F59AC50AF59BC50BF528
:105A50009CC50CF594C50DF595C50EF596C50FF5CD
:105A600097C510F55BEC3EF009C590F50AC591F5B8
:105A70000BC592F50CC593F590C530F591C531F580
:105A800092C532F593C533F5000E1B6E000E1C6EE9
:105A9000200E1D6E410E1E6E8AC517F58BC518F5BA
:105AA0008CC519F58DC51AF50AEC43F017C534F508
:105AB00018C535F519C536F51AC537F5C7EC5EF0CA
:105AC000D8A065EF2DF067EF2DF090EF2DF00501D8
:105AD000864B872B8AC517F58BC518F58CC519F52C
:105AE0008DC51AF5000E1B6E000E1C6E200E1D6E6D
:105AF000410E1E6E0AEC43F017C58AF518C58BF5EA
:105B000019C58CF51AC58DF5660E05018119D8A445
:105B10008CEF2DF08EEF2DF090EF2DF0844B852B38
:105B20008AC59FF58BC5A0F58CC5A1F58DC5A2F5DD
:105B300086C577F587C578F505017F6B7C6B000E10
:105B40007B6F8F6B000E8E6F8AEF2EF090C530F555
:105B500091C531F592C532F593C533F59FC534F53E
:105B6000A0C535F5A1C536F5A2C537F5CCEC4AF090
:105B700030C549F531C54AF532C54BF533C54CF54D
:105B800024EC56F049C594F54AC595F54BC596F5F4
:105B90004CC597F594C509F595C50AF596C50BF55D
:105BA00097C50CF544EC5EF00ABEE2EF2DF00A500A
:105BB00007E10A0E095CD8B0E0EF2DF0E2EF2DF01E
:105BC000F2EF2DF094C509F595C50AF596C50BF5CC
:105BD00097C50CF544EC5EF009C582F50AC583F55E
:105BE000F6EF2DF00501836B090E826F05017F51E1
:105BF000D8A4FDEF2DF0FFEF2DF027EF2EF078BFAA
:105C000006EF2EF004EF2EF027EF2EF09C0E9D25D0
:105C1000D96E080E9E21DA6E2E0EDF6E9D4B9E2BE6
:105C20008807D8A08907010E7F6F27EF2EF09C0E02
:105C30009D25D96E080E9E21DA6E300EDF6E9D4BCB
:105C40009E2B8807D8A089077B07D8A07C077B51AB
:105C50007C11D8A42EEF2EF030EF2EF017EF2EF09F
:105C60009C0E9D25D96E080E9E21DA6E8251300F52
:105C7000DF6E9D4B9E2B8807D8A0890790C530F515
:105C800091C531F592C532F593C533F594C51BF531
:105C900095C51CF596C51DF597C51EF59FC517F54D
:105CA000A0C518F5A1C519F5A2C51AF50AEC43F06F
:105CB00017C534F518C535F519C536F51AC537F5C4
:105CC0005CEC6DF030C590F531C591F532C592F5BB
:105CD00033C593F59FC530F5A0C531F5A1C532F5A3
:105CE000A2C533F5000E346E000E356E200E366EF2
:105CF000410E376ECCEC4AF030C59FF531C5A0F5AA
:105D000032C5A1F533C5A2F505017707D8A07807FC
:105D10008E4B8F2B84518E5D8F51800A4D6E855135
:105D2000800A4D58D8B097EF2EF099EF2EF0A7EFDC
:105D30002EF09EBFA5EF2EF09E5109E14B0E9D5D0A
:105D4000D8A0A5EF2EF0A7EF2EF0A6EF2DF08F6BC9
:105D50004F0E8E6F9C0E8E25D96E080E8F21DA6E37
:105D6000DF6A9C0E4D6E080E4E6E9D514D5E9E512B
:105D70004E5A8E514D240D6E8F514E200E6E9C0E3C
:105D80000F6E080E106E9DC511F59EC512F5F6EC4E
:105D900069F005019D518E5D9D6F9E518F599E6FDB
:105DA0009851D8A4D6EF2EF0D9EF2EF0010EDAEFED
:105DB0002EF0000E8E6F8F6B9851D8B4E2EF2EF05C
:105DC000E4EF2EF0EFEF2EF09D07D8A09E079C0E7B
:105DD0009D25D96E080E9E21DA6E98C5DFF48E518E
:105DE000885F8F51895B70C519F571C51AF59C0ED6
:105DF0009D251B6E080E9E211C6E88C51DF589C54C
:105E00001EF589EC66F019C570F51AC571F512001A
:105E10000601236B010E226F010E206F020E216F0F
:105E2000200E0A6E350E0B6EC3EC67F00601FE51B4
:105E3000D8A41DEF2FF01FEF2FF046EF2FF00A6AC6
:105E4000EA0E096EFCEC70F00601206F0A6AEB0E98
:105E5000096EFCEC70F00601216F140E0501BD6F98
:105E6000060EBE6FD60EBF6F380EC06F20C6C1F5CE
:105E7000C26B21C6C3F5C46BC6EC6CF0140E0A6E7F
:105E8000060E0B6EC3EC67F04CEF2FF0370E0A6E68
:105E9000390E0B6EC3EC67F0690E0A6E350E0B6E91
:105EA000C3EC67F0D00E0A6E380E0B6EC3EC67F0D1
:105EB000BF0E0A6E360E0B6EC3EC67F0020E0601C3
:105EC000A119D8A466EF2FF068EF2FF070EF2FF034
:105ED000F00E0A6E380E0B6EC3EC67F097EF2FF0E2
:105EE000A105D8A476EF2FF078EF2FF080EF2FF0F8
:105EF000F50E0A6E380E0B6EC3EC67F097EF2FF0BD
:105F0000040EA119D8A487EF2FF089EF2FF091EF9D
:105F10002FF0FA0E0A6E380E0B6EC3EC67F097EF97
:105F20002FF0FC0E0A6E370E0B6EC3EC67F0730E8B
:105F30000A6E360E0B6EC3EC67F0060190A1A3EF5C
:105F40002FF0A5EF2FF0ADEF2FF0C40E0A6E380E34
:105F50000B6EC3EC67F0BAEF2FF090B1B2EF2FF0F9
:105F6000B4EF2FF0BAEF2FF0BE0E0A6E380E0B6EA4
:105F7000C3EC67F00D0E0A6E360E0B6EC3EC67F0C5
:105F80003E0E4CEC6FF009C524F60AC525F63D0E11
:105F9000306E0A0E316E030E326E460E336E24C61C
:105FA00009F525C60AF50B6A0C6A000E0EEC58F0CE
:105FB00009C534F50AC535F50BC536F50CC537F5F9
:105FC000CCEC4AF030C52BF631C52CF632C52DF697
:105FD00033C52EF62BC626F62CC627F62DC628F678
:105FE0002EC629F69B0E0A6E370E0B6EC3EC67F0B9
:105FF00026C6DBF527C6DCF528C6DDF529C6DEF5A5
:10600000000E0501DF6F060EE06FE26B140EE16F0C
:106010001CEC6FF0000E0A6E060E0B6EC3EC67F000
:1060200026C630F527C631F528C632F529C633F520
:106030007B0E346E140E356E4E0E366E400E376E7D
:10604000C7EC5EF0D8A027EF30F029EF30F04AEF30
:1060500030F0EC0E306E510E316E580E326E400E36
:10606000336E26C634F527C635F528C636F529C65B
:1060700037F5C7EC5EF0D8A040EF30F042EF30F0DB
:106080004AEF30F0050E0A6E380E0B6EC3EC67F067
:1060900050EF30F0700E0A6E380E0B6EC3EC67F0E6
:1060A0000D0E4CEC6FF009C524F60AC525F626C680
:1060B0001BF527C61CF528C61DF529C61EF524C6E6
:1060C00009F525C60AF50B6A0C6A000E0EEC58F0AD
:1060D00009C517F50AC518F50BC519F50CC51AF54C
:1060E0000AEC43F017C530F518C531F519C532F57E
:1060F0001AC533F5000E346EF00E356E7F0E366E17
:10610000450E376ECCEC4AF030C52BF631C52CF677
:1061100032C52DF633C52EF6870E0A6E370E0B6E7E
:10612000C3EC67F02BC6DBF52CC6DCF52DC6DDF520
:106130002EC6DEF5000E0501DF6F060EE06FE26B86
:10614000140EE16F1CEC6FF0000E0A6E060E0B6E63
:10615000C3EC67F02BC630F52CC631F52DC632F5F1
:106160002EC633F5480E346EE10E356E1A0E366EBD
:10617000400E376EC7EC5EF0D8A0C1EF30F0C3EF31
:1061800030F0E4EF30F0B80E306E1E0E316E250E9A
:10619000326E400E336E2BC634F52CC635F52DC647
:1061A00036F52EC637F5C7EC5EF0D8A0DAEF30F042
:1061B000DCEF30F0E4EF30F0050E0A6E380E0B6EB7
:1061C000C3EC67F0EAEF30F0700E0A6E380E0B6E1B
:1061D000C3EC67F00C0E4CEC6FF009C524F60AC551
:1061E00025F626C61BF527C61CF528C61DF529C6AB
:1061F0001EF524C609F525C60AF50B6A0C6A000EC1
:106200000EEC58F009C517F50AC518F50BC519F5B8
:106210000CC51AF50AEC43F017C530F518C531F571
:1062200019C532F51AC533F5000E346EF00E356E11
:106230007F0E366E450E376ECCEC4AF030C52BF62D
:1062400031C52CF632C52DF633C52EF6910E0A6EE9
:10625000370E0B6EC3EC67F02BC6DBF52CC6DCF5F6
:106260002DC6DDF52EC6DEF5000E0501DF6F060E2C
:10627000E06FE26B140EE16F1CEC6FF0000E0A6E23
:10628000060E0B6EC3EC67F02BC630F52CC631F54D
:106290002DC632F52EC633F5F60E346E280E356E49
:1062A000DC0E366E3F0E376EC7EC5EF0D8A05BEFAB
:1062B00031F05DEF31F07EEF31F0D70E306EA30E8E
:1062C000316EF00E326E3F0E336E2BC634F52CC697
:1062D00035F52DC636F52EC637F5C7EC5EF0D8A0DD
:1062E00074EF31F076EF31F07EEF31F0050E0A6E8B
:1062F000380E0B6EC3EC67F084EF31F0700E0A6E4F
:10630000380E0B6EC3EC67F0800E0A6E350E0B6E06
:10631000C3EC67F0010E06012A6F040E2A6593EFA5
:1063200031F095EF31F097EF31F0E0EF31F00A6A9C
:10633000000E096E2A51BCEC59F009C51EF60AC5BB
:106340001FF606012A510501E36FE46B1F0E0601DB
:106350001E150501E56F000E06011F150501E66F0C
:10636000E351E51907E1E451E619D8A4BAEF31F099
:10637000BCEF31F0C1EF31F0060122519813C5EFA7
:1063800031F006012251FF0A9817D8902235226F6A
:106390002335236F5450D8B4D0EF31F0D2EF31F021
:1063A000DDEF31F0020E2A19D8A4D9EF31F0DBEF7E
:1063B00031F0DDEF31F0E0EF31F02A2B8DEF31F0ED
:1063C000630E0A6E360E0B6EC3EC67F0060198A1E1
:1063D000ECEF31F0EEEF31F0F6EF31F0040E0A6E33
:1063E000390E0B6EC3EC67F0FCEF31F0130E0A6E42
:1063F000390E0B6EC3EC67F01F0E0A6E360E0B6E75
:10640000C3EC67F0060198A308EF32F00AEF32F010
:1064100012EF32F0040E0A6E390E0B6EC3EC67F009
:1064200018EF32F0130E0A6E390E0B6EC3EC67F0E4
:106430000601D851D8B41FEF32F021EF32F059EFF6
:1064400032F0300E0A6E360E0B6EC3EC67F00601AA
:1064500098A52DEF32F02FEF32F037EF32F0040E27
:106460000A6E390E0B6EC3EC67F03DEF32F0130E7F
:106470000A6E390E0B6EC3EC67F0410E0A6E360ED3
:106480000B6EC3EC67F0060198A749EF32F04BEFB3
:1064900032F053EF32F0040E0A6E390E0B6EC3EC7D
:1064A00067F059EF32F0130E0A6E390E0B6EC3EC23
:1064B00067F0950E0A6E350E0B6EC3EC67F00601A1
:1064C00090516FEC70F0060190A169EF32F06BEF24
:1064D00032F005EF33F0916B926B8CEC5AF0CE0EEC
:1064E0000A6E360E0B6EC3EC67F06F0E0A6E370E37
:1064F0000B6EC3EC67F006019105D8A482EF32F071
:1065000084EF32F08CEF32F0220E0A6E390E0B6EF1
:10651000C3EC67F0BDEF32F0020E9119D8A493EFEF
:1065200032F095EF32F09DEF32F0180E0A6E390E10
:106530000B6EC3EC67F0BDEF32F0040E9119D8A4D6
:10654000A4EF32F0A6EF32F0AEEF32F01D0E0A6E7D
:10655000390E0B6EC3EC67F0BDEF32F0080E9119E7
:10656000D8A4B5EF32F0B7EF32F0BDEF32F0780ECD
:106570000A6E380E0B6EC3EC67F07B0E0A6E370E98
:106580000B6EC3EC67F006019205D8A4CAEF32F097
:10659000CCEF32F0D4EF32F0220E0A6E390E0B6ED1
:1065A000C3EC67F005EF33F0020E9219D8A4DBEFCD
:1065B00032F0DDEF32F0E5EF32F0180E0A6E390EF0
:1065C0000B6EC3EC67F005EF33F0040E9219D8A4FC
:1065D000ECEF32F0EEEF32F0F6EF32F01D0E0A6E15
:1065E000390E0B6EC3EC67F005EF33F0080E92190D
:1065F000D8A4FDEF32F0FFEF32F005EF33F0780E64
:106600000A6E380E0B6EC3EC67F0FA0E0A6E350E8A
:106610000B6EC3EC67F01200306A000E2F6E010E95
:10662000346E010E326E336A010E2C6E316AEDEC5F
:1066300071F00601916B926B8CEC5AF0F7C62DF558
:10664000F8C62EF52D0E0A6E310E0B6EC3EC67F0F8
:10665000B6EF33F00D0E2A6E2D0E296ED80EE82EF1
:10666000FED7292EFCD72A2EFAD72D8C2D9E2E80D0
:106670002E92010E356E200E0A6E000E096E35C583
:106680000BF50D6A110E0C6E010E0F6E010E0E6EE3
:1066900005EC5CF05450D8B450EF33F052EF33F0C7
:1066A0005DEF33F0020E3518D8A459EF33F05BEFED
:1066B00033F05DEF33F066EF33F0352A040E3564C6
:1066C00064EF33F066EF33F03BEF33F0020E206EF1
:1066D0002DC521F52EC522F5200E55EC69F00D0EC5
:1066E0002A6E2D0E296ED80EE82EFED7292EFCD745
:1066F0002A2EFAD72D8E2D9C2E822E90010E356ECD
:10670000200E0A6E000E096E35C50BF50D6A110ECE
:106710000C6E010E0F6E000E0E6E05EC5CF0545008
:10672000D8B495EF33F097EF33F0A2EF33F0020EC9
:106730003518D8A49EEF33F0A0EF33F0A2EF33F07A
:10674000ABEF33F0352A040E3564A9EF33F0ABEF2D
:1067500033F080EF33F0020E206E2DC521F52EC5EB
:1067600022F5200E55EC69F02F4A302A30BEC2EFD8
:1067700033F0305009E11E0E2F5CD8A0C2EF33F089
:10678000C4EF33F02AEF33F0010E356E200E0A6E9F
:10679000000E096E35C50BF50D6A110E0C6E010E5B
:1067A0000F6E020E0E6E05EC5CF05450D8B4DBEFA9
:1067B00033F0DDEF33F0E8EF33F0020E3518D8A4F4
:1067C000E4EF33F0E6EF33F0E8EF33F0F1EF33F0DE
:1067D000352A040E3564EFEF33F0F1EF33F0C6EFF6
:1067E00033F0020E206EF7C621F5F8C622F5200E12
:1067F00055EC69F0000E206E420E216E570E8BECA8
:1068000069F0150E296EC60EE82EFED7292EFCD78C
:1068100000D0000E206E570EE5EC68F02B6EF90EDE
:106820000A6E360E0B6EC3EC67F0420E2B18D8A41E
:106830001CEF34F01EEF34F026EF34F0520E0A6EE7
:10684000390E0B6EC3EC67F02CEF34F00E0E0A6EAF
:10685000390E0B6EC3EC67F0F40E0A6E310E0B6E40
:10686000C3EC67F0C686C69EBE8E150E296EC60E98
:10687000E82EFED7292EFCD700D0CEB642EF34F05A
:1068800044EF34F064EF34F0BE9E150E296EC60E50
:10689000E82EFED7292EFCD700D0CEA652EF34F03A
:1068A00054EF34F05CEF34F0FF0E0A6E380E0B6ECE
:1068B000C3EC67F06AEF34F0E60E0A6E380E0B6E2A
:1068C000C3EC67F06AEF34F0CA0E0A6E380E0B6E36
:1068D000C3EC67F04F0E0A6E320E0B6EC3EC67F01E
:1068E000C688C69CBE8C150E296EC60EE82EFED735
:1068F000292EFCD700D0CEB880EF34F082EF34F0F0
:10690000A2EF34F0BE9C150E296EC60EE82EFED7FF
:10691000292EFCD700D0CEA890EF34F092EF34F0BF
:106920009AEF34F0FF0E0A6E380E0B6EC3EC67F070
:10693000A8EF34F00E0E0A6E390E0B6EC3EC67F042
:10694000A8EF34F0CA0E0A6E380E0B6EC3EC67F077
:10695000010E356E200E0A6E000E096E35C50BF560
:106960000D6A0A0E0C6E1F0E0F6E080E0E6E05ECF1
:106970005CF0200E0A6E000E096E35C50BF50D6A2F
:10698000060E0C6E0F6A0C0E0E6E05EC5CF0352ACE
:10699000040E3564CEEF34F0D0EF34F0AAEF34F0CB
:1069A000D00E296ECA0EE82EFED7292EFCD796EC03
:1069B0005CF0306A000E2F6E2F503010D8A4E3EF39
:1069C00034F0E5EF34F0EDEF34F0AA0E0A6E350E38
:1069D0000B6EC3EC67F0F4EF34F0D30E0A6E350E95
:1069E0000B6EC3EC67F0346A200E0A6E000E096E5F
:1069F000040E0B6E0D6A490E0C6E0F6A0A0E0E6EB7
:106A000005EC5CF0B20E0A6E310E0B6EC3EC67F053
:106A100032C517F534C518F5010E03EC49F032C53F
:106A200017F534C518F531C519F5020EB6EC40F06E
:106A300033C517F534C518F531C519F5030EB6EC95
:106A400040F032C517F534C518F531C519F5040EF7
:106A5000B6EC40F096EC5CF0050E2A6E0F0E296E37
:106A6000F10EE82EFED7292EFCD72A2EFAD70000E9
:106A7000200E0A6E000E096E010E0B6E0D6A490E95
:106A80000C6E0F6A0A0E0E6E05EC5CF0000E0A6EBC
:106A9000330E0B6EC3EC67F033C517F534C518F52C
:106AA000040E03EC49F033C517F534C518F531C5AC
:106AB00019F5010EB6EC40F096EC5CF0200E0A6E73
:106AC000000E096E040E0B6E0D6A490E0C6E0F6AF5
:106AD0000A0E0E6E05EC5CF0990E0A6E320E0B6E0D
:106AE000C3EC67F033C517F534C518F5030E03EC96
:106AF00049F033C517F534C518F52CC519F5040E42
:106B0000B6EC40F096EC5CF0200E0A6E000E096EBA
:106B1000030E0B6E0D6A490E0C6E0F6A0A0E0E6E96
:106B200005EC5CF0760E0A6E320E0B6EC3EC67F06D
:106B300032C517F534C518F5040E03EC49F032C51B
:106B400017F534C518F531C519F5030EB6EC40F04C
:106B500096EC5CF0200E0A6E000E096E020E0B6EB3
:106B60000D6A490E0C6E0F6A0A0E0E6E05EC5CF093
:106B7000BC0E0A6E320E0B6EC3EC67F033C517F510
:106B800034C518F5010E03EC49F033C517F534C5CB
:106B900018F52CC519F5020EB6EC40F096EC5CF039
:106BA000200E0A6E000E096E010E0B6E0D6A490E64
:106BB0000C6E0F6A0A0E0E6E05EC5CF0DE0E0A6EAD
:106BC000320E0B6EC3EC67F032C517F534C518F5FD
:106BD000020E03EC49F032C517F534C518F531C57E
:106BE00019F5010EB6EC40F096EC5CF02F4A302A15
:106BF00030BE04EF36F0305009E1020E2F5CD8A011
:106C000004EF36F006EF36F0DCEF34F0410E0A6E9A
:106C1000330E0B6EC3EC67F0EAEC71F0060194934F
:106C2000120090C653F53E0E4CEC6FF009C564F5AA
:106C30000AC565F53D0E306E0A0E316E030E326EDA
:106C4000460E336E64C509F565C50AF50B6A0C6A14
:106C5000000E0EEC58F009C534F50AC535F50BC524
:106C600036F50CC537F5CCEC4AF030C566F531C5C4
:106C700067F532C568F533C569F566C560F567C562
:106C800061F568C562F569C563F5090E4CEC6FF0F6
:106C900009C564F50AC565F560C51BF561C51CF538
:106CA00062C51DF563C51EF564C509F565C50AF520
:106CB0000B6A0C6A000E0EEC58F009C517F50AC5F0
:106CC00018F50BC519F50CC51AF50AEC43F017C5F4
:106CD00030F518C531F519C532F51AC533F5000E72
:106CE000346EF00E356E7F0E366E450E376ECCEC80
:106CF0004AF030C566F531C567F532C568F533C56C
:106D000069F566C530F567C531F568C532F569C501
:106D100033F5CD0E346ECC0E356E4C0E366E3F0E06
:106D2000376EC7EC5EF0D8B098EF36F09AEF36F0D9
:106D30009FEF36F0060190919093DEEF36F066C536
:106D400030F567C531F568C532F569C533F5660EAE
:106D5000346E660E356EA60E366E3F0E376EC7EC7D
:106D60005EF0D8B0B6EF36F0B8EF36F0BDEF36F0E3
:106D7000060190919083DEEF36F066C530F567C569
:106D800031F568C532F569C533F5710E346E3D0EC7
:106D9000356EEA0E366E3F0E376EC7EC5EF0D8B039
:106DA000D4EF36F0D6EF36F0DBEF36F00601908107
:106DB0009093DEEF36F00601908190830A0E4CEC42
:106DC0006FF009C564F50AC565F560C51BF561C5B9
:106DD0001CF562C51DF563C51EF564C509F565C5DD
:106DE0000AF50B6A0C6A000E0EEC58F009C517F58F
:106DF0000AC518F50BC519F50CC51AF50AEC43F0D0
:106E000017C530F518C531F519C532F51AC533F572
:106E1000000E346EF00E356E7F0E366E450E376EF8
:106E2000CCEC4AF030C566F531C567F532C568F57A
:106E300033C569F566C530F567C531F568C532F506
:106E400069C533F5CD0E346ECC0E356E4C0E366EF4
:106E50003F0E376EC7EC5EF0D8B031EF37F033EF4E
:106E600037F038EF37F006019095909777EF37F0CD
:106E700066C530F567C531F568C532F569C533F5C6
:106E8000660E346E660E356EA60E366E3F0E376E8B
:106E9000C7EC5EF0D8B04FEF37F051EF37F056EF58
:106EA00037F006019095908777EF37F066C530F59B
:106EB00067C531F568C532F569C533F5710E346EB5
:106EC0003D0E356EEA0E366E3F0E376EC7EC5EF045
:106ED000D8B06DEF37F06FEF37F074EF37F0060191
:106EE0009085909777EF37F00601908590870B0E8D
:106EF0004CEC6FF009C564F50AC565F560C51BF576
:106F000061C51CF562C51DF563C51EF564C509F5AF
:106F100065C50AF50B6A0C6A000E0EEC58F009C53F
:106F200017F50AC518F50BC519F50CC51AF50AECC5
:106F300043F017C530F518C531F519C532F51AC536
:106F400033F5000E346EF00E356E7F0E366E450E44
:106F5000376ECCEC4AF030C566F531C567F532C501
:106F600068F533C569F566C530F567C531F568C59F
:106F700032F569C533F5CD0E346ECC0E356E4C0E40
:106F8000366E3F0E376EC7EC5EF0D8B0CAEF37F002
:106F9000CCEF37F0D1EF37F006019099909B10EFCE
:106FA00038F066C530F567C531F568C532F569C595
:106FB00033F5660E346E660E356EA60E366E3F0ED7
:106FC000376EC7EC5EF0D8B0E8EF37F0EAEF37F095
:106FD000EFEF37F006019099908B10EF38F066C50F
:106FE00030F567C531F568C532F569C533F5710E01
:106FF000346E3D0E356EEA0E366E3F0E376EC7ECC0
:107000005EF0D8B006EF38F008EF38F00DEF38F04A
:1070100006019089909B10EF38F006019089908BC3
:10702000FC51D8B416EF38F018EF38F01EEF38F0F6
:107030009051FF0A906FFC6B12EF39F03F0E9017E2
:107040008E9753509019D8A428EF38F02AEF38F0D3
:107050002CEF38F012EF39F09051531A53A033EF60
:1070600038F035EF38F04AEF38F090A13AEF38F0C9
:107070003CEF38F044EF38F0320E0A6E380E0B6EEB
:10708000C3EC67F04AEF38F0A50E0A6E370E0B6EB0
:10709000C3EC67F053A24FEF38F051EF38F067EFD1
:1070A00038F0060190A357EF38F059EF38F061EF50
:1070B00038F03B0E0A6E380E0B6EC3EC67F067EFCC
:1070C00038F0AF0E0A6E370E0B6EC3EC67F053A4A8
:1070D0006CEF38F06EEF38F084EF38F0060190A5D1
:1070E00074EF38F076EF38F07EEF38F0440E0A6E29
:1070F000380E0B6EC3EC67F084EF38F0B90E0A6EF1
:10710000370E0B6EC3EC67F053A689EF38F08BEFA8
:1071100038F0A1EF38F0060190A791EF38F093EF27
:1071200038F09BEF38F04D0E0A6E380E0B6EC3EC44
:1071300067F0A1EF38F0C30E0A6E370E0B6EC3EC8A
:1071400067F053A8A6EF38F0A8EF38F0BEEF38F09C
:10715000060190A9AEEF38F0B0EF38F0B8EF38F094
:10716000560E0A6E380E0B6EC3EC67F0BEEF38F0A9
:10717000CD0E0A6E370E0B6EC3EC67F053AAC3EF49
:1071800038F0C5EF38F012EF39F0060190ABCBEFD5
:1071900038F0CDEF38F00CEF39F00A6AE90E096EDD
:1071A000010E0B6E9FEC6CF0030E4A6E700E496E72
:1071B0005C0EE82EFED7492EFCD74A2EFAD700D017
:1071C0000601FE51D8B4E7EF38F0E9EF38F003EFED
:1071D00039F0FC0E126EFF0E136E000E146E000ED0
:1071E000156E176A000E166EC6EC64F0FE0E126E77
:1071F000FF0E136E000E146E000E156E176A000E51
:10720000166EC6EC64F0FF005F0E0A6E380E0B6E51
:10721000C3EC67F012EF39F0D70E0A6E370E0B6E23
:10722000C3EC67F012001E6A000E1D6E060190A5E9
:107230001CEF39F01EEF39F029EF39F090A723EF5A
:1072400039F025EF39F029EF39F0020EA16F72EF16
:107250003AF090A52EEF39F030EF39F034EF39F0F5
:10726000010EA16F72EF3AF090A739EF39F03BEFC2
:1072700039F03FEF39F0040EA16F72EF3AF0110EC2
:107280001C6E3C0E1B6ECB0EE82EFED71B2EFCD7C1
:107290001C2EFAD70000246A24C51DF5030E1C6EAF
:1072A000700E1B6E5C0EE82EFED71B2EFCD71C2E1C
:1072B000FAD700D0010E096E010E0A6E1D0E0B6E7C
:1072C000050E0C6E100EBCEC4FF0030E1C6E700E13
:1072D0001B6E5C0EE82EFED71B2EFCD71C2EFAD799
:1072E00000D0010E1D6E000E096E010E0A6E1D0EFD
:1072F0000B6E050E0C6E100EBCEC4FF0030E1C6EE8
:10730000700E1B6E5C0EE82EFED71B2EFCD71C2EBB
:10731000FAD700D0640E096E010E0A6E1F0E0B6EB6
:10732000050E0C6E100E1DEC45F0210E2424D96EB6
:10733000DA6A050EDA221FC5DFF4242A010E24645E
:10734000A4EF39F0A6EF39F04CEF39F0246A210EA2
:107350002424D96EDA6A050EDA22DF50D8A4B3EFFE
:1073600039F0B5EF39F006EF3AF024C51DF5030EFC
:107370001C6E700E1B6E5C0EE82EFED71B2EFCD70B
:107380001C2EFAD700D0010E096E010E0A6E1D0EDA
:107390000B6E050E0C6E110EBCEC4FF0030E1C6E46
:1073A000700E1B6E5C0EE82EFED71B2EFCD71C2E1B
:1073B000FAD700D0010E1D6E000E096E010E0A6E86
:1073C0001D0E0B6E050E0C6E110EBCEC4FF0030E75
:1073D0001C6E700E1B6E5C0EE82EFED71B2EFCD7AB
:1073E0001C2EFAD700D0640E096E010E0A6E1F0E15
:1073F0000B6E050E0C6E110E1DEC45F0210E2424B3
:10740000D96EDA6A050EDA221FC5DFF4242A010ECE
:1074100024640DEF3AF00FEF3AF0A7EF39F0020EC7
:107420002118D8A416EF3AF018EF3AF01DEF3AF011
:10743000020E06019F6F2DEF3AF02104D8A423EF2E
:107440003AF025EF3AF02AEF3AF0010E06019F6F6D
:107450002DEF3AF0040E06019F6F020E2218D8A4F9
:1074600034EF3AF036EF3AF03AEF3AF0020EA06F0E
:1074700048EF3AF02204D8A440EF3AF042EF3AF055
:1074800046EF3AF0010EA06F48EF3AF0040EA06FFD
:107490009F05D8A44EEF3AF050EF3AF05BEF3AF088
:1074A000020EA019D8A457EF3AF059EF3AF05BEF6B
:1074B0003AF025EF39F09F05D8A461EF3AF063EF79
:1074C0003AF065EF3AF030EF39F0020E9F19D8A488
:1074D0006CEF3AF06EEF3AF070EF3AF03BEF39F0C4
:1074E000F00EA16F040EA119D8A479EF3AF07BEF4A
:1074F0003AF0D3EF3AF0010E236E060E126E2350CF
:1075000026EC5DF0200E0A6E000E096E23C50BF509
:107510000D6A0A0E0C6E060E0F6E080E0E6E05EC4E
:107520005CF05450D8B497EF3AF099EF3AF0A4EFEA
:107530003AF0020E2318D8A4A0EF3AF0A2EF3AF0E6
:10754000A4EF3AF0ADEF3AF0232A040E2364ABEF38
:107550003AF0ADEF3AF07DEF3AF05450D8B4B3EFD3
:107560003AF0B5EF3AF0BAEF3AF0010E0601D56FF6
:10757000BDEF3AF0010E0501F86F860E096E080E98
:107580000A6E3F0E0B6E390E0C6E43EC6EF0390E28
:10759000096E070E0A6E3F0E0B6E390E0C6E43EC31
:1075A0006EF07BEF3BF0020EA119D8A4DAEF3AF0AF
:1075B000DCEF3AF029EF3BF0050E126E010E26ECDF
:1075C0005DF0060E126E020E26EC5DF0200E0A6EC5
:1075D000000E096E020E0B6E0D6A0A0E0C6E060E80
:1075E0000F6E080E0E6E05EC5CF00601D851D8B493
:1075F000FCEF3AF0FEEF3AF017EF3BF0050E126E9B
:10760000030E26EC5DF0060E126E040E26EC5DF005
:10761000200E0A6E000E096E040E0B6E0D6A0A0E25
:107620000C6E060E0F6E080E0E6E05EC5CF05450DC
:10763000D8B41DEF3BF01FEF3BF024EF3BF0010E01
:107640000601D46F7BEF3BF0010E0601D76F7BEF95
:107650003BF0A105D8B42FEF3BF031EF3BF03AEF10
:107660003BF0F00EA119D8A438EF3BF03AEF3BF015
:107670007BEF3BF0050E126E010E26EC5DF0050E61
:10768000126E020E26EC5DF00601D851D8B44BEF15
:107690003BF04DEF3BF057EF3BF0050E126E030E43
:1076A00026EC5DF0050E126E040E26EC5DF05450D3
:1076B000D8B45DEF3BF05FEF3BF064EF3BF0010EC1
:1076C0000601D66F67EF3BF0010E0501F96F7C0EE6
:1076D000096E080E0A6E330E0B6E390E0C6E43ECFB
:1076E0006EF02F0E096E070E0A6E330E0B6E390EFA
:1076F0000C6E43EC6EF00501F951D8B482EF3BF00B
:1077000084EF3BF090EF3BF0010E096E080E0A6E1D
:107710006D0E0B6E340E0C6E43EC6EF0F3EF3BF01F
:10772000F851D8B496EF3BF098EF3BF0A4EF3BF064
:10773000010E096E080E0A6E530E0B6E340E0C6E9F
:1077400043EC6EF0F3EF3BF00601D651D8B4ABEF4B
:107750003BF0ADEF3BF0B9EF3BF0010E096E080EC8
:107760000A6EBB0E0B6E340E0C6E43EC6EF0F3EF34
:107770003BF0D551D8B4BFEF3BF0C1EF3BF0CDEFBC
:107780003BF0010E096E080E0A6EA10E0B6E340E50
:107790000C6E43EC6EF0F3EF3BF0D751D8B4D3EF5F
:1077A0003BF0D5EF3BF0E1EF3BF0010E096E080E28
:1077B0000A6ED10E0B6E330E0C6E43EC6EF0F3EFCF
:1077C0003BF0D451D8B4E7EF3BF0E9EF3BF0F3EFF7
:1077D0003BF0010E096E080E0A6E870E0B6E340E1A
:1077E0000C6E43EC6EF012000501E06BE06B600E76
:1077F000E025D96EDA6A050EDA22DF6AE02B7F0E09
:10780000E06505EF3CF007EF3CF0F7EF3BF00601D9
:1078100090A10DEF3CF00FEF3CF070EF3CF0050154
:10782000F951D8B416EF3CF018EF3CF01EEF3CF0E5
:10783000620EE16F370EE26FCFEF3CF0F851D8B433
:1078400024EF3CF026EF3CF02CEF3CF02E0EE16FE5
:10785000370EE26FCFEF3CF00601D751D8B433EFCB
:107860003CF035EF3CF03CEF3CF0B00E0501E16F31
:10787000360EE26FCFEF3CF0D651D8B442EF3CF079
:1078800044EF3CF04BEF3CF0480E0501E16F370E42
:10789000E26FCFEF3CF0D551D8B451EF3CF053EF4D
:1078A0003CF05AEF3CF0140E0501E16F370EE26F29
:1078B000CFEF3CF0D451D8B460EF3CF062EF3CF035
:1078C00069EF3CF0920E0501E16F360EE26FCFEFEB
:1078D0003CF0EB0E0501E16F360EE26FCFEF3CF0AE
:1078E0000501F951D8B477EF3CF079EF3CF07FEF28
:1078F0003CF0550EE16F370EE26FCFEF3CF0F851E0
:10790000D8B485EF3CF087EF3CF08DEF3CF0210ED2
:10791000E16F370EE26FCFEF3CF00601D751D8B4DC
:1079200094EF3CF096EF3CF09DEF3CF0A10E05018A
:10793000E16F360EE26FCFEF3CF0D651D8B4A3EF33
:107940003CF0A5EF3CF0ACEF3CF03B0E0501E16FE5
:10795000370EE26FCFEF3CF0D551D8B4B2EF3CF028
:10796000B4EF3CF0BBEF3CF0070E0501E16F370EC2
:10797000E26FCFEF3CF0D451D8B4C1EF3CF0C3EF8D
:107980003CF0CAEF3CF0830E0501E16F360EE26F6A
:10799000CFEF3CF0DD0E0501E16F360EE26F600EB9
:1079A0000D6E050E0E6EE1C50FF5E2C510F5E1C5D1
:1079B00009F5E2C50AF528EC6CF009C511F50AC510
:1079C00012F5F6EC69F00501F951D8B4EAEF3CF094
:1079D000ECEF3CF0F2EF3CF0070EE16F350EE26F9A
:1079E0003BEF3DF0F851D8B4F8EF3CF0FAEF3CF043
:1079F00000EF3DF0EE0EE16F340EE26F3BEF3DF035
:107A00000601D651D8B407EF3DF009EF3DF010EF75
:107A10003DF0BB0E0501E16F340EE26F3BEF3DF030
:107A2000D551D8B416EF3DF018EF3DF01FEF3DF003
:107A3000A10E0501E16F340EE26F3BEF3DF0D7512F
:107A4000D8B425EF3DF027EF3DF02EEF3DF0510E7D
:107A50000501E16F350EE26F3BEF3DF0D451D8B434
:107A600034EF3DF036EF3DF03BEF3DF0870E050182
:107A7000E16F340EE26F700E0D6E050E0E6EE1C5F5
:107A80000FF5E2C510F5E1C509F5E2C50AF528ECE8
:107A90006CF009C511F50AC512F5F6EC69F00A6A31
:107AA000090E096EFCEC70F00501906F0A6A0A0E6F
:107AB000096EFCEC70F00501916F0A6A0B0E096EFD
:107AC000FCEC70F00501926F0A6A0C0E096EFCEC7A
:107AD00070F00501936FD10EF66E380EF76EF86AEE
:107AE0000800F5C494F5D20EF66E380EF76EF86AFB
:107AF0000800F5C495F5D30EF66E380EF76EF86AE9
:107B00000800F5C496F5D40EF66E380EF76EF86AD6
:107B10000800F5C497F5D50EF66E380EF76EF86AC4
:107B20000800F5C498F5D60EF66E380EF76EF86AB2
:107B30000800F5C499F5D70EF66E380EF76EF86AA0
:107B40000800F5C49AF5D80EF66E380EF76EF86A8E
:107B50000800F5C49BF50A6A000E096EFCEC70F093
:107B600005019C6F0A6A010E096EFCEC70F00501BC
:107B70009D6F0A6A020E096EFCEC70F005019E6FA3
:107B80000A6A030E096EFCEC70F005019F6F0A6A29
:107B9000040E096EFCEC70F00501A06F0A6A050E78
:107BA000096EFCEC70F00501A16F0A6A060E096E01
:107BB000FCEC70F00501A26F0A6A070E096EFCEC7E
:107BC00070F00501A36F0A6A080E096EFCEC70F0F4
:107BD0000501A46F0A6AE00E096EFCEC70F0050165
:107BE000A66F0A6AE20E096EFCEC70F00501A76F41
:107BF0000A6AE10E096EFCEC70F00501A86F0A6AD2
:107C0000E30E096EFCEC70F00501A96F0A6AE40E40
:107C1000096EFCEC70F00501AA6F1B0EC46F1B0E01
:107C2000C56F1B0EC66F1B0EC76F1A0EC86F100EE6
:107C3000C96F100ECA6F120ECB6F110ECC6FF7C545
:107C4000E0F53BEF3EF07F0EE06529EF3EF02BEFD5
:107C50003EF030EF3EF0000E90EC70F039EF3EF069
:107C6000600EE025D96EDA6A050EDA22DF5090EC5C
:107C700070F00501E02BE051186E196AF651F7C556
:107C80001AF51B6A1A26000E1B22FF0E1A241C6E00
:107C9000FF0E1B201D6E18501C5C1D50800A1E6EAE
:107CA0001950800A1E58D8B058EF3EF05AEF3EF0F7
:107CB00023EF3EF012000C50800B156E0C500C247C
:107CC000176E0BAE66EF3EF068EF3EF069EF3EF0E8
:107CD00017801750D8B46FEF3EF071EF3EF085EF8C
:107CE0003EF01728D8A477EF3EF079EF3EF081EF11
:107CF0003EF0000E096E000E0A6E000E0B6E000EB6
:107D00000C6E0B8E0C6A8DEF3EF0000E096E000EAD
:107D10000A6E000E0B6E000E0C6E1050800B166E6D
:107D200015501618D8B497EF3EF099EF3EF09AEF41
:107D30003EF0158C10501024166E0FAEA2EF3EF0E0
:107D4000A4EF3EF0A5EF3EF016801650D8B4ABEF8E
:107D50003EF0ADEF3EF0C1EF3EF01628D8A4B3EFF1
:107D60003EF0B5EF3EF0BDEF3EF0000E0D6E000EA2
:107D70000E6E000E0F6E000E106E0F8E106AC9EFA1
:107D80003EF0000E0D6E000E0E6E000E0F6E000E19
:107D9000106E1750165CD8B0D0EF3EF0D2EF3EF028
:107DA000F9EF3EF015ACD7EF3EF0D9EF3EF0DBEF48
:107DB0003EF0800E151A17C518F516C517F518C52B
:107DC00016F509C518F50DC509F518C50DF50AC54F
:107DD00018F50EC50AF518C50EF50BC518F50FC533
:107DE0000BF518C50FF50CC518F510C50CF518C521
:107DF00010F5186A175016C511F5126A115E000EBB
:107E0000125A12BE0DEF3FF0125009E11A0E115C2A
:107E1000D8A00DEF3FF00FEF3FF046EF3FF00950D5
:107E20000A100B100C10D8A418EF3FF01BEF3FF016
:107E3000010E1CEF3FF0000E186E000E096E000ED2
:107E40000A6E000E0B6E000E0C6E16C517F54FEF86
:107E50003FF018A02EEF3FF030EF3FF036EF3FF04D
:107E6000D89018300109186E38EF3FF0D8901832CA
:107E700009A03DEF3FF03FEF3FF040EF3FF0188E9D
:107E80000C340C320B320A320932172A1650175CA6
:107E9000D8A04DEF3FF04FEF3FF029EF3FF015BC7A
:107EA00054EF3FF056EF3FF096EF3FF01750D8A455
:107EB0005CEF3FF05EEF3FF068EF3FF0000E096EC1
:107EC000000E0A6E000E0B6E000E0C6EB5EF40F049
:107ED0000D5009260E500A220F500B2210500C2272
:107EE0000CA075EF3FF077EF3FF023EF40F018A0C4
:107EF0007CEF3FF07EEF3FF084EF3FF0D8901830FA
:107F00000109186E86EF3FF0D890183209A08BEF68
:107F10003FF08DEF3FF08EEF3FF0188E0C340C32B7
:107F20000B320A320932172A23EF40F00D50095C58
:107F30000E500A580F500B580C50800A116E1050FA
:107F4000800A1158D8B0A7EF3FF0A9EF3FF0D4EF67
:107F50003FF009500D5C116E0A500E58126E0B5016
:107F60000F58136E0C501058146EFF0E1124096E2A
:107F7000FF0E12200A6EFF0E13200B6EFF0E142050
:107F80000C6E800E151A186C1850D8A4CAEF3FF06A
:107F9000CCEF3FF0DCEF3FF0010E0926000E0A2285
:107FA0000B220C22DCEF3FF00D50095E0E500A5AF6
:107FB0000F500B5A10500C5A09500A100B100C108D
:107FC000D8A4E5EF3FF0E7EF3FF01CEF40F018508A
:107FD000D8A4EDEF3FF0EFEF3FF01CEF40F0000EC4
:107FE000096E000E0A6E000E0B6E000E0C6EB5EFE1
:107FF00040F0D89009360A360B360C3618AE03EF2F
:1080000040F005EF40F006EF40F0098018A00BEFBC
:1080100040F00DEF40F011EF40F0D880183613EF2C
:1080200040F0D89018361750D8B419EF40F01BEF35
:1080300040F01CEF40F017060BAE21EF40F023EFAD
:1080400040F0F9EF3FF0166A18AE29EF40F02BEF41
:1080500040F043EF40F018C511F57F0E1116D8B46B
:1080600034EF40F036EF40F03AEF40F0010E166E7C
:1080700043EF40F009A03FEF40F041EF40F043EF05
:1080800040F036EF40F01650D8B449EF40F04BEFD7
:1080900040F076EF40F0010E0926000E0A220B2276
:1080A0000C220CA056EF40F058EF40F076EF40F075
:1080B00009C511F50AC512F50BC513F50CC514F564
:1080C0001434143213321232113211C509F512C5AB
:1080D0000AF513C50BF514C50CF51728D8B473EFC2
:1080E00040F075EF40F076EF40F0172A1728D8B42B
:1080F0007CEF40F07EEF40F086EF40F01750D8A4C0
:1081000084EF40F086EF40F097EF40F0000E096EEC
:10811000000E0A6E000E0B6E000E0C6E1750D8A4E7
:1081200094EF40F096EF40F097EF40F0156A17A0FB
:108130009CEF40F09EEF40F0A1EF40F00B8EA2EFDD
:1081400040F00B9ED89017300C6E15AEAAEF40F0A1
:10815000ACEF40F0ADEF40F00C8E09C509F50AC553
:108160000AF50BC50BF50CC50CF51200246E1E6A42
:108170001750D8B4BEEF40F0C0EF40F0C7EF40F06A
:10818000050E126E245026EC5DF0CCEF40F0060E8A
:10819000126E245026EC5DF0190E1B6E5A0E1A6EEC
:1081A000B20EE82EFED71A2EFCD71B2EFAD72404C7
:1081B000D8A4DDEF40F0DFEF40F0E7EF40F0EB0E4A
:1081C0000A6E330E0B6EC3EC67F018EF41F0020E2F
:1081D0002418D8A4EEEF40F0F0EF40F0F8EF40F0B4
:1081E000050E0A6E340E0B6EC3EC67F018EF41F00B
:1081F000030E2418D8A4FFEF40F001EF41F009EF7F
:1082000041F01F0E0A6E340E0B6EC3EC67F018EFD0
:1082100041F0040E2418D8A410EF41F012EF41F001
:1082200018EF41F0390E0A6E340E0B6EC3EC67F096
:108230000A6A870E096E2450BCEC59F009C51CF57A
:108240000AC51DF51C50070B206E2050D8A42BEF3B
:1082500041F02DEF41F035EF41F0200E0A6E380E5F
:108260000B6EC3EC67F0C9EF41F02004D8A43BEFDC
:1082700041F03DEF41F045EF41F0EB0E0A6E380E54
:108280000B6EC3EC67F0C9EF41F0020E2018D8A4C2
:108290004CEF41F04EEF41F056EF41F0490E0A6EBF
:1082A000390E0B6EC3EC67F0C9EF41F0030E2018D6
:1082B000D8A45DEF41F05FEF41F077EF41F0185047
:1082C000D8B465EF41F067EF41F06FEF41F0460E33
:1082D0000A6E390E0B6EC3EC67F0C9EF41F0460E23
:1082E0000A6E390E0B6EC3EC67F0C9EF41F0040E55
:1082F0002018D8A47EEF41F080EF41F088EF41F0E4
:108300004C0E0A6E390E0B6EC3EC67F0C9EF41F0EC
:10831000050E2018D8A48FEF41F091EF41F099EFAE
:1083200041F04F0E0A6E390E0B6EC3EC67F0C9EFC9
:1083300041F0060E2018D8A4A0EF41F0A2EF41F0C2
:10834000BAEF41F01850D8B4A8EF41F0AAEF41F0CD
:10835000B2EF41F03B0E0A6E390E0B6EC3EC67F0C4
:10836000C9EF41F03B0E0A6E390E0B6EC3EC67F09D
:10837000C9EF41F0070E2018D8A4C1EF41F0C3EFB8
:1083800041F0C9EF41F0290E0A6E380E0B6EC3ECB6
:1083900067F07A0E0A6E330E0B6EC3EC67F019505D
:1083A000D8B4D5EF41F0D7EF41F0E7EF41F0200E20
:1083B0000A6E000E096E24C50BF50D6A500E0C6E88
:1083C000190E0F6E0E6805EC5CF0F5EF41F0200E13
:1083D0000A6E000E096E24C50BF50D6A500E0C6E68
:1083E000090E0F6E0E6805EC5CF0200E0A6E000E92
:1083F000096E24C50BF50D6A510E0C6E010E0F6E41
:10840000010E0E6E05EC5CF0200E0A6E000E096E79
:1084100024C50BF50D6A890E0C6E0F6A000E0E6EE8
:1084200005EC5CF0D00E1A6ECA0EE82EFED71A2E9E
:10843000FCD70A6A8A0E096E2450BCEC59F009C5B3
:1084400022F50AC523F5030E2216000E2316030E8D
:1084500022182310D8A42FEF42F031EF42F084EF1E
:1084600042F0200E0A6E000E096E24C50BF50D6A4F
:10847000510E0C6E0F6A000E0E6E05EC5CF00A6A6F
:108480008A0E096E2450BCEC59F009C522F50AC5C4
:1084900023F51F6A73EF42F00A6A8A0E096E2450B0
:1084A000BCEC59F009C522F50AC523F5030E2216C6
:1084B000000E2316D00E1A6ECA0EE82EFED71A2E04
:1084C000FCD71F2A0F0E1F18D8A469EF42F06BEFDC
:1084D00042F073EF42F0A30E0A6E380E0B6EC3EC3F
:1084E00067F009EF43F022502310D8A47AEF42F04E
:1084F0007CEF42F04CEF42F0520E0A6E360E0B6EDD
:10850000C3EC67F009EF43F022042310D8A48BEFEB
:1085100042F08DEF42F08FEF42F012EF42F0020E88
:1085200022182310D8B497EF42F099EF42F09BEF56
:1085300042F012EF42F0200E0A6E000E096E24C5C2
:108540000BF50D6A510E0C6E010E0F6E000E0E6EC5
:1085500005EC5CF00A6A8A0E096E2450BCEC59F0F6
:1085600009C522F50AC523F5030E2216000E2316AF
:1085700022502310D8A4BFEF42F0C1EF42F000EF29
:1085800043F0230E0A6E320E0B6EC3EC67F00A6ADC
:10859000890E096E2450BCEC59F009C522F50AC5B4
:1085A00023F522C50CF523C50DF504EC6FF009EF9A
:1085B00043F00A6A8A0E096E2450BCEC59F009C5D2
:1085C00022F50AC523F5030E2216000E2316D00E3F
:1085D0001A6ECA0EE82EFED71A2EFCD71E2A0F0ED0
:1085E0001E18D8A4F6EF42F0F8EF42F000EF43F087
:1085F000F30E0A6E370E0B6EC3EC67F009EF43F013
:1086000022502310D8A407EF43F009EF43F0D9EF2D
:1086100042F012001A50800B236E1A501A24296E51
:1086200019AE15EF43F017EF43F018EF43F0298030
:108630002950D8B41EEF43F020EF43F033EF43F05E
:108640002928D8A426EF43F028EF43F030EF43F079
:10865000000E176E000E186E000E196E000E1A6EC8
:10866000198E3BEF43F0000E176E000E186E000ED1
:10867000196E000E1A6E1E50800B231A1E501E24F7
:10868000246E1DAE46EF43F048EF43F049EF43F050
:1086900024802450D8B44FEF43F051EF43F064EFFF
:1086A00043F02428D8A457EF43F059EF43F061EF8B
:1086B00043F0000E1B6E000E1C6E000E1D6E000EB1
:1086C0001E6E1D8E6CEF43F0000E1B6E000E1C6EB6
:1086D000000E1D6E000E1E6E2450D8B472EF43F0D3
:1086E00074EF43F07CEF43F02950D8A47AEF43F0C5
:1086F0007CEF43F086EF43F0000E176E000E186E0D
:10870000000E196E000E1A6E1CEF45F01D50170278
:10871000F3C42EF5F4C42FF52E50256E266A276A71
:10872000286A2F502A6E2B6A2C6A2D6A1C50180258
:10873000F3C42EF5F4C42FF52E502526000E262264
:10874000272228222F502A26000E2B222C222D22CF
:108750001B501902F3C42EF5F4C42FF52E50252614
:10876000000E2622272228222F502A26000E2B22F6
:108770002C222D2227C528F526C527F525C526F547
:10878000256A1B501802F3C42EF5F4C42FF52E50A1
:1087900025262F502622000E2722000E28221C50AC
:1087A0001702F3C42EF5F4C42FF52E5025262F50B2
:1087B0002622000E2722000E282227C528F526C5CE
:1087C00027F525C526F5256A1B501702F3C42EF59B
:1087D000F4C42FF52E5025262F502622000E2722D6
:1087E000000E28221D501802F3C42EF5F4C42FF5F4
:1087F0002E502A262F502B22000E2C22000E2D2226
:108800001C501902F3C42EF5F4C42FF52E502A265D
:108810002F502B22000E2C22000E2D221D5019024B
:10882000F3C42EF5F4C42FF52E501F6E2F50206E7A
:10883000216A226A21C522F520C521F51FC520F530
:108840001F6A1F502A2620502B2221502C222250F2
:108850002D2225C51FF526C520F527C521F528C5DC
:1088600022F5190E39EF44F0D8902232213220320D
:108870001F32E82E34EF44F01F502A2620502B22BE
:1088800021502C2222502D2227C528F526C527F558
:1088900025C526F5256A245029C51FF5206A1F26FF
:1088A000000E2022820E1F242E6EFF0E20202F6E1F
:1088B0006FEF44F0D8902A362B362C362D3628AE62
:1088C00064EF44F066EF44F067EF44F02A80D890FC
:1088D00025362636273628362E06D8A02F062CAE6B
:1088E00074EF44F076EF44F05AEF44F0246A28AE77
:1088F0007CEF44F07EEF44F0A2EF44F0FF0E25142D
:108900001F6EFF0E2614206EFF0E2714216E7F0EA1
:108910002814226E1F50201021102210D8B493EF7B
:1089200044F095EF44F099EF44F0010E246EA2EF6D
:1089300044F02AA09EEF44F0A0EF44F0A2EF44F0F0
:1089400095EF44F02450D8B4A8EF44F0AAEF44F0D7
:10895000CEEF44F0010E2A26000E2B222C222D22CF
:108960002DA0B5EF44F0B7EF44F0CEEF44F02AC5A8
:108970001FF52BC520F52CC521F52DC522F5223478
:108980002232213220321F321FC52AF520C52BF595
:1089900021C52CF522C52DF52E4A2F2A2FBED9EF41
:1089A00044F02F5008E12E28D8A0D9EF44F0DBEF97
:1089B00044F0E5EF44F0000E2A6E000E2B6E800EA0
:1089C0002C6E7F0E2D6E12EF45F02FBEF2EF44F0AD
:1089D0002F5006E12E04D8B0F0EF44F0F2EF44F04F
:1089E000FDEF44F0000E2A6E000E2B6E000E2C6E72
:1089F000000E2D6E236A12EF45F02EC529F5FF0EED
:108A00002A16FF0E2B167F0E2C16000E2D1629A0EF
:108A10000CEF45F00EEF45F00FEF45F02C8ED8909F
:108A200029302D6E23502D122AC517F52BC518F5A8
:108A30002CC519F52DC51AF51200136E156A000E16
:108A4000146E116A000E106E176A000E166E135027
:108A500000080D6E09500D5C0E6E0A500E5CFE0F84
:108A6000126E122A56EF45F0E40E00D000D0E82E28
:108A7000FCD700D000D0164A172A17BE49EF45F0A0
:108A8000D00E165C070E1758D8A049EF45F04BEFF3
:108A900045F056EF45F0BE94C094BE8E0BC5D9F498
:108AA0000CC5DAF4FB0EDF6E2DEF47F0CEA65BEFC0
:108AB00045F05DEF45F034EF45F0BE92BE9EE40E0A
:108AC00000D000D0E82EFCD700D000D0010E526EAE
:108AD000070E52646EEF45F070EF45F08BEF45F0F6
:108AE000E4EF45F0010E0601CF6FAAEF45F013C584
:108AF000CFF6AAEF45F009C5CFF6AAEF45F00AC5B3
:108B0000CFF6AAEF45F00601CF6BAAEF45F012C5EC
:108B1000CFF6AAEF45F05250010AD8B472EF45F0F3
:108B2000030AD8B477EF45F0010AD8B47BEF45F0DB
:108B3000070AD8B47FEF45F0010AD8B483EF45F0B7
:108B4000030AD8B483EF45F0010AD8B487EF45F0A3
:108B5000AAEF45F0BE94516A070E5164B2EF45F09A
:108B6000B4EF45F0B6EF45F0E1EF45F00601CFBFB9
:108B7000BCEF45F0C0EF45F00D6A0D2AC1EF45F09E
:108B80000D6A0D460D46C0500D18FB0B0D18C06E3A
:108B90000601CF51CF25CF6FB60E00D000D0E82E02
:108BA000FCD700D000D000D0BE84B60E00D000D0DC
:108BB000E82EFCD700D000D000D0BE94512AACEFF4
:108BC00045F0522A68EF45F0BE8EE40E00D000D08A
:108BD000E82EFCD700D000D02BEF46F0E40E00D0FA
:108BE00000D0E82EFCD700D000D0164A172A17BEB6
:108BF00003EF46F0D00E165C070E1758D8A003EF0F
:108C000046F005EF46F02BEF46F0BE94C094BE8EC2
:108C1000196A000E186E17EF46F018500B24D96E23
:108C200019500C20DA6EFF0EDF6E184A192A0A500E
:108C30000D6E0E6A0D50185C1950800A0F6E0E50A2
:108C4000800A0F58D8A027EF46F029EF46F00DEF25
:108C500046F02DEF47F0CEA630EF46F032EF46F06B
:108C6000EEEF45F0BE9E196A000E186E86EF46F0D4
:108C7000516A070E51643FEF46F041EF46F043EF73
:108C800046F084EF46F0BE94B60E00D000D0E82E39
:108C9000FCD700D000D000D0BE84B60E00D000D0EB
:108CA000E82EFCD700D000D000D0CEA85AEF46F076
:108CB0005CEF46F070EF46F018500B24D96E195057
:108CC0000C20DA6E18500B24E16E19500C20E26E65
:108CD000E7500D6ED8900D34FE0BDF6E81EF46F03D
:108CE00018500B24D96E19500C20DA6E18500B2432
:108CF000E16E19500C20E26EE7500D6ED8800D34F5
:108D0000DF6E512A39EF46F0184A192A0A500D6EC3
:108D10000E6A0D50185C1950800A0F6E0E50800AB2
:108D20000F58D8A096EF46F098EF46F038EF46F08F
:108D3000196A000E186E516A070E5164A2EF46F0D0
:108D4000A4EF46F0A6EF46F0F5EF46F0BE94B60E5F
:108D500000D000D0E82EFCD700D000D000D0BE84D8
:108D6000B60E00D000D0E82EFCD700D000D000D046
:108D7000CEA8BDEF46F0BFEF46F0DAEF46F0185050
:108D8000080DF3C40DF5010E0D2614C50EF515C51D
:108D90000FF50D2ACFEF46F0D8900E360F360D2E78
:108DA000CCEF46F0FE0E0E14146EFF0E0F14156E6F
:108DB000F2EF46F01850080DF3C40DF5010E0D2624
:108DC00014C50EF515C50FF50D2AEAEF46F0D8903B
:108DD0000E360F360D2EE7EF46F0010E0E10146E14
:108DE0000F50156E512A9CEF46F0184A192A19BEE9
:108DF00003EF47F0195009E1020E185CD8A003EF09
:108E000047F005EF47F09BEF46F0196A000E186E29
:108E100018EF47F018500B24D96E19500C20DA6E59
:108E2000DF500D6E0D501026000E1122184A192A1F
:108E30000A500D6E0E6A0D50185C1950800A0F6EA4
:108E40000E50800A0F58D8A028EF47F02AEF47F0BD
:108E50000AEF47F0BE94C094BE8E12000501AD6BC0
:108E6000000EAC6FA5C5D9F4A6C5DAF4DEC4F6F4DD
:108E7000DDC4F7F4F86A0800F550250AD8A443EFDA
:108E800047F045EF47F0E4EF48F0A5C5D9F4A6C593
:108E9000DAF4DE2A000EDD220601B76B000EB66F93
:108EA000B6C6C6F6B869B969A5C5D9F4A6C5DAF4D7
:108EB000DEC4B2F5DDC4B3F5B2C5F6F4B3C5F7F45C
:108EC000F86A0800F550640AD8B469EF47F06BEF10
:108ED00047F07AEF47F0B2C5F6F4B3C5F7F4F86A95
:108EE0000800F550690AD8A478EF47F07AEF47F008
:108EF00022EF48F0A7C5D9F4A8C5DAF4DFC4A9F574
:108F0000020EDE26DFC4AAF5000EDD22A9C5D9F4C3
:108F1000AAC5DAF4DEC4AEF5DDC4AFF5010E050175
:108F2000B225A96F000EB321AA6FA5C5D9F4A6C5B5
:108F3000DAF4A9C5DEF4AAC5DDF4500EB46FAFBFF4
:108F4000A4EF47F0A7EF47F0010EA8EF47F0000E9F
:108F5000AB6FB4079C0EB425D96EDA6A080EDA221C
:108F6000AEC509F5AFC50AF50C6A0A0E0B6E1EEC0C
:108F700063F009C50FF50AC510F5EAEC6EF00F5065
:108F8000300FDF6EAEC509F5AFC50AF50C6A0A0EE3
:108F90000B6E07EC62F009C5AEF50AC5AFF5050129
:108FA000AC4BAD2BAE51AF11D8B4D9EF47F0DBEFDE
:108FB00047F0E3EF47F0B451D8A4E1EF47F0E3EF17
:108FC00047F0A9EF47F0B451D8B4E9EF47F0EBEF21
:108FD00047F013EF48F0AB51D8B4F1EF47F0F3EF9F
:108FE00047F013EF48F0B4079C0EB425D96EDA6A47
:108FF000080EDA222D0EDF6EAC4BAD2B13EF48F0CE
:109000009C0EB425D96EDA6A080EDA22DF50A96FF9
:10901000A951096E0A6AA3C50BF5A4C50CF5A2EC0B
:1090200061F00501B42B500EB419D8A41AEF48F022
:109030001CEF48F000EF48F0ACC5A3F5ADC5A4F5B2
:1090400002EF49F0A5C5D9F4A6C5DAF4DEC4B2F53D
:10905000DDC4B3F5B2C5F6F4B3C5F7F4F86A080099
:10906000F5C4B4F53FEF48F0B24BB32B4FEF48F0E7
:109070006C0EB46F4FEF48F0B46B4FEF48F0050142
:10908000B4514C0AD8B434EF48F02A0AD8B438EFB7
:1090900048F00A0AD8B434EF48F03CEF48F0B2C5C3
:1090A000F6F4B3C5F7F4F86A0800F550660AD8A4D8
:1090B0005CEF48F05EEF48F0D8EF48F094EF48F0EE
:1090C000A7C5D9F4A8C5DAF4DFC4A9F5040EDE26D5
:1090D000DFC4AAF5000EDD22A9C5D9F4AAC5DAF4C9
:1090E000DEC4AEF5DEC4AFF5DEC4B0F5DEC4B1F566
:1090F0009FEF48F0A7C5D9F4A8C5DAF4DFC4A9F5F5
:10910000040EDE26DFC4AAF5000EDD22A9C5D9F4BF
:10911000AAC5DAF4DEC4AEF5DEC4AFF5DEC4B0F540
:10912000DEC4B1F59FEF48F0B4514C0AD8B47AEFE1
:1091300048F0200AD8B460EF48F09FEF48F0010EE5
:10914000B225A96F000EB321AA6FA5C5D9F4A6C593
:10915000DAF4A9C5DEF4AAC5DDF4CBEF48F0A3C567
:1091600070F5A4C571F5AEC572F5AFC573F5B0C5A0
:1091700074F5B1C575F5B2C5F6F4B3C5F7F4F86A80
:109180000800F5C476F511EC2AF070C5A3F571C599
:10919000A4F502EF49F0B2C5F6F4B3C5F7F4F86AE6
:1091A0000800F550660AD8B4AFEF48F0D8EF48F0A1
:1091B000A5C5D9F4A6C5DAF4DE2A000EDD22A46B1B
:1091C000000EA36F02EF49F0A5C5D9F4A6C5DAF4E5
:1091D000DEC4F6F4DDC4F7F4F86A0800F550096E51
:1091E0000A6AA3C50BF5A4C50CF5A2EC61F0A5C5F0
:1091F000D9F4A6C5DAF4DE2A000EDD220501A46B3F
:10920000010EA36F12001C6E1750D8B40AEF49F07C
:109210000CEF49F013EF49F0060E126E1C5026ECCD
:109220005DF018EF49F0050E126E1C5026EC5DF053
:10923000010E1B6E1850D8B420EF49F022EF49F010
:1092400048EF49F0200E0A6E000E096E1BC50BF5A3
:109250000D6A060E0C6E0F6A0D0E0E6E05EC5CF0BC
:10926000680E196EE40EE82EFED7192EFCD700D03A
:10927000200E0A6E000E096E1BC50BF50D6A060E58
:109280000C6E0F6A0C0E0E6E05EC5CF06CEF49F084
:10929000200E0A6E000E096E1BC50BF50D6A060E38
:1092A0000C6E0F6A070E0E6E05EC5CF0680E196E00
:1092B000E40EE82EFED7192EFCD700D0200E0A6E41
:1092C000000E096E1BC50BF50D6A060E0C6E0F6ABB
:1092D000060E0E6E05EC5CF0200E0A6E000E096E96
:1092E0001BC50BF50D6A0A0E0C6E1F0E0F6E080ED5
:1092F0000E6E05EC5CF01B2A040E1B6482EF49F035
:1093000084EF49F01AEF49F0050E1A6E0F0E196E30
:10931000F10EE82EFED7192EFCD71A2EFAD7000030
:10932000AA0E0A6E380E0B6EC3EC67F01C04D8A4AC
:109330009CEF49F09EEF49F0A6EF49F0970E0A6EB8
:10934000320E0B6EC3EC67F0D7EF49F0020E1C181B
:10935000D8A4ADEF49F0AFEF49F0B7EF49F0BA0E3E
:109360000A6E320E0B6EC3EC67F0D7EF49F0030EB6
:109370001C18D8A4BEEF49F0C0EF49F0C8EF49F07F
:10938000D40E0A6E380E0B6EC3EC67F0D7EF49F0BF
:10939000040E1C18D8A4CFEF49F0D1EF49F0D7EF55
:1093A00049F05A0E0A6E390E0B6EC3EC67F0175077
:1093B000D8B4DDEF49F0DFEF49F0F6EF49F0200EC9
:1093C0000A6E000E096E1CC50BF50D6A480E0C6E78
:1093D000010E0F6E020E0E6E05EC5CF07E0E0A6E34
:1093E000330E0B6EC3EC67F00BEF4AF0200E0A6EE3
:1093F000000E096E1CC50BF50D6A480E0C6E010EB1
:109400000F6E010E0E6E05EC5CF0600E0A6E330EF0
:109410000B6EC3EC67F0200E0A6E000E096E1CC5C1
:109420000BF50D6A030E0C6E0F6A000E0E6E05EC46
:109430005CF0200E0A6E000E096E1CC50BF50D6A5D
:109440004A0E0C6E0F6A000E0E6E05EC5CF0200EDC
:109450000A6E000E096E1CC50BF50D6A030E0C6E2C
:109460000F6A000E0E6E05EC5CF0200E0A6E000E08
:10947000096E1CC50BF50D6A4A0E0C6E0F6A000EC4
:109480000E6E05EC5CF01750D8B449EF4AF04BEF84
:109490004AF083EF4AF0200E0A6E000E096E1CC5DA
:1094A0000BF50D6A490E0C6E0F6A040E0E6E05EC7C
:1094B0005CF01850D8B45FEF4AF061EF4AF072EFF9
:1094C0004AF0200E0A6E000E096E1CC50BF50D6ADF
:1094D0004B0E0C6E050E0F6E040E0E6E05EC5CF05E
:1094E00091EF4AF0200E0A6E000E096E1CC50BF5B6
:1094F0000D6A4B0E0C6E050E0F6E020E0E6E05EC15
:109500005CF091EF4AF0200E0A6E000E096E1CC549
:109510000BF50D6A490E0C6E0F6A010E0E6E05EC0E
:109520005CF01850D8B497EF4AF099EF4AF0AAEFE0
:109530004AF0200E0A6E000E096E1CC50BF50D6A6E
:10954000520E0C6E030E0F6E060E0E6E05EC5CF0E6
:10955000B9EF4AF0200E0A6E000E096E1CC50BF51D
:109560000D6A520E0C6E030E0F6E030E0E6E05EC9E
:109570005CF0B80E0A6E380E0B6EC3EC67F0090E85
:109580001A6E1E0E196EE40EE82EFED7192EFCD7A9
:109590001A2EFAD700D012003350800B406E335091
:1095A0003324476E32AED7EF4AF0D9EF4AF0DAEF04
:1095B0004AF047804750D8B4E0EF4AF0E2EF4AF073
:1095C000F6EF4AF04728D8A4E8EF4AF0EAEF4AF06D
:1095D000F2EF4AF0000E306E000E316E000E326E69
:1095E000000E336E328E336AFEEF4AF0000E306E9C
:1095F000000E316E000E326E000E336E3750800B4F
:10960000401A37503724486E36AE09EF4BF00BEF57
:109610004BF00CEF4BF048804850D8B412EF4BF0B1
:1096200014EF4BF028EF4BF04828D8A41AEF4BF07A
:109630001CEF4BF024EF4BF0000E346E000E356E35
:10964000000E366E000E376E368E376A30EF4BF0F6
:10965000000E346E000E356E000E366E000E376E44
:109660003450351036103710D8A439EF4BF03BEF9B
:109670004BF053EF4BF0000E306E000E316E000ECB
:10968000326E000E336E800E32127F0E3312405057
:10969000331230C530F531C531F532C532F533C539
:1096A00033F592EF4CF04750D8A459EF4BF05BEFF5
:1096B0004BF065EF4BF0000E306E000E316E000E79
:1096C000326E000E336E92EF4CF0485047C538F5BD
:1096D000396A385E000E395A7F0E3824416E000E0A
:1096E0003920426E30C53CF531C53DF532C53EF5F9
:1096F00033C53FF5000E306E000E316E000E326E37
:10970000000E336E000E436E000E446E000E456E6A
:10971000000E466E486AC5EF4BF04850D8B493EF40
:109720004BF095EF4BF0ACEF4BF0D8903C363D361C
:109730003E363F36D890303631363236333646AE46
:10974000A4EF4BF0A6EF4BF0A7EF4BF03080D89092
:10975000433644364536463634503C5C35503D58E9
:1097600036503E5837503F58D8A0B9EF4BF0BBEFBA
:109770004BF0C4EF4BF0468C34503C5E35503D5AB4
:1097800036503E5A37503F5A482A190E4864CBEF9C
:109790004BF0CDEF4BF08DEF4BF03C503D103E10B9
:1097A0003F10D8B4D6EF4BF0D8EF4BF0F0EF4BF0C2
:1097B0004380F0EF4BF0D8903036313632363336C6
:1097C00046AEE5EF4BF0E7EF4BF0E8EF4BF03080C3
:1097D000D89043364436453646364106D8A0420630
:1097E00032AEF5EF4BF0F7EF4BF0DBEF4BF0486AA2
:1097F00046AEFDEF4BF0FFEF4BF023EF4CF0FF0ECA
:109800004314386EFF0E4414396EFF0E45143A6E41
:109810007F0E46143B6E385039103A103B10D8B4C6
:1098200014EF4CF016EF4CF01AEF4CF0010E486EAE
:1098300023EF4CF030A01FEF4CF021EF4CF023EF62
:109840004CF016EF4CF04850D8B429EF4CF02BEF09
:109850004CF04FEF4CF0010E3026000E3122322238
:10986000332233A036EF4CF038EF4CF04FEF4CF092
:1098700030C538F531C539F532C53AF533C53BF554
:109880003B343B323A323932383238C530F539C59B
:1098900031F53AC532F53BC533F5414A422A42BE5D
:1098A0005AEF4CF0425008E14128D8A05AEF4CF052
:1098B0005CEF4CF067EF4CF0000E426E4168000E1A
:1098C000306E000E316E000E326E000E336E42BEF0
:1098D00074EF4CF0425006E14104D8B072EF4CF006
:1098E00074EF4CF080EF4CF0426A000E416E000EB7
:1098F000306E000E316E000E326E000E336E406A16
:1099000041C547F547A087EF4CF089EF4CF08CEF4D
:109910004CF0328E8DEF4CF0329ED8904730336E43
:1099200047EF4BF01200CAC628F5F7C52EF52B6A93
:109930000601C851D8B49FEF4CF0A1EF4CF02FEFC7
:109940004EF0EAEF4DF02E50D8A4A9EF4CF0ABEF5B
:109950004CF0B0EF4CF01B0E90EC70F009EF4EF0B5
:109960002E04D8A4B6EF4CF0B8EF4CF009EF4EF04F
:1099700098A1BDEF4CF0BFEF4CF0C4EF4CF0000EDF
:1099800090EC70F009EF4EF0010E90EC70F009EFE2
:109990004EF02E50D8A4CFEF4CF0D1EF4CF0D6EFD4
:1099A0004CF01B0E90EC70F009EF4EF02E04D8A492
:1099B000DCEF4CF0DEEF4CF009EF4EF098A3E3EF54
:1099C0004CF0E5EF4CF0EAEF4CF0000E90EC70F04C
:1099D00009EF4EF0010E90EC70F009EF4EF02E50B2
:1099E000D8A4F5EF4CF0F7EF4CF0FCEF4CF01B0E69
:1099F00090EC70F009EF4EF02E04D8A402EF4DF079
:109A000004EF4DF009EF4EF098A509EF4DF00BEF84
:109A10004DF010EF4DF0000E90EC70F009EF4EF0AD
:109A2000010E90EC70F009EF4EF02E50D8A41BEF11
:109A30004DF01DEF4DF022EF4DF01B0E90EC70F04D
:109A400009EF4EF02E04D8A428EF4DF02AEF4DF088
:109A500009EF4EF098A72FEF4DF031EF4DF036EFB4
:109A60004DF0000E90EC70F009EF4EF0010E90EC0E
:109A700070F009EF4EF02E50D8A441EF4DF043EFB7
:109A80004DF048EF4DF01A0E90EC70F009EF4EF0EB
:109A90002E04D8A44EEF4DF050EF4DF009EF4EF0EC
:109AA000F00EA119D8B457EF4DF059EF4DF05EEF1D
:109AB0004DF0000E90EC70F009EF4EF0010E90ECBE
:109AC00070F009EF4EF02E50D8A469EF4DF06BEF17
:109AD0004DF070EF4DF0100E90EC70F009EF4EF07D
:109AE0002E04D8A476EF4DF078EF4DF009EF4EF04C
:109AF000040E2D6E2D0E206E050E216E236A010EB2
:109B0000226E700E25EC6BF0150E256EC60EE82E3B
:109B1000FED7252EFCD700D0000E206E500EE5ECAF
:109B200068F02C6E2C50D8B498EF4DF09AEF4DF0B1
:109B30009FEF4DF0000E90EC70F009EF4EF0010E2B
:109B400090EC70F009EF4EF02E50D8A4AAEF4DF033
:109B5000ACEF4DF0B1EF4DF0100E90EC70F009EF5E
:109B60004EF02E04D8A4B7EF4DF0B9EF4DF009EF49
:109B70004EF0050E2D6E2D0E206E050E216E236A01
:109B8000010E226E700E25EC6BF0150E256EC60EC2
:109B9000E82EFED7252EFCD700D0000E206E500EEA
:109BA000E5EC68F02C6E2C50D8B4D9EF4DF0DBEF1B
:109BB0004DF0E0EF4DF0000E90EC70F009EF4EF03C
:109BC000010E90EC70F009EF4EF0FF0E90EC70F08B
:109BD00009EF4EF02850100AD8B4A3EF4CF0010A58
:109BE000D8B4C9EF4CF0030AD8B4EFEF4CF0010A37
:109BF000D8B415EF4DF0070AD8B43BEF4DF0010A89
:109C0000D8B463EF4DF0030AD8B4A4EF4DF0E5EFFC
:109C10004DF0010E0501F66510EF4EF012EF4EF01B
:109C20002FEF4EF02A6A010E296E1CEF4EF0000E47
:109C300090EC70F0294A2A2A0501F651256E266A11
:109C40002550295C2A50800A276E2650800A275802
:109C5000D8A02DEF4EF02FEF4EF017EF4EF0120080
:109C60000601886B000E876F8B6B010EFB6F836B99
:109C7000010E826F020ECC25846F856B000E85234A
:109C80008D6B000E8C6F000E8C25D96E060E8D210B
:109C9000DA6EDF6A8C4B8D2B8D5109E1820E8C5D63
:109CA000D8A055EF4EF057EF4EF043EF4EF0040EB4
:109CB000CC19D8B45EEF4EF060EF4EF062EF4EF08C
:109CC000BBEF4FF0400E8225096E090E83210A6E0C
:109CD00084C60BF585C60CF5C9EC66F00601866FE7
:109CE0008651C919D8B477EF4EF079EF4EF094EF62
:109CF0004FF0BBEF4FF093EC4CF0BBEF4FF0F4ECB8
:109D00003BF0BBEF4FF0F7C509F5F6C50AF5000EBD
:109D10000B6E060E0C6ECA511DEC45F006018D6BE4
:109D2000000E8C6FABEF4EF008EC71F00009D8B468
:109D30009CEF4EF09EEF4EF094EF4EF0000E0601B9
:109D40008C25D96E060E8D21DA6EDF50AAEC6BF0F1
:109D500006018C4B8D2B0501F6512F6E306A2F506A
:109D600006018C5D8D51800A316E3050800A315869
:109D7000D8A0BDEF4EF0BFEF4EF094EF4EF0BBEF2A
:109D80004FF0150ECB19D8A4C8EF4EF0CAEF4EF025
:109D9000CEEF4EF0040E8B6FD9EF4EF0160ECB19AE
:109DA000D8A4D5EF4EF0D7EF4EF0D9EF4EF0050E18
:109DB0008B6F8B0E206E060E216E236A010E226EB3
:109DC000700E25EC6BF0A00E00D0E82EFDD7F7C585
:109DD00020F5000E216E060E226EF6C523F5246ACC
:109DE0000601D890CA3147EC67F006018D6B000E72
:109DF0008C6F12EF4FF008EC71F00009D8B403EF4C
:109E00004FF005EF4FF0FBEF4EF0000E06018C25F2
:109E1000D96E060E8D21DA6EDF50AAEC6BF00601CA
:109E20008C4B8D2B0501F6512F6E306A2F50060199
:109E30008C5D8D51800A316E3050800A3158D8A027
:109E400024EF4FF026EF4FF0FBEF4EF0BBEF4FF05B
:109E5000CA512F6E0501F7510601896F2FC58AF689
:109E6000100ECB19D8A437EF4FF039EF4FF046EF73
:109E70004FF089C609F58AC60AF5010EBCEC59F007
:109E800009C587F60AC588F686EF4FF0110ECB1983
:109E9000D8A44DEF4FF04FEF4FF05CEF4FF089C675
:109EA00009F58AC60AF5020EBCEC59F009C587F619
:109EB0000AC588F686EF4FF0120ECB19D8A463EFCF
:109EC0004FF065EF4FF072EF4FF089C609F58AC683
:109ED0000AF5030EBCEC59F009C587F60AC588F6E9
:109EE00086EF4FF0130ECB19D8A479EF4FF07BEF2C
:109EF0004FF086EF4FF089C609F58AC60AF5040EC1
:109F0000BCEC59F009C587F60AC588F606018851E8
:109F10008B6F8B5190EC70F087C68BF606018B51DE
:109F200090EC70F0BBEF4FF0CB51000AD8B47BEF50
:109F30004EF0010AD8B47FEF4EF0110AD8B428EFE2
:109F40004FF0010AD8B428EF4FF0030AD8B428EF35
:109F50004FF0010AD8B428EF4FF0070AD8B483EFC6
:109F60004EF0010AD8B4C1EF4EF0030AD8B4C1EFE5
:109F70004EF0BBEF4FF01200136E156A000E146E18
:109F80001A6A000E196E0601BB6B000EBA6FD7EF8E
:109F90004FF0BA510B24D96EBB510C20DA6EDF5052
:109FA0000D6E0D501426000E1522BA4BBB2B0A5015
:109FB0000D6E0E6A0D50BA5DBB51800A0F6E0E50C9
:109FC000800A0F58D8A0E7EF4FF0E9EF4FF0C9EF44
:109FD0004FF014C517F51550166E135000080D6E8E
:109FE00009500D5C0E6E0A500E5C0F6E17500F5C20
:109FF000106E1650105C116E1104126E122A1DEFB5
:10A0000050F0E40E00D000D0E82EFCD700D000D0F5
:10A01000194A1A2A1ABE16EF50F0D00E195C070E14
:10A020001A58D8A016EF50F018EF50F01DEF50F06E
:10A03000BE94C094BE8E3DEF51F0CEA622EF50F0FC
:10A0400024EF50F001EF50F0BE92BE9EE40E00D01F
:10A0500000D0E82EFCD700D000D0010E526E070EC3
:10A06000526435EF50F037EF50F055EF50F0AEEF4F
:10A0700050F00601CF6B74EF50F013C5CFF674EFBC
:10A0800050F009C5CFF674EF50F00AC5CFF674EF63
:10A0900050F017C5CFF674EF50F016C5CFF674EF39
:10A0A00050F012C5CFF674EF50F05250010AD8B4F8
:10A0B00039EF50F0030AD8B43DEF50F0010AD8B49C
:10A0C00041EF50F0070AD8B445EF50F0010AD8B478
:10A0D00049EF50F0030AD8B44DEF50F0010AD8B45C
:10A0E00051EF50F074EF50F0BE94516A070E516476
:10A0F0007CEF50F07EEF50F080EF50F0ABEF50F07F
:10A100000601CFBF86EF50F08AEF50F00D6A0D2A9E
:10A110008BEF50F00D6A0D460D46C0500D18FB0B2D
:10A120000D18C06E0601CF51CF25CF6FB60E00D0EF
:10A1300000D0E82EFCD700D000D000D0BE84B60EF0
:10A1400000D000D0E82EFCD700D000D000D0BE94C4
:10A15000512A76EF50F0522A2FEF50F0BE8EE40EC7
:10A1600000D000D0E82EFCD700D000D0D4EF50F0C3
:10A17000E40E00D000D0E82EFCD700D000D0194A61
:10A180001A2A1ABECDEF50F0D00E195C070E1A58DD
:10A19000D8A0CDEF50F0CFEF50F0D4EF50F0BE94F8
:10A1A000C094BE8E3DEF51F0CEA6D9EF50F0DBEF5C
:10A1B00050F0B8EF50F0BE9EE40E00D000D0E82E74
:10A1C000FCD700D000D00601BB6B000EBA6F28EFA1
:10A1D00051F0BA510B24D96EBB510C20DA6EDF500E
:10A1E000186E516A070E5164F8EF50F0FAEF50F014
:10A1F000FCEF50F025EF51F018BE01EF51F005EFE4
:10A2000051F00D6A0D2A06EF51F00D6A0D460D460C
:10A21000C0500D18FB0B0D18C06E18501824186E86
:10A22000B60E00D000D0E82EFCD700D000D000D071
:10A23000BE84B60E00D000D0E82EFCD700D000D0EF
:10A2400000D0BE94512AF2EF50F00601BA4BBB2B5E
:10A250000A500D6E0E6A0D50BA5DBB51800A0F6E2A
:10A260000E50800A0F58D8A038EF51F03AEF51F055
:10A27000E9EF50F0BE94C094BE8E1200396A010E10
:10A28000386E600E0A6E000E096E000E0B6E0D6ABF
:10A290007F0E0C6EAD0E0F6E000E0E6E05EC5CF0B8
:10A2A000D00E126ECA0EE82EFED7122EFCD7600E0C
:10A2B0000A6E000E096E000E0B6E0D6A570E0C6EC4
:10A2C000800E0F6E060E0E6E05EC5CF0680E126EC0
:10A2D000E40EE82EFED7122EFCD700D0600E0A6ED8
:10A2E000000E096E000E0B6E0D6A000E0C6E400E15
:10A2F0000F6E000E0E6E05EC5CF0020E136EA00EDB
:10A30000126E920EE82EFED7122EFCD7132EFAD71D
:10A3100000D0010E3A6E200E0A6E000E096E000E7D
:10A320000B6E0D6A000E0C6E3AC50EF50F6A05EC49
:10A330005CF0680E126EE40EE82EFED7122EFCD7EB
:10A3400000D03A2A040E3A64A8EF51F0AAEF51F077
:10A350008BEF51F00A6A000E096E030EBCEC59F047
:10A3600009C536F50AC537F51F0E3614126E000EF4
:10A370003714136E030E12181310D8A4C2EF51F045
:10A38000C4EF51F0C9EF51F0010E0601D86FCBEFC9
:10A3900051F0010E546E010E3A6E0A6A000E096EFB
:10A3A0003A50BCEC59F009C536F50AC537F53A50B4
:10A3B000126E136A1F0E3614146E000E3714156ECB
:10A3C0001250141807E113501518D8A4EAEF51F0F1
:10A3D000ECEF51F0F1EF51F0385006019813F5EF22
:10A3E00051F03850FF0A06019817D8903834386E6B
:10A3F0003934396E5450D8B400EF52F002EF52F0B5
:10A400000DEF52F0020E3A18D8A409EF52F00BEFFC
:10A4100052F00DEF52F016EF52F03A2A040E3A6461
:10A4200014EF52F016EF52F0CDEF51F022EEC0F1E2
:10A4300011EE16F11F0EDBC4E3F4E806FCE2396A04
:10A44000000E386E010E3A6E200E0A6E000E096E76
:10A450003AC50BF50D6A2E0E0C6ED8903834D96EB5
:10A460003934DA6E160ED926050EDA22DEC40EF560
:10A47000DDC40FF505EC5CF0384A392A200E0A6E6F
:10A48000000E096E3AC50BF50D6A2F0E0C6ED890B2
:10A490003834D96E3934DA6E160ED926050EDA2222
:10A4A000DEC40EF5DDC40FF505EC5CF0384A392A40
:10A4B000200E0A6E000E096E3AC50BF50D6A320EBB
:10A4C0000C6ED8903834D96E3934DA6E160ED9261F
:10A4D000050EDA22DEC40EF5DDC40FF505EC5CF0E6
:10A4E000384A392A200E0A6E000E096E3AC50BF55D
:10A4F0000D6A330E0C6ED8903834D96E3934DA6E5A
:10A50000160ED926050EDA22DEC40EF5DDC40FF5CF
:10A5100005EC5CF0384A392A5450D8B492EF52F026
:10A5200094EF52F09FEF52F0020E3A18D8A49BEF2E
:10A5300052F09DEF52F09FEF52F0A8EF52F03A2AFE
:10A54000040E3A64A6EF52F0A8EF52F024EF52F056
:10A55000680E126EE40EE82EFED7122EFCD700D045
:10A560000601916B926B95691F0E966F1200D8ECE5
:10A5700070F00009D8B4BFEF52F0C1EF52F0DEEF37
:10A5800053F0D5EC6BF00501ED6F400EF425D96E5C
:10A59000090EF521DA6EEDC5DFF457EF53F0550ED5
:10A5A00009014019D8B4D7EF52F0D9EF52F089EF32
:10A5B00053F078EC6CF0DEEF53F009014151D8A470
:10A5C000E4EF52F0E6EF52F0EBEF52F0010E06012D
:10A5D000C86F89EF53F0030E4119D8A4F2EF52F07F
:10A5E000F4EF52F0D9EF52F0010E0601C76F89EF78
:10A5F00053F042C9CCF689EF53F043C9CBF689EF4B
:10A6000053F044C9CAF689EF53F045C9F7F589EF0D
:10A6100053F046C9F6F589EF53F00601C851D8B496
:10A6200014EF53F016EF53F089EF53F047C9C9F612
:10A6300089EF53F00601C851D8B421EF53F023EF4E
:10A6400053F089EF53F0AA0E09014819D8A42BEF53
:10A6500053F02DEF53F089EF53F0F0EC71F030EC44
:10A660004EF0F3EC71F0D9EF52F00601C851D8A4C6
:10A670003CEF53F03EEF53F0D9EF52F0CC510501CF
:10A68000ED6FEE6B040EED27000EEE23F451ED5D41
:10A69000EE51800AEF6FF551800AEF59D8B053EFB1
:10A6A00053F055EF53F089EF53F0D9EF52F0F4C562
:10A6B000EDF5F5C5EEF5EE51000AD8B462EF53F0B2
:10A6C00035EF53F0ED51000AD8B4CFEF52F0010A44
:10A6D000D8B4DDEF52F0030AD8B4F9EF52F0010A12
:10A6E000D8B4FDEF52F0070AD8B401EF53F0010AD5
:10A6F000D8B405EF53F0030AD8B409EF53F0010AB8
:10A70000D8B40DEF53F00F0AD8B41AEF53F035EF69
:10A7100053F00601C751D8B490EF53F092EF53F0C5
:10A72000DBEF53F0CC510501ED6FEE6B030EED271F
:10A73000000EEE23F451ED1907E1F551EE19D8A4FE
:10A74000A4EF53F0A6EF53F0AFEF53F0400EF42513
:10A75000D96E090EF521DA6EDF500601C96F0601C8
:10A76000CC510501ED6FEE6B040EED27000EEE23CC
:10A77000F451ED1907E1F551EE19D8A4C2EF53F0E9
:10A78000C4EF53F0DBEF53F0400EF425D96E090E01
:10A79000F521DA6EAA0EDE18D8A4D1EF53F0D3EF6C
:10A7A00053F0DBEF53F0F0EC71F02FEC57F0F3ECDB
:10A7B00071F0DEEF53F00501F44BF52B12007BEC4A
:10A7C0006FF0150E0501F06FC60EE82EFED7F02FC4
:10A7D000FCD70000BC0E096ED40E0A6EBAEC71F004
:10A7E000F3EC71F0F00E0601A16F906B000E206E7D
:10A7F000500EE5EC68F060EC71F00601D96FEDECFD
:10A8000071F098EC6EF074EC64F03EEC51F011ECE9
:10A8100036F011EC36F004EC55F0E8EC58F0F00EA0
:10A820000601A119D8B417EF54F019EF54F04DEF09
:10A8300054F0010E0501F36F200E0A6E000E096E32
:10A84000F3C50BF50D6A110E0C6E010E0F6E020EA4
:10A850000E6E05EC5CF05450D8B431EF54F033EF89
:10A8600054F03FEF54F0020E0501F319D8A43BEF6A
:10A8700054F03DEF54F03FEF54F049EF54F0050130
:10A88000F32B040EF36547EF54F049EF54F01CEF3F
:10A8900054F09CEC24F04FEF54F004EC55F03EECF7
:10A8A00051F00A6AEA0E096EFCEC70F00501F26FD5
:10A8B000F229D8B45EEF54F060EF54F064EF54F036
:10A8C0000601FE6B67EF54F0010E0601FE6FEDEC22
:10A8D00071F0D00E0501F06FC90EE82EFED7F02FF3
:10A8E000FCD700D00601D16B13EC39F0AEEC70F060
:10A8F0000601C04BC12BB7EC52F0D2EF54F0060169
:10A900008EA785EF54F087EF54F076EF54F011ECFA
:10A9100036F076EF54F006018EA191EF54F093EFEC
:10A9200054F076EF54F09CEC24F076EF54F00601EE
:10A930008EAB9DEF54F09FEF54F076EF54F075EC32
:10A9400063F076EF54F0060190B1A9EF54F0ABEF4D
:10A9500054F0AFEF54F0AFEC1CF076EF54F08EA350
:10A96000B4EF54F0B6EF54F076EF54F074EC64F0BA
:10A9700076EF54F006018EADC0EF54F0C2EF54F004
:10A9800076EF54F0ADEC68F076EF54F0060194A346
:10A99000CCEF54F0CEEF54F076EF54F00CEC33F0F3
:10A9A00076EF54F00F0E0601C0150501F06F000E92
:10A9B0000601C1150501F16FF151000AD8B4E3EFAA
:10A9C00054F076EF54F0F051000AD8B476EF54F01A
:10A9D000010AD8B47FEF54F0030AD8B48BEF54F0D7
:10A9E000010AD8B497EF54F0070AD8B4A3EF54F093
:10A9F000010AD8B4BAEF54F0030AD8B4C6EF54F041
:10AA000076EF54F081EF18F02C6A000E2B6E296A55
:10AA1000320E2A6E060190A510EF55F012EF55F098
:10AA200014EF55F0050E2A6EBE9CD00E256ECA0E90
:10AA3000E82EFED7252EFCD7BE8C0601D16B05EF84
:10AA400056F00D0E266E2D0E256ED80EE82EFED772
:10AA5000252EFCD7262EFAD7060190A132EF55F00D
:10AA600034EF55F041EF55F02B8C2B9E2C802C921F
:10AA7000020E206E2BC521F52CC522F5200E55ECBB
:10AA800069F0010E2D6E200E0A6E000E096E2DC5A6
:10AA90000BF50D6A110E0C6E010E0F6E010E0E6E8F
:10AAA00005EC5CF05450D8B458EF55F05AEF55F01F
:10AAB00065EF55F0020E2D18D8A461EF55F063EF45
:10AAC00055F065EF55F06EEF55F02D2A040E2D640C
:10AAD0006CEF55F06EEF55F043EF55F00D0E266E0E
:10AAE0002D0E256ED80EE82EFED7252EFCD7262E4D
:10AAF000FAD7060190A17FEF55F081EF55F08EEF68
:10AB000055F02B8E2B9C2C822C90020E206E2BC588
:10AB100021F52CC522F5200E55EC69F0010E2D6EA5
:10AB2000200E0A6E000E096E2DC50BF50D6A110E72
:10AB30000C6E010E0F6E000E0E6E05EC5CF05450A4
:10AB4000D8B4A5EF55F0A7EF55F0B2EF55F0020ECF
:10AB50002D18D8A4AEEF55F0B0EF55F0B2EF55F088
:10AB6000BBEF55F02D2A040E2D64B9EF55F0BBEF65
:10AB700055F090EF55F0292A020E2964C2EF55F0E6
:10AB8000C4EF55F005EF56F0296A110E266E3C0E03
:10AB9000256ECB0EE82EFED7252EFCD7262EFAD713
:10ABA0000000CEA6D6EF55F0D8EF55F005EF56F0E1
:10ABB000290E266E960E256E7F0EE82EFED7252EC8
:10ABC000FCD7262EFAD70000290E266E960E256E8B
:10ABD0007F0EE82EFED7252EFCD7262EFAD70000B2
:10ABE00013EC39F0D00E256ECA0EE82EFED7252EB6
:10ABF000FCD7F00E0601A119D8B401EF56F003EF0F
:10AC000056F005EF56F00FEF56F00601D1512A5CD1
:10AC1000D8B00DEF56F00FEF56F021EF55F0020EC1
:10AC2000276E000E096E010E0A6E270E0B6E050EC2
:10AC30000C6E080EBCEC4FF0D00E256ECA0EE82E3E
:10AC4000FED7252EFCD71200D6C76CF5D7C76DF5F9
:10AC5000D8C76EF5D9C76FF549C56CF54AC56DF50E
:10AC60004BC56EF54CC56FF5810E0501606FFF0E8B
:10AC7000616F6CC562F56DC563F56EC564F56FC532
:10AC800065F5180E49EF56F0D89065336433633399
:10AC90006233E82E44EF56F0625160256A6F000E71
:10ACA00061216B6F6BBF5EEF56F06B5109E1170EC0
:10ACB0006A5DD8A05EEF56F060EF56F06AEF56F08E
:10ACC00049C549F54AC54AF54BC54BF54CC54CF548
:10ACD0002EEF57F06BBF6FEF56F071EF56F0E2EFCB
:10ACE00056F06AC560F5FF0E616FFF0E626F7F0E52
:10ACF000636F000E646F606780EF56F088EF56F068
:10AD000064356433633362336133602F7BEF56F015
:10AD100061C566F562C567F563C568F564C569F523
:10AD2000050166516C15606F67516D15616F685153
:10AD30006E15626F69516F15636F60516111621119
:10AD40006311D8A4A6EF56F0A8EF56F0AAEF56F07C
:10AD500060EF56F06CC560F56DC561F56EC562F5C6
:10AD60006FC563F5200EBAEF56F0D89063336233A7
:10AD700061336033E82EB5EF56F060516111621116
:10AD80006311D8B4C6EF56F0C8EF56F0D0EF56F0C6
:10AD900066516C2767516D2368516E2369516F238B
:10ADA000661D606F671D616F681D626F691D636F4F
:10ADB00060516C1761516D1762516E1763516F17B7
:10ADC00026EF57F06CC560F56DC561F56EC562F58F
:10ADD0006FC563F5200EF2EF56F0D89063336233FF
:10ADE00061336033E82EEDEF56F06051611162116E
:10ADF0006311D8A4FEEF56F000EF57F00AEF57F0BA
:10AE0000000E6C6F000E6D6F000E6E6F000E6F6F98
:10AE100026EF57F0D8906C35606F6D35616F6E35E9
:10AE2000626F6F35636F6051611162116311D8B445
:10AE30001CEF57F01EEF57F026EF57F0000E6C6F27
:10AE4000000E6D6F800E6E6FBF0E6F6F6CC549F593
:10AE50006DC54AF56EC54BF56FC54CF51200010E78
:10AE60000601346F306B010E2F6F020ECC25316F4F
:10AE7000326B000E3223410E096E090E0A6E31C686
:10AE80000BF532C60CF5C9EC66F00601336FC951FB
:10AE90003319D8B44EEF57F050EF57F0E8EF57F0B2
:10AEA00078EC6CF0000E90EC70F00DEF58F058EC70
:10AEB0005BF007EF58F0F7C509F5F6C50AF5470E40
:10AEC0000B6E090E0C6ECA51BCEC4FF007EF58F038
:10AED000CA510501EB6FF7510601356FEBC536F628
:10AEE000090147510501EB6F090148510601376F10
:10AEF000EBC538F6100ECB19D8A481EF57F083EFCD
:10AF000057F095EF57F0200E0A6E000E096E010EF5
:10AF10000B6E35C60CF536C60DF537C60EF538C6C0
:10AF20000FF505EC5CF0E4EF57F0110ECB19D8A447
:10AF30009CEF57F09EEF57F0B0EF57F0200E0A6EDF
:10AF4000000E096E020E0B6E35C60CF536C60DF5F9
:10AF500037C60EF538C60FF505EC5CF0E4EF57F098
:10AF6000120ECB19D8A4B7EF57F0B9EF57F0CBEFCB
:10AF700057F0200E0A6E000E096E030E0B6E35C6DA
:10AF80000CF536C60DF537C60EF538C60FF505ECCF
:10AF90005CF0E4EF57F0130ECB19D8A4D2EF57F0C2
:10AFA000D4EF57F0E4EF57F0200E0A6E000E096E52
:10AFB000040E0B6E35C60CF536C60DF537C60EF50C
:10AFC00038C60FF505EC5CF00601346B07EF58F05E
:10AFD000CB51000AD8B407EF58F0010AD8B457EFA4
:10AFE00057F0110AD8B468EF57F0010AD8B468EFE7
:10AFF00057F0030AD8B468EF57F0010AD8B468EFE5
:10B0000057F0070AD8B45BEF57F0E4EF57F078EC4D
:10B010006CF00601345190EC70F01200116E11507A
:10B02000D8B415EF58F017EF58F039EF58F00CBEC0
:10B030001EEF58F01CEF58F039EF58F009C50DF528
:10B040000AC50EF50BC50FF50CC510F50D1E0E1E2D
:10B050000F1E101E0D2A000E0E220F2210220DC5EB
:10B0600013F50EC514F50FC515F510C516F541EF0E
:10B0700058F009C513F50AC514F50BC515F50CC52F
:10B0800016F509500A100B100C10D8A44AEF58F00E
:10B090004CEF58F056EF58F0000E096E000E0A6E95
:10B0A000000E0B6E000E0C6EE7EF58F0960E126E4F
:10B0B00060EF58F0122AD89016321532143213323B
:10B0C000000E13140D6E000E14140E6E000E1514E7
:10B0D0000F6EFE0E1614106E0D500E100F10101085
:10B0E000D8A475EF58F077EF58F05AEF58F085EF85
:10B0F00058F0122A010E1326000E142215221622D1
:10B10000D8901632153214321332000E13140D6E0D
:10B11000000E14140E6E000E15140F6EFF0E161492
:10B12000106E0D500E100F101010D8A49AEF58F09A
:10B130009CEF58F079EF58F0A4EF58F01206D89031
:10B14000133614361536163615BEA9EF58F0ABEF88
:10B1500058F0B3EF58F0020E1260B1EF58F0B3EFB1
:10B1600058F09EEF58F012B0B8EF58F0BAEF58F020
:10B17000BBEF58F0159ED890123212C50DF50E6A2D
:10B180000F6A106A0DC510F50F6A0E6A0D6A0D5030
:10B1900013120E5014120F50151210501612115097
:10B1A000D8B4D5EF58F0D7EF58F0DFEF58F00CBE19
:10B1B000DEEF58F0DCEF58F0DFEF58F0168E13C5D5
:10B1C00009F514C50AF515C50BF516C50CF51200E1
:10B1D0000A6AE90E096E000E0B6E9FEC6CF00F6AA6
:10B1E0000A6A0A0E096EFCEC70F00F6E2E0E0F1834
:10B1F000D8B4FDEF58F0FFEF58F07FEF59F00A6A2E
:10B20000E00E096EFDC50BF59FEC6CF00A6AE10ECD
:10B21000096E000E0B6E9FEC6CF00A6AE20E096E6E
:10B22000000E0B6E9FEC6CF00A6AE30E096E000EC6
:10B230000B6E9FEC6CF00A6AE40E096E000E0B6E4A
:10B240009FEC6CF00A6A090E096E310E0B6E9FECD2
:10B250006CF00A6A0A0E096E2E0E0B6E9FEC6CF0F3
:10B260000A6A0B0E096E300E0B6E9FEC6CF00A6AC8
:10B270000C0E096E300E0B6E9FEC6CF00A6A000E1D
:10B28000096E390E0B6E9FEC6CF00A6A010E096EA6
:10B29000380E0B6E9FEC6CF00A6A020E096E370EC8
:10B2A0000B6E9FEC6CF00A6A030E096E360E0B6E85
:10B2B0009FEC6CF00A6A040E096E350E0B6E9FEC63
:10B2C0006CF00A6A050E096E2D0E0B6E9FEC6CF089
:10B2D0000A6A060E096E340E0B6E9FEC6CF00A6A59
:10B2E000070E096E330E0B6E9FEC6CF00A6A080EA7
:10B2F000096E320E0B6E9FEC6CF0BBEF59F00A6AD0
:10B30000E20E096EFCEC70F00F6E0FC5C2F606017E
:10B31000C36B0A6AE10E096EFCEC70F00F6E0F5001
:10B320000E6E0D6A0D500601C2130E50C3130A6A49
:10B33000E30E096EFCEC70F00601D36F0A6AE40EAE
:10B34000096EFCEC70F00601D26F0A6AE00E096E1D
:10B35000FCEC70F00501FD6FC80EFD65B2EF59F011
:10B36000B4EF59F0BBEF59F00A6AE00E096E010E16
:10B370000B6E9FEC6CF012000D6E0D500B6E0C6A94
:10B38000070ED8900B360C36E82EC1EF59F0000EA0
:10B390000B100601BE6FA00E0C10BF6F09C5BCF6E6
:10B3A0000AC5BDF6BE8EBE82B60E00D000D0E82E15
:10B3B000FCD700D000D000D0010E526E030E5264B4
:10B3C000E4EF59F0E6EF59F0F8EF59F079EF5AF061
:10B3D000BEC64FF5BFC650F507EF5AF0BCC64FF5D5
:10B3E000BDC650F507EF5AF04F68506807EF5AF0A6
:10B3F0005250010AD8B4E8EF59F0030AD8B4EEEF7E
:10B4000059F0010AD8B4F4EF59F007EF5AF0BE949E
:10B41000B60E00D000D0E82EFCD700D000D000D06F
:10B42000516A0F0E516417EF5AF019EF5AF01BEFE3
:10B430005AF075EF5AF0030E5218D8B422EF5AF0B2
:10B4400024EF5AF046EF5AF050BE29EF5AF02DEF94
:10B450005AF00B6A0B2A2EEF5AF00B6A0B460B467A
:10B46000C0500B18FB0B0B18C06ED8904F344F6EAA
:10B470005034506ED50EE82EFED70000BE84D50E97
:10B48000E82EFED70000BE9472EF5AF0BE94D50E9F
:10B49000E82EFED70000BE84D50EE82EFED70000B1
:10B4A000CEA055EF5AF057EF5AF066EF5AF04FC55D
:10B4B0000BF550C50CF5D8900B360C36FE0E0B1460
:10B4C0004F6EFF0E0C14506E72EF5AF0010E4FC506
:10B4D0000BF550C50CF5D8900B360C360B104F6E93
:10B4E0000C50506E512A11EF5AF0C094522ADEEFE0
:10B4F00059F0D50EE82EFED70000BE94BE92150E70
:10B500000B6EC60EE82EFED70B2EFCD700D04FC513
:10B5100009F550C50AF51200266A040E276E270E9B
:10B52000206E050E216E236A010E226E700E25EC30
:10B530006BF091C627F5150E256EC60EE82EFED7C8
:10B54000252EFCD700D0000E206E500EE5EC68F0E2
:10B55000286E2850D8B4AFEF5AF0B1EF5AF0E4EFAC
:10B560005AF0810E2818D8B4B8EF5AF0BAEF5AF052
:10B57000C3EF5AF0B30E2818D8A4C1EF5AF0C3EFA6
:10B580005AF0C8EF5AF0010E0601916FE7EF5AF03A
:10B59000820E2818D8B4CFEF5AF0D1EF5AF0DAEF74
:10B5A0005AF0B20E2818D8A4D8EF5AF0DAEF5AF0B1
:10B5B000DFEF5AF0020E0601916FE7EF5AF0040E2A
:10B5C0000601916FE7EF5AF0080E0601916F2750C0
:10B5D0009119D8B4EEEF5AF0F0EF5AF0F2EF5AF0BA
:10B5E000050E9413050E276E270E206E050E216E94
:10B5F000236A010E226E700E25EC6BF092C627F5C1
:10B60000150E256EC60EE82EFED7252EFCD700D0CF
:10B61000000E206E500EE5EC68F0286E2850D8B46D
:10B6200014EF5BF016EF5BF049EF5BF0810E28182A
:10B63000D8B41DEF5BF01FEF5BF028EF5BF0B30EAB
:10B640002818D8A426EF5BF028EF5BF02DEF5BF015
:10B65000010E0601926F4CEF5BF0820E2818D8B4F1
:10B6600034EF5BF036EF5BF03FEF5BF0B20E281883
:10B67000D8A43DEF5BF03FEF5BF044EF5BF0020ED0
:10B680000601926F4CEF5BF0040E0601926F4CEFD7
:10B690005BF0080E0601926F27509219D8B453EF51
:10B6A0005BF055EF5BF057EF5BF0050E9413120063
:10B6B00047C9E9F5C80E0501F719D8A462EF5BF098
:10B6C00064EF5BF0C2EF5BF0AFEF5BF00A6AE00E95
:10B6D000096E000E0B6E9FEC6CF004EF5CF00A6AD2
:10B6E000E10E096E000E0B6E9FEC6CF00A6AE20E22
:10B6F000096E000E0B6E9FEC6CF00A6AE30E096E89
:10B70000000E0B6E9FEC6CF00A6AE40E096E000EE0
:10B710000B6E9FEC6CF0010E0501FD6F0601C36B13
:10B72000000EC26FD36BD26B04EF5CF00A6AE90EB5
:10B73000096E010E0B6E9FEC6CF0050E0501E86FB3
:10B740000F0EE76FF10EE82EFED7E72FFCD7E82F9C
:10B75000FAD7FF0004EF5CF0FF0004EF5CF0E95162
:10B76000800AD8B466EF5BF0010AD8B46FEF5BF0E3
:10B770007F0AD8B496EF5BF0010AD8B4ACEF5BF067
:10B7800004EF5CF0C90EF719D8A4C9EF5BF0CBEF5A
:10B790005BF0E0EF5BF0D5EF5BF008EC2FF004EF2F
:10B7A0005CF00CEC33F004EF5CF0E951010AD8B422
:10B7B000CDEF5BF0030AD8B4D1EF5BF004EF5CF09F
:10B7C000D20EF719D8A4E7EF5BF0E9EF5BF004EFD6
:10B7D0005CF0EA6BEAC509F50A6A470EEA25D96EFC
:10B7E000DA6A090EDA22DF500B6E9FEC6CF005016D
:10B7F000EA2B080EEA65FFEF5BF001EF5CF0EAEF81
:10B800005BF0010E0601FD6F12000B50106E116A05
:10B81000070ED89010361136E82E09EF5CF009506B
:10B8200010100601BE6F0A501110BF6F0CC5BCF698
:10B830000DC5BDF6BE8EBE82B60E00D000D0E82E7D
:10B84000FCD700D000D000D0010E526E030E52641F
:10B850002CEF5CF02EEF5CF042EF5CF08BEF5CF0D5
:10B86000BEC64FF5BFC650F551EF5CF0BCC64FF5F4
:10B87000BDC650F551EF5CF00EC54FF50FC550F544
:10B8800051EF5CF05250010AD8B430EF5CF0030A7B
:10B89000D8B436EF5CF0010AD8B43CEF5CF051EF5D
:10B8A0005CF0BE94516A0F0E516459EF5CF05BEF8F
:10B8B0005CF05DEF5CF088EF5CF050BE62EF5CF036
:10B8C00066EF5CF0106A102A67EF5CF0106A1046B1
:10B8D0001046C0501018FB0B1018C06ED8904F3493
:10B8E0004F6E5034506EB60E00D000D0E82EFCD70C
:10B8F00000D000D000D0BE84B60E00D000D0E82E1C
:10B90000FCD700D000D000D0BE94512A53EF5CF099
:10B91000522A26EF5CF0C094BE92150E106EC60E31
:10B92000E82EFED7102EFCD700D01200010E146EA8
:10B93000200E0A6E000E096E14C50BF50D6A110E6D
:10B940000C6E010E0F6E020E0E6E05EC5CF0200EFA
:10B950000A6E000E096E14C50BF50D6A520E0C6EC0
:10B96000010E0F6E060E0E6E05EC5CF0200E0A6ED8
:10B97000000E096E14C50BF50D6A030E0C6E0F6AEE
:10B98000010E0E6E05EC5CF0200E0A6E000E096EC4
:10B9900014C50BF50D6A030E0C6E0F6A010E0E6EC8
:10B9A00005EC5CF0200E0A6E000E096E14C50BF556
:10B9B0000D6A4A0E0C6E0F6A000E0E6E05EC5CF0FE
:10B9C000200E0A6E000E096E14C50BF50D6A490EA5
:10B9D0000C6E0F6A050E0E6E05EC5CF0200E0A6E02
:10B9E000000E096E14C50BF50D6A4B0E0C6E050E9C
:10B9F0000F6E050E0E6E05EC5CF05450D8B403EFDC
:10BA00005DF005EF5DF010EF5DF0020E1418D8A4A4
:10BA10000CEF5DF00EEF5DF010EF5DF019EF5DF0F3
:10BA2000142A040E146417EF5DF019EF5DF098EF1F
:10BA30005CF0050E136E0F0E126EF10EE82EFED79F
:10BA4000122EFCD7132EFAD700001200166E16C560
:10BA500015F50A6A140E096E1550BCEC59F009C5AB
:10BA600013F50AC514F5050E1218D8A43AEF5DF0C7
:10BA70003CEF5DF071EF5DF0138213901604D8A4D3
:10BA800044EF5DF046EF5DF04AEF5DF006019B810B
:10BA9000A6EF5DF0020E1618D8A451EF5DF053EF3B
:10BAA0005DF057EF5DF006019C81A6EF5DF0030E9F
:10BAB0001618D8A45EEF5DF060EF5DF064EF5DF006
:10BAC00006019D81A6EF5DF0040E1618D8A46BEF59
:10BAD0005DF06DEF5DF0A6EF5DF006019E81A6EFD3
:10BAE0005DF0030E1312040E14121604D8A47BEF9B
:10BAF0005DF07DEF5DF081EF5DF006019B91A6EFBB
:10BB00005DF0020E1618D8A488EF5DF08AEF5DF0A4
:10BB10008EEF5DF006019C91A6EF5DF0030E161806
:10BB2000D8A495EF5DF097EF5DF09BEF5DF0060117
:10BB30009D91A6EF5DF0040E1618D8A4A2EF5DF05B
:10BB4000A4EF5DF0A6EF5DF006019E91200E0A6E57
:10BB5000000E096E15C50BF50D6A140E0C6E13C59B
:10BB60000EF514C50FF505EC5CF0120029EC71F030
:10BB70000009D8B4BEEF5DF0C0EF5DF0FAEF5DF004
:10BB8000CDEF5DF094EC71F043EF5EF01CEC72F0E1
:10BB900043EF5EF0000E43EF5EF0B8C712F5B9C791
:10BBA00013F502D8DEEF5DF00500FA6E0701AC5127
:10BBB000FD6EAD51FE6EFF6AFA501200166E176AE6
:10BBC0001750000AD8B4E7EF5DF0CAEF5DF01650E9
:10BBD000010AD8B4CAEF5DF0030AD8B4C2EF5DF031
:10BBE000010AD8B4C6EF5DF0070AD8B4CAEF5DF019
:10BBF000CAEF5DF01EEC71F00009D8B402EF5EF000
:10BC000004EF5EF042EF5EF00701C951030B00093B
:10BC1000D8B40DEF5EF00FEF5EF01BEF5EF0010E9B
:10BC2000166EC951030B176E1650175EC9511718BF
:10BC3000FC0B1718C96FC3C7D9F4C4C7DAF4DF50B7
:10BC4000186EC34BC42BC507D8A0C607C551C61173
:10BC5000D8A42DEF5EF02FEF5EF037EF5EF085ECAD
:10BC600067F0166E16501A6E1B6A3AEF5EF01B6A8A
:10BC7000030E1A6E1AC519F51850E2EC71F019503E
:10BC800043EF5EF0030E12000B340C34126E1250B0
:10BC9000D8A44DEF5EF04FEF5EF059EF5EF0000E6E
:10BCA000096E000E0A6E000E0B6E000E0C6EC6EFD3
:10BCB0005EF009C50DF50AC50EF50BC50FF50CC5EF
:10BCC00010F5200E69EF5EF0D89010320F320E3270
:10BCD0000D32E82E64EF5EF00D50116E0B8EFF0EEC
:10BCE0000916FF0E0A16FF0E0B16000E0C16960E06
:10BCF000125E12BE80EF5EF07EEF5EF096EF5EF0B9
:10BD00001250800A970FD8B088EF5EF08AEF5EF08D
:10BD10008CEF5EF04FEF5EF0D8900C320B320A32AF
:10BD20000932123E8CEF5EF0AEEF5EF01F0E126431
:10BD30009CEF5EF09EEF5EF0A6EF5EF04FEF5EF0E0
:10BD4000D89009360A360B360C3612061250D8A493
:10BD5000ACEF5EF0AEEF5EF0A0EF5EF01150D8B445
:10BD6000B4EF5EF0B6EF5EF0BEEF5EF00C1E0B1EA1
:10BD70000A1E096C000E0A220B220C2209C509F5C5
:10BD80000AC50AF50BC50BF50CC50CF51200000E23
:10BD90003014386E000E3114396E800E32143A6E43
:10BDA0007F0E33143B6E385039103A103B10D8A434
:10BDB000DCEF5EF0DEEF5EF0E6EF5EF0000E306E80
:10BDC000000E316E000E326E000E336E000E341413
:10BDD000386E000E3514396E800E36143A6E7F0EB2
:10BDE00037143B6E385039103A103B10D8A4FBEF93
:10BDF0005EF0FDEF5EF005EF5FF0000E346E000EBA
:10BE0000356E000E366E000E376E33AE0AEF5FF001
:10BE10000CEF5FF015EF5FF0306C311ED8B0312AB7
:10BE2000321ED8B0322A800E335637AE1AEF5FF08A
:10BE30001CEF5FF025EF5FF0346C351ED8B0352A6B
:10BE4000361ED8B0362A800E3756000E301A000E35
:10BE5000311A000E321A800E331A000E341A000EF8
:10BE6000351A000E361A800E371A3450305C3550B1
:10BE700031583650325837503358D8B042EF5FF00F
:10BE800044EF5FF047EF5FF0D89048EF5FF0D88065
:10BE90001200800E0501C05DD8A051EF5FF053EF96
:10BEA0005FF059EF5FF00701E36B4B0EE26FC8EFF5
:10BEB0005FF0C30ECC6F050ECD6FBDC5D0F5BEC50E
:10BEC000D1F5C05109E1020EBF5DD8A06AEF5FF065
:10BED0006CEF5FF077EF5FF0FF0EBF25D96FFF0EBD
:10BEE000C021DA6FD36B000ED26F7DEF5FF0DA6B9B
:10BEF000010ED96FD36B010ED26FD00EB56F050E48
:10BF0000B66FC1C5B7F5C2C5B8F5CC0EB96F050E91
:10BF1000BA6FC1EC69F0B5C5CEF5B6C5CFF5050170
:10BF2000BF51C011D8B497EF5FF099EF5FF0C8EF41
:10BF30005FF0CFBF9EEF5FF0A0EF5FF0C8EF5FF064
:10BF4000FF0EBF25C76FFF0EC021C86FC751CE5D62
:10BF5000CF51800AC96FC851800AC959D8A0B3EF20
:10BF60005FF0B5EF5FF0BDEF5FF0FF0EBF25CA6F6A
:10BF7000FF0EC021CB6FC1EF5FF0CEC5CAF5CFC5B4
:10BF8000CBF5CA51BD25D96ECB51BE21DA6EDF6A21
:10BF90001200000EF66EE10EF76E000EF86E02EE65
:10BFA000C0F110EE20F00900F5C4EEF4E550E150C8
:10BFB000FAE1D00EF66ECA0EF76E000EF86E02EEC3
:10BFC00000F010EE9CF00900F5C4EEF4E550E150ED
:10BFD000FAE1420EF66EC80EF76E000EF86E01EE34
:10BFE00000F310EEA6F00900F5C4EEF4E550E150C0
:10BFF000FAE1720EF66EE00EF76E000EF86E01EECC
:10C00000DBF210EE24F00900F5C4EEF4E550E15047
:10C01000FAE14E0EF66EE40EF76E000EF86E0900B1
:10C02000F5C4FDF502EE00F2800EEE6AE806FDE1D1
:10C0300002EE00F1C00EEE6AE806FDE102EE9CF0B1
:10C04000500EEE6AE806FDE101EEA6F3460EEE6A3A
:10C05000E806FDE101EE8EF24D0EEE6AE806FDE126
:10C0600001EEF4F1090EEE6AE806FDE101EE4FF192
:10C07000090EEE6AE806FDE10401080E5D6F300E60
:10C080005E6F000E5F6F0001DFEF53F0DAC713F54C
:10C09000DBC714F5DCC715F5DDC716F509C513F5C3
:10C0A0000AC514F50BC515F50CC516F513C50DF528
:10C0B00014C50EF515C50FF516C510F5180E66EF6B
:10C0C00060F0D89010320F320E320D32E82E61EF50
:10C0D00060F00D50116E126A11501210D8A473EF57
:10C0E00060F075EF60F093EF60F0D89013340D6E50
:10C0F00014340E6E15340F6E1634106E0D500E1073
:10C100000F101010D8A487EF60F089EF60F08EEF69
:10C1100060F00A6A020E096EC1EF60F00A6A030E4F
:10C12000096EC1EF60F011281210D8A49AEF60F0E8
:10C130009CEF60F0BEEF60F013C50DF514C50EF571
:10C1400015C50FF516C510F5090ED8900D360E362B
:10C150000F361036E82EA5EF60F00D500E100F10C0
:10C160001010D8B4B6EF60F0B9EF60F0010EBAEF7E
:10C1700060F0000E096E0A6AC1EF60F00A6A040EF0
:10C18000096E1200166E126A1650D8B4CAEF60F02B
:10C19000CCEF60F02CEF61F016AED1EF60F0D3EF92
:10C1A00060F0DDEF60F010C5D9F411C5DAF42D0EA2
:10C1B000DF6E104A112AE5EF60F010C5D9F411C501
:10C1C000DAF42B0EDF6ED9EF60F0136A270E156ECE
:10C1D000100E146E16C509F50A6A14C50BF515C5BF
:10C1E0000CF574EC68F00950176E1750D8A4FBEFEB
:10C1F00060F0FDEF60F005EF61F01250D8B403EF8E
:10C2000061F005EF61F014EF61F01750300F10C5C9
:10C21000D9F411C5DAF4DF6E104A112A175014024E
:10C22000F350165E010E126E14C509F515C50AF518
:10C230000C6A0A0E0B6E74EC68F009C514F50AC599
:10C2400015F5132A040E136428EF61F02AEF61F04C
:10C25000EAEF60F034EF61F010C5D9F411C5DAF4FB
:10C26000300EDF6E104A112A10C5D9F411C5DAF468
:10C27000DF6A1200270E196E100E186E166A105023
:10C280001110D8B446EF61F048EF61F094EF61F01F
:10C29000176A10C509F50A6A18C50BF519C50CF51A
:10C2A00074EC68F009501A6E1A50D8A45AEF61F075
:10C2B0005CEF61F064EF61F01650D8B462EF61F0AA
:10C2C00064EF61F07CEF61F01A50300F12C5D9F4C1
:10C2D00013C5DAF4DF6E124A132A1A501802F3C497
:10C2E00014F5F4C415F51902F35015261450105E18
:10C2F0001550115A010E166E18C509F519C50AF523
:10C300000C6A0A0E0B6E74EC68F009C518F50AC5C4
:10C3100019F5172A040E176490EF61F092EF61F09F
:10C3200049EF61F09CEF61F012C5D9F413C5DAF45E
:10C33000300EDF6E124A132A12C5D9F413C5DAF48F
:10C34000DF6A12000B500C10D8B4A9EF61F0ABEF0C
:10C3500061F0B4EF61F00B500C10D8A4B2EF61F0B3
:10C36000B4EF61F0B9EF61F0095022EC72F006EF22
:10C3700062F020EE09F00B50D9260C50DA22DE5084
:10C38000DE10D8B4C6EF61F0C8EF61F0E3EF61F002
:10C3900020EE09F00B50D9260C50DA2210EE02F0F4
:10C3A0000B50E1260C50E222DE50E65CE650800A9B
:10C3B000116EDE50800A1158D8B0E1EF61F0E3EF62
:10C3C00061F006EF62F020EE02F00B50D9260C501F
:10C3D000DA22DEC40DF5DDC40EF50BC5D9F40CC5AB
:10C3E000DAF4DEC40FF5DDC410F50D500F24D96E5C
:10C3F0000E501020DA6E09C5DFF420EE02F00B506B
:10C40000D9260C50DA22DE2A000EDD2212000E6A36
:10C410000CBE0FEF62F00DEF62F015EF62F00B6CE7
:10C420000C1ED8B00C2A010E0E6E0ABE1CEF62F074
:10C430001AEF62F022EF62F0096C0A1ED8B00A2AE5
:10C44000010E0E1A106A000E0F6E0B500C10D8B4AD
:10C450002CEF62F02EEF62F056EF62F0010E0D6EDF
:10C4600036EF62F0D8900B360C360D2A0CAE3BEF4F
:10C4700062F03DEF62F032EF62F0D8900F36103686
:10C480000B50095C0C500A58D8A049EF62F04BEFF2
:10C4900062F050EF62F00B50095E0C500A5A0F80A8
:10C4A000D8900C320B320D2E3DEF62F00E50D8B406
:10C4B0005CEF62F05EEF62F062EF62F00F6C101EF4
:10C4C000D8B0102A0FC509F510C50AF51200000EE4
:10C4D0005624D96EDA6A090EDA22DF6A0201B2A79F
:10C4E00074EF62F076EF62F08AEF62F0000E56248D
:10C4F000D96EDA6A090EDA22DF8202D88AEF62F098
:10C500000500FA6E0701F251FD6EF351FE6EFF6AEF
:10C51000FA5012000201B2A390EF62F092EF62F0C3
:10C52000A6EF62F0000E5624D96EDA6A090EDA22FE
:10C53000DF8402D8A6EF62F00500FA6E0701F05121
:10C54000FD6EF151FE6EFF6AFA501200000E562485
:10C55000D96EDA6A090EDA22DF50D8B4B2EF62F08F
:10C56000B4EF62F0C3EF62F002D8C1EF62F00500F1
:10C57000FA6E0701EE51FD6EEF51FE6EFF6AFA5042
:10C580001200C5EF62F0FBEC6FF012001F6A1C0492
:10C59000D8A4CDEF62F0CFEF62F0D3EF62F0040EDB
:10C5A0001F6EF9EF62F0020E1C18D8A4DAEF62F0E9
:10C5B000DCEF62F0E0EF62F0080E1F6EF9EF62F060
:10C5C000030E1C18D8A4E7EF62F0E9EF62F0F9EF70
:10C5D00062F0100E1F6EF9EF62F0040E206E12EF83
:10C5E00063F0330E206E12EF63F0020E206E12EF36
:10C5F00063F01C501D6E1E6A1E50000AD8B403EF73
:10C6000063F01DEF63F01D50010AD8B4EDEF62F046
:10C61000030AD8B4F1EF62F0010AD8B4F5EF62F082
:10C620001DEF63F020C509F5060E0A6E1AC50BF55D
:10C630001BC50CF51F501DEC45F012000E6A0ABE1A
:10C6400026EF63F024EF63F02CEF63F0096C0A1E11
:10C65000D8B00A2A010E0E6E0CBE33EF63F031EF34
:10C6600063F037EF63F00B6C0C1ED8B00C2A0B5044
:10C670000C10D8B43EEF63F040EF63F064EF63F06A
:10C68000010E0D6E48EF63F0D8900B360C360D2A74
:10C690000CAE4DEF63F04FEF63F044EF63F00B50DF
:10C6A000095C0C500A58D8A058EF63F05AEF63F0B9
:10C6B0005EEF63F00B50095E0C500A5AD8900C32B2
:10C6C0000B320D2E4FEF63F00E50D8B46AEF63F0CB
:10C6D0006CEF63F070EF63F0096C0A1ED8B00A2AA1
:10C6E00009C509F50AC50AF512005450D8B47BEF04
:10C6F00063F07DEF63F081EF63F0020E136E83EF62
:10C7000063F0040E136E146AC0EF63F0DB0E1424A2
:10C71000D96EDA6A060EDA22DF50126E0A6A870EC6
:10C72000096E1428BCEC59F009C510F50AC511F5BD
:10C73000DB0E1424D96EDA6A060EDA221050070BCB
:10C74000DF6EDB0E1424D96EDA6A060EDA2212507E
:10C75000DE18D8B4AEEF63F0B0EF63F0BFEF63F074
:10C7600014C50EF5010E0F6E0E2AB9EF63F0D890C6
:10C770000F360E2EB7EF63F00F5006019513142AF3
:10C780001350145CD8A0C7EF63F0C9EF63F086EFD5
:10C7900063F006018E9B1200000E0914116E000E4C
:10C7A0000A14126E800E0B14136E7F0E0C14146E8E
:10C7B0001150121013101410D8A4E1EF63F0E3EF3E
:10C7C00063F0EBEF63F0000E096E000E0A6E000ED0
:10C7D0000B6E000E0C6E000E0D14116E000E0E147A
:10C7E000126E800E0F14136E7F0E1014146E115003
:10C7F000121013101410D8A400EF64F002EF64F0CC
:10C800000AEF64F0000E0D6E000E0E6E000E0F6E3D
:10C81000000E106E0D5009180FE10E500A180CE1B1
:10C820000F500B1809E110500C18D8B41AEF64F02F
:10C830001CEF64F01FEF64F0D89020EF64F0D88014
:10C8400012007B7C7D7E7F807B7C7D7E0000800073
:10C85000800040002000106E20202020202020207A
:10C86000006E2020202020202020006E53444934D8
:10C87000204F7574006E5344493320496E20006E7A
:10C880002B202020202020006E4E6F4C6F636B0009
:10C890006E4E6F4C6F636B006E4E6F4C6F636B0030
:10C8A0006E4E6F4C6F636B006E5365632049500092
:10C8B0006E507269204950006E4243383830006E25
:10C8C00020202020006E20202020006E54656D70F6
:10C8D000006E486F7374006E312E3533006E322E49
:10C8E0003030006E4D414300060190A37AEF64F0B2
:10C8F0007CEF64F07EEF64F0C5EF64F0F7C628F5D6
:10C90000F8C629F5F793F89799A189EF64F08BEFB2
:10C9100064F08FEF64F0F78DF79F91EF64F0F79D6F
:10C92000F78F9AA196EF64F098EF64F09CEF64F0B3
:10C93000F881F8939EEF64F0F883F891F751281886
:10C9400009E1F8512918D8B4A8EF64F0AAEF64F00F
:10C95000B3EF64F0020E206EF7C621F5F8C622F59B
:10C96000200E55EC69F0CFB0B8EF64F0BAEF64F088
:10C97000C3EF64F0000E206E200E48EC66F020C578
:10C98000F9F621C5FAF606018E931200000E1D6E0F
:10C99000150E1E6E000E12141F6EFF0E1314206E65
:10C9A000000E1414216E000E1514226E12C518F517
:10C9B00013C519F514C51AF515C51BF5D8901B320A
:10C9C0001A321932183218507F0B1C6E1FC509F528
:10C9D00020C50AF521C50BF522C50CF537EC6DF025
:10C9E0001FC509F520C50AF521C50BF522C50CF5B3
:10C9F000F6EC6AF01C50186E196AD8901836193681
:10CA000018501D2619501E221DC5D9F41EC5DAF472
:10CA100016C5DEF417C5DDF41FC509F520C50AF5F6
:10CA200021C50BF522C50CF512EC6DF012000701C3
:10CA3000C9893BEF65F005EC72F0080E67EF65F011
:10CA400005EC72F0070E67EF65F00701C529E6EC0B
:10CA500071F0040E67EF65F0070E0701C719D8B42F
:10CA600034EF65F036EF65F038EF65F008EC72F002
:10CA70000F0E67EF65F0B2C712F5B3C713F502D812
:10CA80004BEF65F00500FA6EA651FD6EA751FE6EE4
:10CA9000FF6AFA501200146E156A1550000AD8B4D5
:10CAA00054EF65F02CEF65F01450010AD8B42CEF68
:10CAB00065F0030AD8B420EF65F0010AD8B41BEF83
:10CAC00065F0070AD8B425EF65F02CEF65F0120089
:10CAD0006E327831324720456E636170202B2032F0
:10CAE00078313247204465636170006E2020202039
:10CAF00020202020202020202020202020006E2008
:10CB00002020202020202020202020202020200045
:10CB10006E202020202020202020202020202020C7
:10CB2000006E2020202020202020202020202020D7
:10CB300020006E536563204C696E6B006E50726905
:10CB4000204C696E6B006E53444932204F7574005F
:10CB50006E5344493120496E20006E536563204670
:10CB60004543006E507269204645430034EC71F035
:10CB70000009D8A4BEEF65F0C0EF65F0C3EF65F023
:10CB8000040E00EF66F00701C951030B0009D8B489
:10CB9000CCEF65F0CEEF65F0DAEF65F0010E166EC2
:10CBA000C951030B176E1650175EC9511718FC0BAD
:10CBB0001718C96FC507D8A0C607C551C611D8B484
:10CBC000E4EF65F0E6EF65F0F2EF65F002EC72F08D
:10CBD000C3C7D9F4C4C7DAF4DF6E0701C34BC42B53
:10CBE000C0EF65F017EC65F0186E02EC72F0C3C789
:10CBF000D9F4C4C7DAF4DF6E0701C34BC42B185055
:10CC00001200096E010E0A6E0701C9B70AEF66F03D
:10CC10000CEF66F046EF66F009C5C2F7C995C98703
:10CC2000FC0EC9170F0EC76F010EC16FF40EC06F57
:10CC3000C989400EA66FE40EA76F000EB26F000EFA
:10CC4000B36F400EA86FE40EA96F000EB46F000E14
:10CC5000B56F400EAA6FE40EAB6F000EB66F000EFC
:10CC6000B76F400EAC6FE40EAD6F000EB86F000EE4
:10CC7000B96F3C0EAE6FE40EAF6F000EBA6F000ED0
:10CC8000BB6F14EC72F04BEC70F00A6A0A501200A1
:10CC9000256E276A000E266E255001EC66F000090D
:10CCA000D8B455EF66F057EF66F04CEF66F0780EAB
:10CCB0000E6EDF0E0F6E260E106E050E116EF0EC6E
:10CCC00070F0200E096E050E0A6E0C6A010E0B6ED6
:10CCD0005DEC70F0000E0E6E000E0F6E000E106E0A
:10CCE000000E116EE4EC70F0D2EC71F091EC6FF08C
:10CCF000E806D8B47EEF66F080EF66F076EF66F077
:10CD000027C522F52650236E2250206E23C521F51B
:10CD100012001EBE90EF66F08EEF66F093EF66F0A5
:10CD20001E6A000E1D6E216A000E206EA3EF66F0D3
:10CD30000A6A200E096E19C50BF51AC50CF5A2EC8E
:10CD400061F0204A212A1D50205C2150800A1F6E6C
:10CD50001E50800A1F58D8A0B0EF66F0B2EF66F000
:10CD600098EF66F01BC512F51CC513F519C514F52F
:10CD70001AC515F5A1EC6DF01BC509F51CC50AF522
:10CD800028EC6CF01D500924196E1E500A201A6EF2
:10CD90001200116A0E6A000E0D6EFBEF66F00D5068
:10CDA0000924D96E0E500A20DA6EDF50111A106A6B
:10CDB000000E0F6E11AEDFEF66F0E1EF66F0E7EF09
:10CDC00066F0115011248C0A116EE9EF66F0D890CC
:10CDD00011360F4A102A10BEF7EF66F0105009E125
:10CDE000080E0F5CD8A0F7EF66F0F9EF66F0DAEF07
:10CDF00066F00D4A0E2A0B500D5C0C500E58D8A050
:10CE000004EF67F006EF67F0CFEF66F01150120005
:10CE1000A290CE0E096EC40E0A6EA6EC71F0A2921C
:10CE2000FE0E096EDA0E0A6EA1EC71F00201A56B1E
:10CE3000A66BA76BA86BA96BAA6BB00EAB6F800E2D
:10CE4000AC6FAD6B8A0EAE6FAF6BB06BB16BB26B8C
:10CE5000B36B480E096EE40E0A6EB0EC71F0460E2C
:10CE6000096EE40E0A6EABEC71F02E0E096EE40E44
:10CE70000A6EB5EC71F00601DA6B0501FC6BFB6B19
:10CE8000400E576E566A556AFA6BA2801200256EE4
:10CE900021C528F522C529F523C526F524C527F582
:10CEA000255001EC66F00009D8B459EF67F05BEF4C
:10CEB00067F050EF67F0C60E0E6EDB0E0F6E260E9B
:10CEC000106E050E116EF0EC70F0200E096E050E5E
:10CED0000A6E0C6A010E0B6E5DEC70F0000E0E6EA9
:10CEE000000E0F6E000E106E000E116EE4EC70F06E
:10CEF000D2EC71F091EC6FF0E806D8B482EF67F0F5
:10CF000084EF67F07AEF67F012000701C9899AEFA2
:10CF100067F005EC72F0070EC2EF67F00701C52954
:10CF2000E6EC71F0030EC2EF67F008EC72F00A0E47
:10CF3000C2EF67F0B2C712F5B3C713F502D8AAEF74
:10CF400067F00500FA6EA651FD6EA751FE6EFF6AEE
:10CF5000FA501200146E156A1550000AD8B4B3EFD7
:10CF600067F095EF67F01450010AD8B495EF67F0B9
:10CF7000030AD8B489EF67F0060AD8B48EEF67F0D9
:10CF800095EF67F01200E4EF67F008EC71F000092C
:10CF9000D8B4CDEF67F0CFEF67F0C5EF67F00AC503
:10CFA000F6F40BC5F7F4000EF86E150EF76403D017
:10CFB0000800F55005D0F6C4E9F4F7C4EAF4EF50E0
:10CFC000AAEC6BF00A4A0B2A0AC5F6F40BC5F7F473
:10CFD000000EF86E150EF76403D00800F55005D06A
:10CFE000F6C4E9F4F7C4EAF4EF500009D8A4FBEF63
:10CFF00067F0FDEF67F0C5EF67F01200FFEC6BF034
:10D000000701C951030B0009D8B409EF68F00BEF11
:10D0100068F018EF68F029EC71F00009D8B413EF4C
:10D0200068F015EF68F018EF68F0100E0701C76F91
:10D030000701C751020D070EF324F66E310EF420DE
:10D04000F76EF86A000EF8220900F5C41CF5090015
:10D05000F5C41DF502D836EF68F00500FA6E1C50D5
:10D06000FD6E1D50FE6EFF6AFA5012000701C76F79
:10D0700012000D6E09500A10D8B441EF68F043EF6A
:10D0800068F05DEF68F00D50020DA60EF324D96E26
:10D09000070EF420DA6E09C5DEF40AC5DDF40D5082
:10D0A000020DB20EF324D96E070EF420DA6E0BC512
:10D0B000DEF40CC5DDF473EF68F00D50020DA60E22
:10D0C000F324D96E070EF420DA6E400EDE6EE40E05
:10D0D000DD6E0D50020DB20EF324D96E070EF42052
:10D0E000DA6EDE6ADD6A12000E6A000E0D6E0B50FB
:10D0F0000C10D8B47EEF68F080EF68F0A8EF68F00D
:10D10000010E0F6E88EF68F0D8900B360C360F2AA0
:10D110000CAE8DEF68F08FEF68F084EF68F0D89078
:10D120000D360E360B50095C0C500A58D8A09BEFF8
:10D1300068F09DEF68F0A2EF68F00B50095E0C50AC
:10D140000A5A0D80D8900C320B320F2E8FEF68F0F8
:10D150000DC509F50EC50AF512000601D22B3C0ECD
:10D16000D219D8A4B6EF68F0B8EF68F0DBEF68F03A
:10D17000D26BD32B180ED319D8A4C1EF68F0C3EF2C
:10D1800068F0D4EF68F0D36BC24BC32B0A6AE10E90
:10D19000096EC3510B6E9FEC6CF00A6AE20E096EC9
:10D1A000C2C60BF59FEC6CF00A6AE30E096ED3C69B
:10D1B0000BF59FEC6CF00A6AE40E096ED2C60BF513
:10D1C0009FEC6CF006018E9D1200216E226A2150A8
:10D1D00001EC66F00009D8B4F0EF68F0F2EF68F007
:10D1E000E7EF68F0A20E0E6EDF0E0F6E220E106ECD
:10D1F000050E116EF0EC70F0200E096E050E0A6E31
:10D200000C6A010E0B6E5DEC70F0000E0E6E000EDF
:10D210000F6E000E106E000E116EE4EC70F0D2EC8A
:10D2200071F091EC6FF0E806D8B419EF69F01BEFDC
:10D2300069F011EF69F02250120014EC72F0020E46
:10D240000701C86F30EF69F094EC71F054EF69F0AA
:10D250001CEC72F054EF69F086EC71F054EF69F059
:10D26000B4C712F5B5C713F502D840EF69F0050051
:10D27000FA6EA851FD6EA951FE6EFF6AFA501200B7
:10D28000166E176A1750000AD8B449EF69F02CEFF0
:10D2900069F01650020AD8B424EF69F0010AD8B434
:10D2A00028EF69F02CEF69F01200236E235001EC97
:10D2B00066F00009D8B45FEF69F061EF69F056EFEE
:10D2C00069F0CC0E0E6EDF0E0F6E210E106E050E85
:10D2D000116EF0EC70F0200E096E050E0A6E0C6AED
:10D2E000010E0B6E5DEC70F0000E0E6E000E0F6EF8
:10D2F000000E106E000E116EE4EC70F0D2EC71F0C6
:10D3000091EC6FF0E806D8B488EF69F08AEF69F025
:10D3100080EF69F01200226E225001EC66F00009E5
:10D32000D8B495EF69F097EF69F08CEF69F04E0E85
:10D330000E6EDF0E0F6E210E106E050E116EF0ECEC
:10D3400070F0200E096E050E0A6E0C6A010E0B6E4F
:10D350005DEC70F0000E0E6E000E0F6E000E106E83
:10D36000000E116EE4EC70F0D2EC71F091EC6FF005
:10D37000E806D8B4BEEF69F0C0EF69F0B6EF69F027
:10D380001200B7C5BBF5B8C5BCF50601B56B000EFC
:10D39000B46FE2EF69F0B5C5A3F5B6C5A4F5BB0E51
:10D3A0000501A56F050EA66FB9C5A7F5BAC5A8F505
:10D3B0002EEC47F00501A3510601B4270501A45145
:10D3C0000601B523BBC5F6F4BCC5F7F4F86A08003E
:10D3D000F5500009D8A4EFEF69F0F1EF69F0CBEF59
:10D3E00069F0B4C6B5F5B5C6B6F512000FC516F5A9
:10D3F00010C517F50DC514F50EC515F51CEF6AF02F
:10D4000016C5F6F417C5F7F4000EF86E150EF7649E
:10D4100003D00800F55005D0F6C4E9F4F7C4EAF4E7
:10D42000EF50136E164A172A14C5D9F415C5DAF44D
:10D4300013C5DFF4144A152A1106D8A012061128C4
:10D4400006E11228D8A427EF6AF029EF6AF000EF6E
:10D450006AF01200FC0E0701C917020EC86FC995C9
:10D4600039EF6AF01AEC72F05DEF6AF00F0E5DEFC3
:10D470006AF0B6C712F5B7C713F502D849EF6AF0DC
:10D480000500FA6EAA51FD6EAB51FE6EFF6AFA50AE
:10D490001200146E156A1550000AD8B452EF6AF0E3
:10D4A00036EF6AF01450020AD8B432EF6AF0010A7B
:10D4B000D8B432EF6AF036EF6AF01200C0BA63EF08
:10D4C0006AF066EF6AF0010E67EF6AF0000EFF0A7D
:10D4D000056E053A0546C0500518DF0B0518C06EED
:10D4E0000601D12B3A0E8E137EEF6AF08E8191EFFA
:10D4F0006AF0410E8E13D16B91EF6AF0D1510F0A91
:10D50000D8B476EF6AF0110AD8B476EF6AF0330A2D
:10D51000D8B476EF6AF0110AD8B479EF6AF091EFD7
:10D520006AF01200800EBE6EBF6AC06A390EC66E07
:10D53000C768800EC86E0401106B3E0E086F006B4A
:10D54000216B096B016B116B0201896B886B876B17
:10D55000866B0401226B026B0A6B180E126F036953
:10D560000B69136904690C691469080E246F140EA1
:10D570000201706F370E146F380E156F200E176F83
:10D58000170E726F130E716F12000B6A000E0A6E87
:10D59000CEBACDEF6AF0CFEF6AF0E2EF6AF0E5EFD6
:10D5A0006AF0350EE82EFED700000A4A0B2A200E3C
:10D5B0000A5C4E0E0B58D8A0E0EF6AF0E2EF6AF07A
:10D5C000E5EF6AF0000EF5EF6AF0CEAAEAEF6AF036
:10D5D000ECEF6AF0D1EF6AF0680E096EE40EE82E07
:10D5E000FED7092EFCD700D0010E1200000E091440
:10D5F0000E6EFF0E0A140F6E000E0B14106E000E4E
:10D600000C14116E000ED6BE010E0D6E10C545F045
:10D610000FC544F000014151F80B0609416FD69E39
:10D62000550E426FAA0E426F408140B11AEF6BF067
:10D630001CEF6BF015EF6BF00DB002D0D69E01D051
:10D64000D68EF80E000141171200246E245001EC12
:10D6500066F00009D8B42FEF6BF031EF6BF026EFD6
:10D660006BF020C509F521C50AF522C50BF523C5C8
:10D670000CF55DEC70F0000E0E6E000E0F6E000EDD
:10D68000106E000E116EE4EC70F0D2EC71F091ECC3
:10D690006FF0E806D8B44FEF6BF051EF6BF047EF47
:10D6A0006BF01200B5A257EF6BF059EF6BF05BEF28
:10D6B0006BF07EEF6BF0B5A060EF6BF062EF6BF09C
:10D6C00064EF6BF07EEF6BF002019AA56AEF6BF0EE
:10D6D0006CEF6BF06EEF6BF07EEF6BF09AAF73EF69
:10D6E0006BF075EF6BF077EF6BF07EEF6BF097A957
:10D6F0007CEF6BF07EEF6BF052EF6BF012000CBE24
:10D7000084EF6BF086EF6BF090EF6BF009C509F5D5
:10D710000AC50AF50BC50BF50CC50CF5A9EF6BF0A6
:10D7200009C50DF50AC50EF50BC50FF50CC510F5AD
:10D730000D1E0E1E0F1E101E0D2A000E0E220F2291
:10D7400010220DC509F50EC50AF50FC50BF510C55C
:10D750000CF51200096E5750D8B4B1EF6BF0B3EF6F
:10D760006BF0ABEF6BF0A2B2B8EF6BF0BAEF6BF00F
:10D77000BEEF6BF009C5A3F2D3EF6BF0A292400E9F
:10D780000501FC25D96EDA6A0A0EDA2209C5DFF432
:10D79000FC2B3F0EFC65CFEF6BF0D1EF6BF0D2EFBF
:10D7A0006BF0FC6B5706A28212000501FA51D8B447
:10D7B000DCEF6BF0DEEF6BF0D5EF6BF0000E552475
:10D7C000D96EDA6A090EDA22DF500601DA6F000E2E
:10D7D0005524D96EDA6A0A0EDA22DF50096E552A0C
:10D7E0003F0E5564F6EF6BF0F8EF6BF0F9EF6BF06E
:10D7F000556AA2900501FA07A2800950120055EC63
:10D8000071F00009D8B407EF6CF009EF6CF00DEF80
:10D810006CF011EC72F027EF6CF03FEC71F0000946
:10D82000D8B415EF6CF017EF6CF01BEF6CF00BEC4D
:10D8300072F027EF6CF04AEC71F00009D8B423EFD6
:10D840006CF025EF6CF027EF6CF00EEC72F012002C
:10D8500009C50BF50AC50CF530EF6CF0094A0A2A28
:10D8600009C5F6F40AC5F7F4000EF86E150EF76454
:10D8700003D00800F55005D0F6C4E9F4F7C4EAF483
:10D88000EF500009D8A447EF6CF049EF6CF02EEF91
:10D890006CF00B50095C096E0C500A580A6E1200AD
:10D8A0001E6E010E1F6E0701C9B559EF6CF05BEFDC
:10D8B0006CF076EF6CF0C9851F6AC551E6EC71F02B
:10D8C0001E50D8B466EF6CF068EF6CF06FEF6CF040
:10D8D000040E0701C76F64EC6FF074EF6CF0030E79
:10D8E0000701C76F13EC71F09FEC70F01F5012002E
:10D8F0000501F56B000EF46F0A6A000E096E400E0A
:10D900000924D96E090E0A20DA6EDF6A094A0A2A4A
:10D910000A5009E1800E095CD8A091EF6CF093EFFA
:10D920006CF07FEF6CF00601CC6BCB6BCA6B050122
:10D93000F76BF66B0601C96BC86BC76B1200000E64
:10D94000D6BE010E0C6E380E0001456F0A50446FB2
:10D9500009C543F00BC546F04151F80B0309416F6F
:10D96000D69E550E426FAA0E426F408140B1BBEF6A
:10D970006CF0BDEF6CF0B6EF6CF00CB002D0D69E40
:10D9800001D0D68EF80E000141171200C10E05011C
:10D99000C56F050EC66FBDC5C7F5BEC5C8F5CA6B58
:10D9A000000EC96FD16B000ED06FC70EB56F050E9C
:10D9B000B66FBFC5B7F5C0C5B8F5C50EB96F050ED2
:10D9C000BA6FC1EC69F00501C951BD25D96ECA51C4
:10D9D000BE21DA6EDF6A1200FAC407F5FBC408F54F
:10D9E000B198C4C605F5C5C606F510EC70F0070180
:10D9F000EC51ED11D8B4FFEF6CF001EF6DF00DEFCD
:10DA00006DF002D80DEF6DF00500FA6EEC51FD6E71
:10DA1000ED51FE6EFF6AFA50120008C5FBF407C50F
:10DA2000FAF41100000ED6BE010E0D6E0BC545F0C6
:10DA30000AC544F009C543F000014151F80B05093E
:10DA4000416FD69E550E426FAA0E426F408140B183
:10DA50002CEF6DF02EEF6DF027EF6DF00DB002D0D2
:10DA6000D69E01D0D68EF80E000141171200000E8E
:10DA7000D6BE010E0D6E0BC545F00AC544F009C5B2
:10DA800043F000014151F80B0209416FD69E550E3B
:10DA9000426FAA0E426F408140B151EF6DF053EFDB
:10DAA0006DF04CEF6DF00DB002D0D69E01D0D68E49
:10DAB000F80E000141171200000E341A000E351A3C
:10DAC000000E361A800E371A30C509F531C50AF531
:10DAD00032C50BF533C50CF534C50DF535C50EF55E
:10DAE00036C50FF537C510F55BEC3EF009C530F5CE
:10DAF0000AC531F50BC532F50CC533F51200400EE1
:10DB0000576085EF6DF087EF6DF09FEF6DF0400E81
:10DB10000501FB25D96EDA6A0A0EDA22DF5002010E
:10DB2000A36F0501FB2B3F0EFB6599EF6DF09BEF9B
:10DB30006DF09CEF6DF0FB6B572AA0EF6DF0A29299
:10DB40001200186A000E176EB1EF6DF016C509F5D8
:10DB50000A6A14C50BF515C50CF5A2EC61F0174A5D
:10DB6000182A17501224D96E18501320DA6EDF507D
:10DB7000166E1650D8A4BFEF6DF0C1EF6DF0A6EF92
:10DB80006DF0120003011F6B206B060E216F850ED6
:10DB90001D6FEE0E1C6FB1981C511DC30BF50C6A66
:10DBA0000BC50CF50B6A0B100601C46F0C50C56F4A
:10DBB000A1884A0E096EE40E0A6EBAEC71F0010EED
:10DBC00003011E6F120020EE02F01250D9261350EE
:10DBD000DA22DEC409F5DDC40AF512C5D9F413C58D
:10DBE000DAF4DEC40BF5DDC40CF55DEC70F0000E6C
:10DBF0000E6E000E0F6E000E106E000E116EF0EC29
:10DC000070F0020E1200FFFFFAC401F5FBC402F52A
:10DC10000701F451F511D8B410EF6EF012EF6EF069
:10DC20001EEF6EF002D81EEF6EF00500FA6EF45192
:10DC3000FD6EF551FE6EFF6AFA50120002C5FBF44C
:10DC400001C5FAF41100FFFFFAC403F5FBC404F5A3
:10DC50000701F651F711D8B430EF6EF032EF6EF0E5
:10DC60003EEF6EF002D83EEF6EF00500FA6EF65110
:10DC7000FD6EF751FE6EFF6AFA50120004C5FBF408
:10DC800003C5FAF4110009C50DF50AC50EF50BC55B
:10DC9000F6F40CC5F7F40B4A0C2AF86A0DC5D9F452
:10DCA0000EC5DAF40D4A0E2A0800F5C4DFF4DF5081
:10DCB000D8A45DEF6EF05FEF6EF047EF6EF01200EC
:10DCC00009500A100B100C10D8B469EF6EF06BEF0E
:10DCD0006EF073EF6EF0000E091A000E0A1A000EB5
:10DCE0000B1A800E0C1A09C509F50AC50AF50BC5F1
:10DCF0000BF50CC50CF512000B6E0B3A0F0E0B1644
:10DD00000A0E0B6086EF6EF088EF6EF090EF6EF00B
:10DD1000300E0B24096E0A6A000E0A2296EF6EF08E
:10DD2000370E0B24096E0A6A000E0A2209501200EF
:10DD3000256A000E246E150E2412540E2512060EAE
:10DD4000206E24C521F525C522F5200E55EC69F07D
:10DD5000241E251E4A0E206E24C521F525C522F558
:10DD6000200E55EC69F012000B6E0F0E0B160A0E0A
:10DD70000B60BDEF6EF0BFEF6EF0C7EF6EF0300ED0
:10DD80000B24096E0A6A000E0A22CDEF6EF0370EE0
:10DD90000B24096E0A6A000E0A22095012000301C0
:10DDA000D96BDA6BDB6BDC6BDF6BE06BE56BE76B26
:10DDB000EC6BEE6BEF6BF06BF16BF26BF46B100EC8
:10DDC000F56FF66BF76BF86BF96B2F0EFA6F840E2D
:10DDD000F36F120010BEEFEF6EF0F1EF6EF0F7EFA1
:10DDE0006EF00FC50FF510C510F503EF6FF00FC5FE
:10DDF00011F510C512F5111E121E114A122A11C575
:10DE00000FF512C510F512000D507CEC6EF00E6E81
:10DE10000D50B4EC6EF00F6E0C507CEC6EF0106E8A
:10DE20000C50B4EC6EF0116E126A0E0E0A6E050EF6
:10DE30000B6EC3EC67F01200DFC5BDF5E0C5BEF5A3
:10DE4000E1C5BFF5E2C5C0F5550E0501C16F390E3C
:10DE5000C26FDBC5C3F5DCC5C4F5DDC5C5F5DEC5E0
:10DE6000C6F549EC5FF01200D68AD69E550E040125
:10DE7000596FAA0E596F59915F6B300E5E6F080E85
:10DE80005D6F550E596FAA0E596F5981D68E0301D9
:10DE900066836681658912000D6E0DC5ECF3030182
:10DEA000F38FF39DF381F3B158EF6FF05AEF6FF0FA
:10DEB00053EF6FF0EB510C6E0B6AEA510B24096EB5
:10DEC000000E0C200A6E12000701C951FC0B02095A
:10DED000C96FC505C611D8A470EF6FF072EF6FF06F
:10DEE00074EF6FF017EC65F0D8800701C235E2ECF3
:10DEF00071F0040E120034EC6FF06AEC71F0BCECBF
:10DF000070F074EC71F092EC6AF09BEC71F0CEEC76
:10DF100071F0CFEC6EF0C2EC6DF008EC67F0D68ECD
:10DF20001200010E096E0701C9B599EF6FF09BEF62
:10DF30006FF0A5EF6FF0C997C26914EC72F0CAECEC
:10DF400070F0C9EC71F0C8C709F50950120012C58C
:10DF500009F513C50AF50C6A010E0B6E5DEC70F045
:10DF6000000E0E6E000E0F6E000E106E000E116E83
:10DF7000F0EC70F0040E120012C509F513C50AF595
:10DF80000C6A020E0B6E5DEC70F0000E0E6E000E51
:10DF90000F6E000E106E000E116EF0EC70F0020E9F
:10DFA000120012C509F513C50AF50C6A010E0B6EB5
:10DFB0005DEC70F0000E0E6E000E0F6E000E106E17
:10DFC000000E116EF0EC70F0020E120012C509F591
:10DFD00013C50AF50C6A020E0B6E5DEC70F0000EB4
:10DFE0000E6E000E0F6E000E106E000E116EF0EC35
:10DFF00070F0040E1200000E5624D96EDA6A0A0E72
:10E00000DA22A1C2DFF4562A3F0E56640AEF70F0FE
:10E010000CEF70F00DEF70F0566A0501FA2B12004C
:10E0200003011EA516EF70F018EF70F020EF70F0EE
:10E030001E9106501D6F05C51CF31E8124EF70F064
:10E0400006501D6F05C51CF31200F9EC71F0F6ECDB
:10E0500071F00009D8B42FEF70F031EF70F037EFA6
:10E0600070F0000EE6EC71F0000EE2EC71F0000EC4
:10E0700012000808080800080004000200018000DF
:10E080004000200010000800040002000100FFFF13
:10E09000FFFF01010101020194BF51EF70F053EF46
:10E0A00070F05CEF70F09A6B9B6B976B8D69510E03
:10E0B000876F510E866F948F12000701C9A963EF15
:10E0C00070F065EF70F06EEF70F009C5C3F70AC528
:10E0D000C4F70BC5C5F70CC5C6F7C9991200136E76
:10E0E00013507CEC6EF00C6E1350B4EC6EF00D6EB1
:10E0F0000E6A0C0E0A6E050E0B6EC3EC67F0120072
:10E10000090680184000601A090680184000601A4D
:10E11000090680184000601A090680184000601A3D
:10E120000A6E08EC71F00009D8B499EF70F09BEF1B
:10E1300070F091EF70F00A50AAEC6BF01200A5EFAE
:10E1400070F052EC6BF0FEEC67F00701C9B5ABEF75
:10E1500070F0ADEF70F0A1EF70F01200000ED6BEBF
:10E16000010E096ED69E00017851040009B002D05C
:10E17000D69E01D0D68E1200040E0201946F800E3E
:10E18000956F180E966F030E9C6F9A6B9B6B976B37
:10E190008D691200A594A596A590A59202019B9168
:10E1A0009B959B9F9B9D9B9397939795979112000F
:10E1B0000501FA51D8A4DFEF70F0E2EF70F0010E24
:10E1C000E3EF70F0000E12000EC509F50FC50AF559
:10E1D00010C50BF511C50CF5020E39EC68F01200F4
:10E1E0000EC509F50FC50AF510C50BF511C50CF5DF
:10E1F000000E39EC68F01200380E0001456F0A502D
:10E20000446F09C543F0F80E411740814651120092
:10E210005750D8A40EEF71F011EF71F0010E12EF0C
:10E2200071F0000E12000701C951FC0B0209C96F01
:10E23000C251C225E2EC71F0030E1200020199BB3B
:10E2400024EF71F027EF71F0010E28EF71F0000E4E
:10E250001200020195BB2FEF71F032EF71F0010E49
:10E2600033EF71F0000E1200020199B13AEF71F034
:10E270003DEF71F0010E3EEF71F0000E1200020151
:10E280009AB545EF71F048EF71F0010E49EF71F06A
:10E29000000E1200020197B950EF71F053EF71F0C8
:10E2A000010E54EF71F0000E120002019ABF5BEFF5
:10E2B00071F05EEF71F0010E5FEF71F0000E120071
:10E2C000F0B865EF71F068EF71F0010E69EF71F071
:10E2D000000E12000001606B616B636B646B656B19
:10E2E000666B676B686B1200600E0001AD6FAF6B01
:10E2F000B36B080EB16FB06BAC6B1200C4EC71F075
:10E300000701C995020EC86F0F0E1200C4EC71F020
:10E310000701C995C86B0F0E1200FCEC71F0F9EC07
:10E3200071F0BFEC71F012000701C551E6EC71F01D
:10E3300064EC6FF012001A0E0001786F170E796FFF
:10E34000120009C5F4F70AC5F5F7120009C5F6F77A
:10E350000AC5F7F7120009C5F0F70AC5F1F7120070
:10E3600009C5F2F70AC5F3F7120009C5EEF70AC5A9
:10E37000EFF7120009C5ECF70AC5EDF71200070127
:10E38000C995C86B0F0E12000201949F9985948F56
:10E3900012000201949F9A6B99851200820E03016C
:10E3A000D76F1200000E50EC6CF01200FCEC71F014
:10E3B000090E1200FFEC71F0040E1200FFEC71F078
:10E3C000030E1200096E09C58CF21200096E09C510
:10E3D0008DF2120000017881120000017891120084
:10E3E00003011E91120003011E81120002018D51D2
:10E3F00012000201949B12000201958D120002018D
:10E40000959D120002018B5112000201948D1200A1
:10E410000201949D120002019A951200020197993F
:10E42000120002019A9F120002019A6B1200FBEC8B
:10E430006FF01200010E1200020E1200050E120003
:10E44000010E12001200120012001200110001FF52
:10E45000FFFFFFFFFFFFFFFFFFFFFFFFFFFFFFFFCC
:10E46000FFFFFFFFFFFFFFFFFFFFFFFFFFFFFFFFBC
:10E47000FFFFFFFFFFFFFFFFFFFFFFFFFFFFFFFFAC
:10E48000FFFFFFFFFFFFFFFFFFFFFFFFFFFFFFFF9C
:10FFF000FFFFFFFFFFFFFFFFFFFFFFFFFFFF497A4C
:020000040020DA
:10000000FFFFFFFFFFFFFFFFFFFFFFFFFFFFFFFF00
:10001000FFFFFFFFFFFFFFFFFFFFFFFFFFFFFFFFF0
:10002000FFFFFFFFFFFFFFFFFFFFFFFFFFFFFFFFE0
:10003000FFFFFFFFFFFFFFFFFFFFFFFFFFFFFFFFD0
:020000040030CA
:080000008CFFEFFFADCFFFFF05
:01000900FFF7
:00000001FF
